:04000003F000B45500
:020000040000FA
:1000000000040020810A000015070000610A0000BA
:100010001F07000029070000330700000000000050
:10002000000000000000000000000000A50A000021
:100030003D070000000000004707000051070000D6
:100040005B070000650700006F07000079070000EC
:10005000830700008D07000097070000A10700003C
:10006000AB070000B5070000BF070000C90700008C
:10007000D3070000DD070000E7070000F1070000DC
:10008000FB070000050800000F0800001908000029
:10009000230800002D080000370800004108000078
:1000A0004B080000550800005F08000069080000C8
:1000B000730800007D080000870800009108000018
:1000C0009B080000A5080000AF080000B908000068
:1000D000C3080000CD080000D7080000E1080000B8
:1000E000EB080000F5080000FF0800000909000007
:1000F000130900001D090000270900003109000054
:100100003B0900001FB500F003F88DE80F001FBD8C
:1001100000F0ACBC40F6FC7108684FF01022401CA7
:1001200008D00868401C09D00868401C04D0086842
:1001300000F037BA9069F5E79069F9E7704770B554
:100140000B46010B184400F6FF70040B4FF0805073
:100150000022090303692403406943431D1B104621
:1001600000F048FA29462046BDE8704000F042BA47
:10017000F0B54FF6FF734FF4B4751A466E1E11E0DA
:10018000A94201D3344600E00C46091B30F8027B3B
:10019000641E3B441A44F9D19CB204EB134394B25D
:1001A00004EB12420029EBD198B200EB134002EBB2
:1001B000124140EA0140F0BDF34992B00446D1E952
:1001C0000001CDE91001FF224021684600F0F4FB58
:1001D00094E80F008DE80F00684610A902E004C8FB
:1001E00041F8042D8842FAD110216846FFF7C0FF7C
:1001F0001090AA208DF8440000F099F9FFF78AFFCB
:1002000040F6FC7420684FF01025401C0FD0206889
:1002100010226946803000F078F92068401C08D030
:100220002068082210A900F070F900F061F9A869AF
:10023000EEE7A869F5E74FF080500369406940F6A2
:10024000FC71434308684FF01022401C06D0086838
:1002500000F58050834203D2092070479069F7E788
:100260000868401C04D00868401C03D00020704778
:100270009069F9E70420704770B504460068C34DE3
:10028000072876D2DFE800F033041929631E250021
:10029000D4E9026564682946304600F062F92A46CE
:1002A0002146304600F031F9AA002146304600F0E0
:1002B00057FB002800D0032070BD00F009FC4FF46C
:1002C000805007E0201D00F040F90028F4D100F034
:1002D000FFFB60682860002070BD241D94E80700C3
:1002E000920000F03DFB0028F6D00E2070BDFFF715
:1002F000A2FF0028FAD1D4E901034FF0805100EBAE
:10030000830208694D69684382420ED840F6F8704E
:1003100005684FF010226D1C09D0056805EB8305B8
:100320000B6949694B439D4203D9092070BD55694A
:10033000F4E70168491C03D00068401C02D003E0C8
:100340005069FAE70F2070BD2046FFF735FFFFF731
:1003500072FF0028F7D1201D00F0F7F80028F2D135
:1003600060680028F0D100F0E2F8FFF7D3FE00F05B
:10037000BFF8072070BD10B50C46182802D0012028
:10038000086010BD2068FFF777FF206010BD41684E
:10039000054609B1012700E0002740F6F8742068FF
:1003A0004FF01026401C2BD02068AA68920000F065
:1003B000D7FA38B3A86881002068401C27D020688D
:1003C000FFF7BDFED7B12068401C22D026684FF051
:1003D0008050AC686D68016942695143A9420DD9EA
:1003E000016940694143A14208D92146304600F0E5
:1003F000B8F822462946304600F087F800F078F831
:100400007069D2E700F093F8FFF784FEF6E77069B1
:10041000D6E77669DBE740F6FC7420684FF01026DB
:10042000401C23D02068401C0CD02068401C1FD0EA
:100430002568206805F18005401C1BD027683879A5
:10044000AA2819D040F6F8700168491C42D001680A
:10045000491C45D00168491C3ED001680968491C07
:100460003ED00168491C39D000683EE0B069DAE747
:10047000B569DEE7B769E2E710212846FFF778FEA5
:100480003968814222D12068401C05D0D4F8001080
:1004900001F18002C03107E0B169F9E730B108CA63
:1004A00051F8040D984201D1012000E000208A4259
:1004B000F4D158B1286810B1042803D0FEE72846CB
:1004C000FFF765FF3149686808600EE0FFF722FE1C
:1004D00000F00EF87169BBE77169BFE7706904E06D
:1004E0004FF480500168491C01D000F0CBFAFEE7C0
:1004F000BFF34F8F26480168264A01F4E06111439B
:100500000160BFF34F8F00BFFDE72DE9F0411746B3
:100510000D460646002406E03046296800F054F8EF
:10052000641C2D1D361DBC42F6D3BDE8F08140F69B
:10053000FC700168491C04D0D0F800004FF48051D1
:10054000FDE54FF010208069F8E74FF080510A690F
:10055000496900684A43824201D810207047002050
:10056000704770B50C4605464FF4806608E0284693
:1005700000F017F8B44205D3A4F5806405F5805562
:10058000002CF4D170BD0000F40A0000000000202F
:100590000CED00E00400FA05144801680029FCD0C5
:1005A0007047134A0221116010490B68002BFCD0E0
:1005B0000F4B1B1D186008680028FCD0002010603D
:1005C00008680028FCD07047094B10B501221A605A
:1005D000064A1468002CFCD0016010680028FCD08A
:1005E0000020186010680028FCD010BD00E4014015
:1005F00004E5014070B50C46054600F073F810B9EB
:1006000000F07EF828B121462846BDE8704000F091
:1006100007B821462846BDE8704000F037B8000012
:100620007FB5002200920192029203920A0B000B06
:100630006946012302440AE0440900F01F0651F80C
:10064000245003FA06F6354341F82450401C8242F8
:10065000F2D80D490868009A10430860081D016827
:10066000019A1143016000F03DF800280AD00649C4
:1006700010310868029A10430860091D0868039A3F
:10068000104308607FBD00000006004030B50F4CED
:10069000002200BF04EB0213D3F800582DB9D3F8A1
:1006A000045815B9D3F808581DB1521C082AF1D3C3
:1006B00030BD082AFCD204EB0212C2F80008C3F8CD
:1006C00004180220C3F8080830BD000000E0014013
:1006D0004FF08050D0F83001082801D0002070473A
:1006E000012070474FF08050D0F83011062905D016
:1006F000D0F83001401C01D0002070470120704725
:100700004FF08050D0F830010A2801D00020704707
:100710000120704708208F490968095808471020B0
:100720008C4909680958084714208A4909680958FA
:100730000847182087490968095808473020854923
:100740000968095808473820824909680958084744
:100750003C20804909680958084740207D490968BC
:100760000958084744207B49096809580847482028
:1007700078490968095808474C207649096809589A
:10078000084750207349096809580847542071499F
:1007900009680958084758206E49096809580847E8
:1007A0005C206C4909680958084760206949096854
:1007B00009580847642067490968095808476820AC
:1007C00064490968095808476C2062490968095852
:1007D000084770205F4909680958084774205D4937
:1007E00009680958084778205A490968095808478C
:1007F0007C205849096809580847802055490968EC
:10080000095808478420534909680958084788202F
:1008100050490968095808478C204E490968095809
:10082000084790204B4909680958084794204949CE
:10083000096809580847982046490968095808472F
:100840009C204449096809580847A0204149096883
:1008500009580847A4203F49096809580847A820B3
:100860003C49096809580847AC203A4909680958C1
:100870000847B0203749096809580847B420354966
:10088000096809580847B8203249096809580847D3
:10089000BC203049096809580847C0202D4909681B
:1008A00009580847C4202B49096809580847C82037
:1008B0002849096809580847CC2026490968095879
:1008C0000847D0202349096809580847D4202149FE
:1008D000096809580847D8201E4909680958084777
:1008E000DC201C49096809580847E02019490968B3
:1008F00009580847E4201749096809580847E820BB
:100900001449096809580847EC2012490968095830
:100910000847F0200F49096809580847F4200D4995
:10092000096809580847F8200A490968095808471A
:10093000FC2008490968095808475FF48070054998
:10094000096809580847000003480449024A034B54
:100950007047000000000020000B0000000B0000AA
:1009600040EA010310B59B070FD1042A0DD310C82C
:1009700008C9121F9C42F8D020BA19BA884201D97E
:10098000012010BD4FF0FF3010BD1AB1D30703D0C6
:10099000521C07E0002010BD10F8013B11F8014B7C
:1009A0001B1B07D110F8013B11F8014B1B1B01D198
:1009B000921EF1D1184610BD02F0FF0343EA032254
:1009C00042EA024200F005B87047704770474FF0A6
:1009D00000020429C0F0128010F0030C00F01B800C
:1009E000CCF1040CBCF1020F18BF00F8012BA8BF1A
:1009F00020F8022BA1EB0C0100F00DB85FEAC17CDE
:100A000024BF00F8012B00F8012B48BF00F8012B90
:100A100070474FF0000200B51346944696462039C1
:100A200022BFA0E80C50A0E80C50B1F12001BFF4A7
:100A3000F7AF090728BFA0E80C5048BF0CC05DF80D
:100A400004EB890028BF40F8042B08BF704748BF5B
:100A500020F8022B11F0804F18BF00F8012B7047CF
:100A6000014B1B68DB6818470000002009480A4951
:100A70007047FFF7FBFFFFF745FB00BD20BFFDE719
:100A8000064B1847064A1060016881F308884068E1
:100A900000470000000B0000000B000017040000DE
:100AA000000000201EF0040F0CBFEFF30881EFF3ED
:100AB0000981886902380078182803D100E0000015
:100AC000074A1047074A12682C3212681047000084
:100AD00000B5054B1B68054A9B58984700BD0000B0
:100AE0007703000000000020F00A0000040000006E
:100AF000001000000000000000FFFFFF0090D00386
:1010000080130020B157020069C00000175702008A
:1010100069C0000069C0000069C000000000000055
:101020000000000000000000000000000D58020059
:1010300069C000000000000069C0000069C0000035
:10104000755802007B58020069C0000069C00000AA
:1010500069C0000069C0000069C0000069C00000EC
:101060008158020069C0000069C000008758020072
:1010700069C000008D580200935802009958020080
:1010800069C0000069C0000069C0000069C00000BC
:1010900069C0000069C0000069C0000069C00000AC
:1010A00069C000009F58020069C0000069C00000CC
:1010B00069C0000069C0000069C0000069C000008C
:1010C000A558020069C0000069C0000069C00000A6
:1010D00069C0000069C0000069C0000069C000006C
:1010E00069C0000069C0000069C0000069C000005C
:1010F00069C0000069C0000069C0000069C000004C
:1011000069C0000069C0000000F002F824F03FFB55
:101110000AA090E8000C82448344AAF10107DA4552
:1011200001D124F034FBAFF2090EBAE80F0013F03E
:10113000010F18BFFB1A43F001031847584C020077
:10114000784C02000A444FF0000C10F8013B13F0F9
:10115000070408BF10F8014B1D1108BF10F8015B10
:10116000641E05D010F8016B641E01F8016BF9D103
:1011700013F0080F1EBF10F8014BAD1C0C1B09D15A
:101180006D1E58BF01F801CBFAD505E014F8016BCC
:1011900001F8016B6D1EF9D59142D6D3704700005E
:1011A0000023002400250026103A28BF78C1FBD870
:1011B000520728BF30C148BF0B6070471FB500F011
:1011C0003DF88DE80F001FBD1EF0040F0CBFEFF3BC
:1011D0000880EFF30980014A10470000ABBF000010
:1011E000F0B44046494652465B460FB402A0013077
:1011F00001B50648004700BF01BC86460FBC8046CB
:10120000894692469B46F0BC7047000009110000D9
:101210008269034981614FF001001044704700006A
:101220002512000001B41EB400B514F0CBFE01B4C9
:101230000198864601BC01B01EBD000024F0A4BA8E
:1012400070B51A4C054609202070A01C00F0D1F89A
:101250005920A08029462046BDE8704008F0CEB84D
:1012600008F0D7B870B50C461149097829B1A0F13A
:1012700060015E2908D3012013E0602804D06928AA
:1012800002D043F201000CE020CC0A4E94E80E009C
:1012900006EB8000A0F58050241FD0F8806E284611
:1012A000B047206070BD012070470000080000209A
:1012B00018000020F05802003249884201D2012073
:1012C00070470020704770B50446A0F500002E4E10
:1012D000B0F1786F02D23444A4F500042948844266
:1012E00001D2012500E0002500F043F848B125B9FE
:1012F000B44204D32548006808E0012070BD0020F6
:1013000070BD002DF9D1B442F9D321488442F6D200
:10131000F3E710B50446A0F50000B0F1786F03D2F2
:1013200019480444A4F5000400F023F84FF080416C
:1013300030B11648006804E08C4204D2012003E07A
:1013400013488442F8D2002080F0010010BD10B58F
:1013500020B1FFF7DEFF08B1012010BD002010BD55
:1013600010B520B1FFF7AFFF08B1012010BD00207C
:1013700010BD084808490068884201D10120704723
:101380000020704700600200000000201C000020C8
:101390000800002054000020BEBAFECA10B5044662
:1013A0000021012000F03DF800210B2000F039F869
:1013B0000421192000F035F804210D2000F031F847
:1013C00004210E2000F02DF804210F2000F029F850
:1013D0000421C84300F025F80621162000F021F86A
:1013E0000621152000F01DF82046FFF729FF0020F8
:1013F00010BDB62101807047FFF732BF114870471A
:1014000010487047104A10B514680F4B0F4A083344
:101410001A60FFF727FF0C48001D046010BD7047DD
:1014200070474907090E002804DB00F1E02080F82E
:101430000014704700F00F0000F1E02080F8141D48
:101440007047000003F9004210050240010000014E
:10145000FE48002101604160018170472DE9F7439A
:10146000044692B091464068FFF771FF40B1606852
:10147000FFF776FF20B9607800F00300022801D062
:10148000012000E00020F14E30724846FFF71BFFBC
:1014900018B1102015B0BDE8F0834946012001F0D5
:1014A0008EFE0028F6D101258DF842504FF4C05031
:1014B000ADF84000002210A9284606F009FC0028DB
:1014C000E8D18DF842504FF428504FF00008ADF8A5
:1014D000400047461C216846CDF81C8024F0EFF8F8
:1014E0009DF81C0008AA20F00F00401C20F0F0001E
:1014F00010308DF81C0020788DF81D0061789DF863
:101500001E0061F3420040F001008DF81E009DF8BE
:1015100000000AA940F002008DF800002089ADF813
:101520003000ADF83270608907AFADF834000B972A
:10153000606810AC0E900A94684606F0BCF900286A
:10154000A8D1BDF8200030808DF8425042F601202D
:10155000ADF840009DF81E0008AA20F00600801C8F
:1015600020F001008DF81E000220ADF83000ADF82B
:10157000340013A80E900AA9684606F09CF90028CA
:1015800088D1BDF820007080311D484600F033F945
:10159000002887D18DF8425042F6A620ADF84000D1
:1015A0001C216846CDF81C8024F089F89DF81C00A9
:1015B000ADF8345020F00F00401C20F0F000103047
:1015C0008DF81C009DF81D0008AA20F0FF008DF882
:1015D0001D009DF81E000AA920F0060040F0010041
:1015E000801C8DF81E009DF800008DF8445040F0DE
:1015F00002008DF80000CDE90A4711A80E90ADF861
:101600003050684606F057F9002899D1BDF82000FF
:10161000F08000203EE73EB504460820ADF800000B
:101620002046FFF750FE08B110203EBD21460120A4
:1016300001F0C5FD0028F8D12088ADF804006088CD
:10164000ADF80600A088ADF80800E088ADF80A0003
:101650007E4801AB6A468088002106F035FDBDF862
:1016600000100829E1D003203EBD1FB5044600202C
:1016700002900820ADF80800CDF80CD02046FFF706
:1016800022FE10B1102004B010BD704802AA81885B
:101690004FF6FF7006F05AFF0028F4D1BDF808108D
:1016A000082901D00320EEE7BDF800102180BDF825
:1016B00002106180BDF80410A180BDF80610E18021
:1016C000E1E701B582B00220ADF800005F4802AB4F
:1016D0006A464088002106F0F7FCBDF80010022998
:1016E00000D003200EBD1CB5002100910221ADF8F1
:1016F00000100190FFF70DFE08B110201CBD5348EB
:101700006A4641884FF6FF7006F020FFBDF80010D2
:101710000229F3D003201CBDFEB54C4C06461546ED
:10172000207A0F46C00705D00846FFF7CCFD18B158
:101730001020FEBD0F20FEBDF82D01D90C20FEBDEE
:101740003046FFF7C0FD18BB208801A905F0B8FDA1
:101750000028F4D130788DF80500208801A906F022
:1017600091FC0028EBD100909DF800009DF8051039
:1017700040F002008DF80000090703D040F0080097
:101780008DF800002088694606F019FC0028D6D1A3
:10179000ADF8085020883B4602AA002106F094FCD0
:1017A000BDF80810A942CAD00320FEBD7CB505468D
:1017B0000020009001900888ADF800000C462846F3
:1017C0000195FFF7C4FD18B92046FFF7A2FD08B147
:1017D00010207CBD15B1BDF8000050B11B486A4611
:1017E00001884FF6FF7006F0B1FEBDF800102180B1
:1017F0007CBD0C207CBD30B593B0044600200D4666
:101800000090142101A823F05AFF1C2108A823F0FE
:1018100056FF9DF80000CDF808D020F00F00401CC6
:1018200020F0F00010308DF800009DF8010020F04D
:10183000FF008DF801009DF8200040F002008DF8B7
:10184000200001208DF8460002E000002002002068
:1018500042F60420ADF8440011A801902088ADF8AC
:101860003C006088ADF83E00A088ADF84000E088FC
:10187000ADF842009DF8020006AA20F00600801C88
:1018800020F001008DF802000820ADF80C00ADF842
:1018900010000FA8059001A908A806F00CF8002870
:1018A00003D1BDF818002880002013B030BD00001F
:1018B000F0B5007B059F1E4614460D46012800D05A
:1018C000FFDF0C2030803A203880002C08D0287AA6
:1018D000032806D0287B012800D0FFDF1720608175
:1018E000F0BDA889FBE72DE9F04786B0144691F8D2
:1018F0000C900E9A0D46B9F1010F0BD01021007B10
:101900002E8A8846052807D0062833D0FFDF06B088
:10191000BDE8F0870221F2E7E8890C2100EB4000E6
:1019200001EB4000188033201080002CEFD0E889B4
:10193000608100271AE00096688808F1020301AA76
:10194000696900F084FF06EB0800801C07EB470183
:1019500086B204EB4102BDF8040090810DF106014E
:1019600040460E3212F0D3FD7F1CBFB26089B842F0
:10197000E1D8CCE734201080E889B9F1010F11D00B
:10198000122148430E301880002CC0D0E8896081B5
:101990004846B9F1010F00D00220207300270DF155
:1019A000040A1FE00621ECE70096688808F10203AC
:1019B00001AA696900F04BFF06EB0800801C86B2A3
:1019C000B9F1010F12D007EBC70004EB4000BDF8DE
:1019D0000410C18110220AF10201103023F0CEFD63
:1019E0007F1CBFB26089B842DED890E707EB4701A1
:1019F00004EB4102BDF80400D0810AF10201404627
:101A0000103212F084FDEBE72DE9F0470E4688B066
:101A100090F80CC096F80C80378AF5890C20109944
:101A200002F10C044FF0000ABCF1030F08D0BCF126
:101A3000040F3ED0BCF1070F7DD0FFDF08B067E791
:101A400005EB850C00EB4C00188031200880002A43
:101A5000F4D0A8F1060000F0FF09558125E0182117
:101A600001A823F02CFE00977088434601AA7169F3
:101A700000F0EDFEBDF804002080BDF80600E08017
:101A8000BDF808002081A21C0DF10A01484612F0A1
:101A90003EFDB9F1000F00D018B184F804A0A4F8FD
:101AA00002A007EB080087B20A346D1EADB2D6D291
:101AB000C4E705EB850C00EB4C0018803220088051
:101AC000002ABBD0A8F1050000F0FF09558137E0DE
:101AD00000977088434601AA716900F0B8FE9DF82E
:101AE0000600BDF80410E1802179420860F300018E
:101AF00062F34101820862F38201C20862F3C3010A
:101B0000020962F30411420962F34511820962F38A
:101B100086112171C0096071BDF80700208122463D
:101B20000DF10901484612F0F2FC18B184F802A048
:101B3000A4F800A000E007E007EB080087B20A3431
:101B40006D1EADB2C4D279E7A8F1020084B205FBE4
:101B500008F000F10E0CA3F800C035230B80002A1A
:101B6000A6D055819481009783B270880E32716936
:101B700000F06DFE62E72DE9F84F1E460A9D0C4607
:101B800081462AB1607A00F58070D080E0891081AA
:101B900099F80C000C274FF000084FF00E0A0D28A2
:101BA00073D2DFE800F09E070E1C28303846556AD5
:101BB00073737300214648460095FFF779FEBDE830
:101BC000F88F207B9146082802D0032800D0FFDF41
:101BD000378030200AE000BFA9F80A80EFE7207BB9
:101BE0009146042800D0FFDF378031202880B9F1EA
:101BF000000FF1D1E3E7207B9146042800D0FFDFFE
:101C000037803220F2E7207B9146022800D0FFDFA8
:101C100037803320EAE7207B1746022800D0FFDF19
:101C20003420A6F800A02880002FC8D0A7F80A808A
:101C3000C5E7207B1746042800D0FFDF3520A6F833
:101C400000A02880002FBAD04046A7F80A8012E0F2
:101C5000207B1746052802D0062800D0FFDF102081
:101C6000308036202880002FA9D0E0897881A7F81D
:101C70000E80B9F80E00B881A1E7207B91460728B5
:101C800000D0FFDF37803720B0E72AE04FF01200A6
:101C900018804FF038001700288090D0E0897881B4
:101CA000A7F80E80A7F8108099F80C000A2805D034
:101CB0000B2809D00C280DD0FFDF80E7207B0A28F5
:101CC00000D0FFDF01200AE0207B0B2800D0FFDFDF
:101CD000042004E0207B0C2800D0FFDF05203873AF
:101CE0006DE7FFDF6BE770B50C46054601F0ABFB17
:101CF00020B10078222804D2082070BD43F20200EF
:101D000070BD0521284610F075FE206008B1002046
:101D100070BD032070BD30B44880087820F00F00FB
:101D2000C01C20F0F000903001F8080B1DCA81E8BB
:101D30001D0030BC07F0E3BB2DE9FF4784B000274E
:101D40008246029707989046894612300AF0DCF9DD
:101D5000401D20F00306079828B907A95046FFF751
:101D6000C2FF002854D1B9F1000F05D00798017BBC
:101D700019BB052504681BE098F80000092803D06A
:101D80000D2812D0FFDF46E0079903254868B0B35D
:101D9000497B42887143914239D98AB2B3B2011D5D
:101DA00010F09BFC0446078002E0079C04250834E1
:101DB0000CB1208810B1032D29D02CE00798012107
:101DC00012300AF0D3F9ADF80C00024602AB2946F6
:101DD000504608F000FA070001D1A01C02900798B5
:101DE0003A461230C8F80400A8F802A003A94046F9
:101DF000029B0AF0C8F9D8B10A2817D200E006E021
:101E0000DFE800F007091414100B0D14141213204E
:101E100014E6002012E6112010E608200EE643F238
:101E200003000BE6072009E60D2007E6032005E680
:101E3000BDF80C002346CDE900702A4650460799AC
:101E400000F015FD57B9032D08D10798B3B2417BB7
:101E5000406871438AB2011D10F053FCB9F1000FC4
:101E6000D7D0079981F80C90D3E72DE9FE4F914622
:101E70001A881C468A468046FAB102AB494608F0E9
:101E8000AAF9050019D04046A61C278810F0F6FED6
:101E90003246072629463B46009610F004FB208870
:101EA0002346CDE900504A465146404600F0DFFC4B
:101EB000002020800120BDE8FE8F0020FBE710B548
:101EC00086B01C46AAB104238DF800301388ADF803
:101ED00008305288ADF80A208A788DF80E200988DB
:101EE000ADF80C1000236A462146FFF725FF06B027
:101EF00010BD1020FBE770B50D46052110F07AFDEE
:101F0000040000D1FFDF294604F11200BDE8704053
:101F10000AF015B92DE9F8430D468046002607F072
:101F2000EBFA04462878102878D2DFE800F0773BF7
:101F30003453313112313131083131313131287975
:101F4000001FC0B2022801D0102810D114BBFFDF3F
:101F500035E004B9FFDF0521404610F04BFD007B62
:101F6000032806D004280BD0072828D0FFDF072637
:101F700055E02879801FC0B2022820D050B1F6E782
:101F80002879401FC0B2022819D0102817D0EEE7D8
:101F900004B9FFDF13E004B9FFDF287901280ED16F
:101FA000172137E00521404610F024FD070000D13D
:101FB000FFDF07F1120140460AF09EF82CB12A46D5
:101FC00021464046FFF7A7FE29E01321404602F0D4
:101FD000F7FC24E004B9FFDF0521404610F00AFDBC
:101FE000060000D1FFDF694606F112000AF08EF804
:101FF000060000D0FFDFA988172901D2172200E0D0
:102000000A46BDF80000824202D9014602E005E01E
:102010001729C5D3404600F03AFCD0E7FFDF304631
:10202000BDE8F883401D20F0030219B102FB01F066
:10203000001D00E000201044704713B5009848B11F
:102040000024684610F0F3FA002C02D1F74A0099F8
:1020500011601CBD01240020F4E72DE9F0470C4677
:1020600015462421204623F02AFB05B9FFDFA87876
:1020700060732888DFF8B4A3401D20F00301AF7817
:102080008946DAF8000010F0F0FA060000D1FFDF10
:102090004FF000082660A6F8008077B109FB07F131
:1020A000091D0AD0DAF8000010F0DFFA060000D1AE
:1020B000FFDF6660C6F8008001E0C4F8048029886C
:1020C00004F11200BDE8F0470AF008B82DE9F04726
:1020D000804601F112000D4681460AF015F8401DB8
:1020E000D24F20F003026E7B14462968386810F046
:1020F000E7FA3EB104FB06F2121D03D069683868A6
:1021000010F0DEFA052010F01DFC0446052010F04A
:1021100021FC201A012802D1386810F09BFA4946A8
:102120004046BDE8F04709F0EEBF70B50546052111
:1021300010F060FC040000D1FFDF04F1120128461A
:10214000BDE8704009F0D8BF2DE9F04F91B04FF0D5
:10215000000BADF834B0ADF804B047880C46054626
:1021600092460521384610F045FC060000D1FFDFFD
:1021700024B1A780A4F806B0A4F808B029780922F1
:102180000B20B2EB111F7DD12A7A04F11001382700
:102190004FF00C084FF001090391102A73D2DFE8C9
:1021A00002F072F2F1F07F08D2888D9F3DDBF3EEF2
:1021B000B6B6307B022800D0FFDFA88908EBC0014B
:1021C000ADF804103021ADF83410002C25D060811A
:1021D000B5F80E9000271DE004EBC708317C88F8A5
:1021E0000E10F189A8F80C10CDF80090688804232F
:1021F00004AA296900F02BFBBDF81010A8F81010F4
:1022000009F10400BDF812107F1C1FFA80F9A8F82C
:102210001210BFB26089B842DED80DE1307B0228CF
:1022200000D0FFDFE98908EBC100ADF804003020E1
:10223000ADF83400287B0A90001FC0B20F90002C2C
:10224000EBD06181B5F81090002725E0CDF8009023
:102250006888696903AA0A9B00F0F9FA0A9804EBF6
:10226000C70848441FFA80F908F10C0204A90F9826
:1022700012F04DF918B188F80EB0A8F80CB0BDF8FE
:102280000C1001E0D4E0CFE0A8F81010BDF80E105B
:102290007F1CA8F81210BFB26089B842D6D8CBE034
:1022A0000DA8009001AB224629463046FFF71BFBE4
:1022B000C2E0307B082805D0FFDF03E0307B082830
:1022C00000D0FFDFE8891030ADF804003620ADF80B
:1022D0003400002C3FD0A9896181F189A18127E0D8
:1022E000307B092800D0FFDFA88900F10C01ADF890
:1022F00004103721ADF83410002C2CD06081E8890F
:102300000090AB89688804F10C02296956E0E889DD
:102310003921103080B2ADF80400ADF83410002C33
:1023200074D0A9896181287A0E280AD002212173EC
:10233000E989E181288A0090EB8968886969039AB4
:102340003CE00121F3E70DA8009001AB22462946AD
:102350003046FFF759FB6FE0307B0A2800D0FFDFE3
:102360001220ADF80400ADF834704CB3A989618136
:10237000A4F810B0A4F80EB084F80C905CE020E053
:1023800002E031E039E042E0307B0B2800D0FFDF93
:10239000288AADF834701230ADF8040084B10421FD
:1023A0002173A9896181E989E181298A2182688A69
:1023B00000902B8A688804F11202696900F047FADC
:1023C0003AE0307B0C2800D0FFDF1220ADF804008B
:1023D000ADF834703CB305212173A4F80AB0A4F819
:1023E0000EB0A4F810B027E00DA8009001AB224673
:1023F00029463046FFF75CFA1EE00DA8009001ABBD
:10240000224629463046FFF7B6FB15E034E03B2173
:10241000ADF80400ADF8341074B3A4F80690A4F835
:1024200008B084F80AB007E0FFDF05E010000020E4
:10243000297A012917D0FFDFBDF80400AAF80000AF
:102440006CB1BDF834002080BDF804006080BDF898
:102450003400392803D03C2801D086F80CB011B0E4
:102460000020BDE8F08F3C21ADF80400ADF8341039
:1024700014B1697AA172DFE7AAF80000EFE72DE94D
:10248000F84356880F46804615460521304610F021
:10249000B1FA040000D1FFDF123400943B464146FC
:1024A00030466A6809F0A3FFBAE570B50D4605210C
:1024B00010F0A0FA040000D1FFDF294604F1120059
:1024C000BDE8704009F02DBE70B50D46052110F035
:1024D00091FA040000D1FFDF294604F11200BDE8A3
:1024E000704009F04BBE70B50546052110F082FA28
:1024F000040000D1FFDF04F1080321462846BDE8AF
:1025000070400422B1E470B50546052110F072FA5E
:10251000040000D1FFDF214628462368BDE8704053
:102520000522A2E470B50646052110F063FA040006
:1025300000D1FFDF04F1120009F0E6FD401D20F09C
:10254000030511E0011D008803224318214630468F
:10255000FFF78BFC00280BD0607BABB2684382B2E4
:102560006068011D10F003F9606841880029E9D115
:1025700070BD70B50E46054606F0BEFF040000D1E2
:10258000FFDF0120207266726580207820F00F0046
:10259000C01C20F0F00030302070BDE8704006F024
:1025A000AEBF2DE9F0438BB00D461446814606A917
:1025B000FFF799FB002814D14FF6FF7601274FF45F
:1025C00020588CB103208DF800001020ADF81000C9
:1025D00007A8059007AA204604A911F0B7FF78B113
:1025E00007200BB0BDE8F0830820ADF808508DF847
:1025F0000E708DF80000ADF80A60ADF80C800CE0AC
:102600000698A17801742188C1818DF80E70ADF80B
:102610000850ADF80C80ADF80A606A4602214846C1
:10262000069BFFF789FBDCE708B501228DF8022045
:1026300042F60202ADF800200A4603236946FFF77E
:102640003EFC08BD08B501228DF8022042F60302C7
:10265000ADF800200A4604236946FFF730FC08BDA8
:1026600000B587B079B102228DF800200A88ADF854
:1026700008204988ADF80A1000236A460521FFF7B3
:102680005BFB07B000BD1020FBE709B1072316E490
:102690000720704770B588B00D461446064606A957
:1026A000FFF721FB00280ED17CB10620ADF80850C1
:1026B0008DF80000ADF80A40069B6A460821DC81CF
:1026C0003046FFF739FB08B070BD05208DF80000DB
:1026D000ADF80850F0E700B587B059B107238DF881
:1026E0000030ADF80820039100236A460921FFF766
:1026F00023FBC6E71020C4E770B588B00C46064639
:10270000002506A9FFF7EFFA0028DCD10698012181
:10271000123009F02BFD9CB12178062921D2DFE887
:1027200001F0200505160318801E80B2C01EE28845
:1027300080B20AB1A3681BB1824203D90C20C2E760
:102740001020C0E7042904D0A08850B901E0062079
:10275000B9E7012913D0022905D004291CD0052985
:102760002AD00720AFE709208DF800006088ADF877
:102770000800E088ADF80A00A068039023E00A2072
:102780008DF800006088ADF80800E088ADF80A0018
:10279000A0680A25039016E00B208DF800006088E1
:1027A000ADF80800A088ADF80A00E088ADF80C008C
:1027B000A0680B25049006E00C208DF800006078DE
:1027C0008DF808000C256A4629463046069BFFF71F
:1027D000B3FA78E700B587B00D228DF80020ADF888
:1027E000081000236A461946FFF7A6FA49E700B524
:1027F00087B071B102228DF800200A88ADF8082058
:102800004988ADF80A1000236A460621FFF794FABA
:1028100037E7102035E770B586B0064601200D4633
:10282000ADF808108DF80000014600236A463046D6
:10283000FFF782FA040008D12946304605F05EFC15
:102840000021304605F078FC204606B070BDF8B592
:102850001C4615460E46069F10F0FEF92346FF1D46
:10286000BCB231462A4600940FF0E9FDF8BD30B401
:102870001146DDE902423CB1032903D0002330BCFC
:1028800008F034BB0123FAE71A8030BC704770B5FA
:102890000C460546FFF72FFB2146284605F03DFC78
:1028A0002846BDE87040012105F046BC4FF0E0220B
:1028B0004FF400400021C2F88001BFF34F8FBFF3F7
:1028C0006F8F1748016001601649900208607047D9
:1028D000134900B500220A600A60124B4FF0607283
:1028E0001A60002808BF00BD0F4A104BDFF840C037
:1028F00001280CD002281CBFFFDF00BD03200860A8
:102900001A604FF4000000BFCCF8000000BD0220A8
:1029100008601A604FF04070F6E700B5FFDF00BDB9
:1029200000F5004008F50140A002002014F5004029
:1029300004F5014070B50B2000F0BDF9082000F04F
:10294000BAF900210B2000F0D4F90021082000F092
:10295000D0F9F44C01256560A5600020C4F8400161
:10296000C4F84401C4F848010B2000F0B5F9082070
:1029700000F0B2F90B2000F091F9256070BD10B5A0
:102980000B2000F098F9082000F095F9E5480121A6
:1029900041608160E4490A68002AFCD10021C0F846
:1029A0004011C0F84411C0F848110B2000F094F910
:1029B000BDE81040082000F08FB910B50B2000F0E2
:1029C0008BF9BDE81040082000F086B900B530B1A1
:1029D000012806D0022806D0FFDF002000BDD34822
:1029E00000BDD34800BDD248001D00BD70B5D1491F
:1029F0004FF000400860D04DC00BC5F80803CF4829
:102A000000240460C5F840410820C43500F053F9A3
:102A1000C5F83C41CA48047070BD08B5C14A0021E0
:102A200028B1012811D002281CD0FFDF08BD4FF4C7
:102A30008030C2F80803C2F84803BB483C3001604C
:102A4000C2F84011BDE80840D0E74FF40030C2F8AA
:102A50000803C2F84803B44840300160C2F844118A
:102A6000B3480CE04FF48020C2F80803C2F84803D2
:102A7000AD4844300160C2F84811AD48001D0068FF
:102A8000009008BD70B516460D460446022800D9D0
:102A9000FFDF0022A348012304F110018B4000EB6B
:102AA0008401C1F8405526B1C1F84021C0F8043373
:102AB00003E0C0F80833C1F84021C0F8443370BDCA
:102AC0002DE9F0411D46144630B1012833D00228CB
:102AD00038D0FFDFBDE8F081891E002221F07F4160
:102AE0001046FFF7CFFF012D23D00020944D924FC9
:102AF000012668703E61914900203C39086002203F
:102B0000091D08608D490420303908608B483D3428
:102B1000046008206C6000F0DFF83004C7F804039C
:102B2000082000F0BBF88349F007091F08602E70E9
:102B3000D0E70120DAE7012B02D00022012005E0D6
:102B40000122FBE7012B04D000220220BDE8F04166
:102B500098E70122F9E774480068704770B500F003
:102B6000D8F8704C0546D4F840010026012809D158
:102B7000D4F80803C00305D54FF48030C4F8080327
:102B8000C4F84061D4F8440101280CD1D4F80803FA
:102B9000800308D54FF40030C4F80803C4F844613A
:102BA000012012F0A9FCD4F8480101280CD1D4F876
:102BB0000803400308D54FF48020C4F80803C4F884
:102BC0004861022012F098FC5E48056070BD70B547
:102BD00000F09FF85A4D0446287850B1FFF706FFE1
:102BE000687818B10020687012F086FC55480460BF
:102BF00070BD0320F8E74FF0E0214FF40010C1F85A
:102C000000027047152000F067B84B4901200861A9
:102C1000082000F061B848494FF47C10C1F808035F
:102C20000020024601EB8003C3F84025C3F8402191
:102C3000401CC0B20628F5D37047410A43F609523A
:102C40005143C0F3080010FB02F000F5807001EB67
:102C50005020704710B5430B48F2376463431B0C98
:102C60005C020C60384C03FB0400384B4CF2F72438
:102C700043435B0D13FB04F404EB402000F580702C
:102C80004012107008681844086010BD2C48406855
:102C9000704729490120C1F800027047002809DB6C
:102CA00000F01F02012191404009800000F1E02066
:102CB000C0F80011704700280DDB00F01F02012151
:102CC00091404009800000F1E020C0F88011BFF37E
:102CD0004F8FBFF36F8F7047002809DB00F01F0292
:102CE000012191404009800000F1E020C0F88012ED
:102CF00070474907090E002804DB00F1E02080F846
:102D00000014704700F00F0000F1E02080F8141D5F
:102D100070470C48001F00680A4A0D49121D1160D7
:102D20007047000000B0004004B500404081004002
:102D300044B1004008F5014000800040408500405B
:102D40003400002014050240F7C2FFFF6F0C0100A1
:102D5000010000010A4810B5046809490948083112
:102D6000086012F05DFC0648001D046010BD0649B5
:102D7000002008604FF0E0210220C1F88002704777
:102D80001005024001000001FC1F004010B50D209D
:102D900000F077F8C4B26FF0040000F072F8C0B22F
:102DA000844200D0FFDF3E490120086010BD70B5AD
:102DB0000D2000F048F83B4C0020C4F8000101252C
:102DC000C4F804530D2000F04FF825604FF0E021C7
:102DD0006014C1F8000170BD10B50D2000F033F88B
:102DE0003048012141600021C0F80011BDE81040C9
:102DF0000D2000F039B82C4810B504682A492B483A
:102E0000083108602749D1F80001012804D0FFDF0C
:102E10002548001D046010BD2148001D00680022E7
:102E2000C0B2C1F8002113F047F8F1E710B51D4812
:102E3000D0F800110029FBD0FFF7DDFFBDE81040FE
:102E40000D2000F011B800280DDB00F01F02012159
:102E500091404009800000F1E020C0F88011BFF3EC
:102E60004F8FBFF36F8F7047002809DB00F01F0200
:102E7000012191404009800000F1E020C0F880125B
:102E80007047002804DB00F1E02090F8000405E022
:102E900000F00F0000F1E02090F8140D4009704799
:102EA00004D5004000D000401005024001000001A0
:102EB0004FF0E0214FF00070C1F8800101F5C071C2
:102EC000BFF34F8FBFF36F8FC1F80001384B8022E3
:102ED00083F8002441F8800C704700B502460420B6
:102EE000344903E001EBC0031B792BB1401EC0B293
:102EF000F8D2FFDFFF2000BD41F8302001EBC00118
:102F000000224A718A7101220A7100BD294A0021FA
:102F100002EBC0000171704710B50446042800D3CD
:102F2000FFDF244800EBC4042079012800D0FFDF34
:102F30006079A179401CC0B2814200D060714FF02D
:102F4000E0214FF00070C1F8000210BD2DE9F04102
:102F500019480568184919480831086014480426BA
:102F600090F80004134F4009154C042818D0FFDFD7
:102F700016E0217807EBC1000279012A08D14279D5
:102F800083799A4204D04279827157F831008047A0
:102F90002078401CC0B22070042801D3002020708B
:102FA000761EF6B2E5D20448001D0560BDE8F0814A
:102FB00019E000E0D80500201005024001000001E2
:102FC000500000200548064A0168914201D10021C5
:102FD000016004490120086070470000540000208F
:102FE000BEBAFECA40E5014070B50C46054609F080
:102FF0009BFB21462846BDE870400AF080BC704724
:103000002CFFFFFFDBE5B15100600200B600FFFFBF
:103010008C00000069915B00935FFEEDA0843C731F
:10302000F87462145E06C0CB72F2136030B5F84DCE
:103030000446062CA9780ED2DFE804F0030E0E0E2B
:103040000509FFDF08E0022906D0FFDF04E00329BD
:1030500002D0FFDF00E0FFDFAC7030BD30B50446CA
:103060001038EB4D07280CD2DFE800F0040C060CFA
:103070000C0C0C00FFDF05E0287E112802D0FFDFDA
:1030800000E0FFDF2C7630BD2DE9F04111F0C8FBE8
:10309000044612F0A1FD201AC5B206200FF052FC22
:1030A000044606200FF056FC211AD94C207E122827
:1030B00018D000200F1807200FF044FC0646072008
:1030C0000FF048FC301A3918207E13280CD000204D
:1030D0000144A078042809D000200844281AC0B26E
:1030E000BDE8F0810120E5E70120F1E70120F4E7E8
:1030F000C74810B590F825004108C54800F12600E2
:1031000005D00DF018FBBDE8104006F00BB80DF02F
:10311000F3FAF8E730B50446A1F120000D460A287D
:103120004AD2DFE800F005070C1C2328353A3F445B
:10313000FFDF42E0207820283FD1FFDF3DE0B448A8
:103140008178052939D0007E122836D020782428AD
:1031500033D0252831D023282FD0FFDF2DE0207851
:1031600022282AD0232828D8FFDF26E0207822280A
:1031700023D0FFDF21E0207822281ED024281CD075
:1031800026281AD0272818D0292816D0FFDF14E0C7
:103190002078252811D0FFDF0FE0207825280CD0DB
:1031A000FFDF0AE02078252807D0FFDF05E0207840
:1031B000282802D0FFDF00E0FFDF257030BD1FB5FB
:1031C00004466A46002001F03CFEB4B1BDF802207E
:1031D0004FF6FF700621824201D1ADF80210BDF812
:1031E0000420824201D1ADF80410BDF808108142DC
:1031F00003D14FF44860ADF8080068460EF014F9AA
:1032000005F090FF04B010BD70B514460D4606469B
:10321000FEF759F858B90DB1A54201D90C2070BD7F
:10322000002408E056F82400FEF74DF808B11020FD
:1032300070BD641CE4B2AC42F4D3002070BD2DE933
:10324000F04105461F4690460E4600240068FEF7F2
:1032500087F830B9A98828680844401EFEF780F82E
:1032600008B110203CE728680028A88802D0B8429E
:1032700002D850E00028F5D0092031E72968085D20
:10328000B8B1671CCA5D152A2ED03CDC152A3AD28B
:10329000DFE802F03912222228282A2A313139396E
:1032A00039393939393939392200085D30BB641C64
:1032B000A4B2A242F9D833E00228DDD1A01C085CF8
:1032C00088F80000072801D2400701D40A2007E748
:1032D000307840F0010015E0C143C90707E001283C
:1032E00007D010E00620FBE60107A1F1805100297C
:1032F000F5D01846F4E63078810701D50B20EFE6CB
:1033000040F0020030702868005D384484B2A8881C
:10331000A04202D2B0E74FF4485382B2A242ADD8E5
:103320000020DDE610B5027843F2022354080122A2
:10333000022C12D003DC3CB1012C16D106E0032C88
:1033400010D07F2C11D112E0002011E080790324ED
:10335000B4EB901F09D10A700BE08079B2EB901F9B
:1033600003D1F8E780798009F5D0184610BDFF2019
:103370000870002010BD08B500208DF8000024481A
:1033800090F82E1049B190F82F0002280ED0032893
:103390000ED0FFDF9DF8000008BD1D4869462530AE
:1033A00001F09EFD0028F5D0FFDFF3E7032000E0E9
:1033B00001208DF80000EDE738B50C46054669465A
:1033C00001F08EFD00280DD19DF80010207861F3EA
:1033D0004700207055F8010FC4F80100A888A4F830
:1033E0000500002038BD38B51378A8B1022813D0E5
:1033F000FF281AD007A46D46246800944C7905EB89
:103400009414247864F347031370032809D00FE061
:10341000EC0100200302FF0123F0FE0313700228D9
:10342000F3D1D8B240F0010005E043F0FE00107087
:10343000107820F0010010700868C2F80100888838
:10344000A2F8050038BD02210FF0D4BA38B50C46F9
:103450000978222901D2082038BDADF800008DF886
:10346000022068460DF0A9F905F05CFE050003D1C5
:1034700021212046FFF74EFE284638BD1CB500200E
:103480008DF80000CDF80100ADF80500FB4890F87C
:103490002E00022801D0012000E000208DF8070056
:1034A00068460DF0FAFA002800D0FFDF1CBD0022AC
:1034B0000A80437892B263F3451222F040020A80F8
:1034C00000780C282BD2DFE800F02A06090E11162E
:1034D000191C1F220C2742F0110009E042F01D00C8
:1034E00008800020704742F0110012E042F0100006
:1034F00040F00200F4E742F01000F1E742F0010072
:10350000EEE742F0010004E042F00200E8E742F09A
:10351000020040F00400E3E742F00400E0E7072087
:1035200070472DE9FF478AB00025BDF82C60824620
:103530001C4691468DF81C50700703D56068FDF756
:10354000C2FE68B9CD4F4FF0010897F82E0058B170
:1035500097F82F00022807D16068FDF701FF18B126
:1035600010200EB0BDE8F087300702D5A089802872
:103570003ED8700705D4B9F1000F02D097F82400A7
:10358000A0B3E07DC0F300108DF81B00627D072022
:10359000032162B3012A2DD0022AE2D0042AE0D10D
:1035A0008DF81710F00628D4A27D07202AB3012A2F
:1035B00023D0022A24D0042AD3D18DF8191000BFB9
:1035C0008DF81590606810B307A9FFF7ABFE0028CF
:1035D000C7D19DF81C00FF2816D0606850F8011F65
:1035E000CDF80F108088ADF8130014E000E001E082
:1035F0000720B6E78DF81780D4E78DF81980DFE74C
:1036000002208DF81900DBE743F20220A9E7CDF88C
:103610000F50ADF81350E07B40B9207C30B9607C8E
:1036200020B9A07C10B9E07CC00601D0062098E744
:103630008DF800A0BDF82C00ADF80200A068019044
:10364000A068029004F10F0001F03EFC8DF80C0020
:10365000FFF791FE8DF80D009DF81C008DF80E000F
:103660008DF816508DF81850E07D08A900F00F0075
:103670008DF81A0068460EF015F805F053FD70E756
:10368000F0B58FB000258DF830508DF814508DF8BE
:10369000345006468DF828500195029503950495FF
:1036A00019B10FC901AC84E80F00744CA07805284B
:1036B00001D004280CD101986168884200D120B95A
:1036C0000398E168884203D110B108200FB0F0BD23
:1036D000207DC00601D51F2700E0FF273B460DAA2D
:1036E00005A903A8FFF7ABFD0028EFD1A08AC10709
:1036F00002D0C00600D4EE273B460AAA0CA901A8B6
:10370000FFF79DFD0028E1D19DF81400C00701D00E
:103710000A20DBE7A08A410708D4A17D31B19DF8DA
:103720002810890702D043F20120CFE79DF8281026
:10373000C90709D0400707D4208818B144F2506166
:10374000884201D90720C1E78DF818508DF819601B
:10375000BDF80800ADF81A000198079006A80DF012
:10376000BBFF05F0DFFC0028B0D18DF820508DF8AC
:103770002160BDF81000ADF822000398099008A858
:103780000DF0C9FF05F0CEFC00289FD101AD241D2E
:1037900095E80F0084E80F00002097E770B586B029
:1037A0000D46040005D0FDF7DBFD20B1102006B06A
:1037B00070BD0820FBE72078C107A98802D0FF2947
:1037C00002D303E01F2901D20920F0E7800763D468
:1037D000FFF75AFC38B12178C1F3C100012804D0A9
:1037E000032802D005E01320E1E7244890F82400E4
:1037F000C8B1C8074FF001064FF0000502D08DF8A0
:103800000F6001E08DF80F50FFF7B5FD8DF8000057
:1038100020786946C0F3C1008DF8010060788DF80A
:103820000250C20801D00720C1E730B3C20701D05F
:103830008DF80260820705D59DF8022042F0020251
:103840008DF80220400705D59DF8020040F00400E5
:103850008DF80200002022780B18C2F38002DA7083
:1038600001EB40026388D380401CA388C0B253811F
:103870000228F0D3207A78B905E001E0EC010020BD
:103880008DF80260E6E7607A30B9A07A20B9E07A74
:1038900010B9207BC00601D0062088E704F108009B
:1038A00001F012FB8DF80E0068460DF0BFFA05F02E
:1038B00039FC002889D18DF810608DF81150E0880E
:1038C000ADF81200ADF8145004A80DF002FB05F09D
:1038D00029FC002888D12078C00701D0152000E0FD
:1038E0001320FFF7BBFB002061E72DE9FF47022013
:1038F000FB4E8DF804000027708EADF80600B84628
:1039000043F202094CE001A80EF0DBFF050006D0EF
:10391000708EA8B3A6F83280ADF806803EE0039C16
:10392000A07F01072DD504F124000090A28EBDF8E0
:103930000800214604F1360301F05FFC050005D0C4
:103940004D452AD0112D3CD0FFDF3AE0A07F20F07A
:103950000801E07F420862F3C711A177810861F393
:103960000000E07794F8210000F01F0084F82000A8
:103970002078282826D129212046FFF7CBFB21E0FB
:1039800014E040070AD5BDF8080004F10E0101F06B
:10399000B1FA05000DD04D4510D100257F1CFFB2B6
:1039A00002200EF0CFFF401CB842ACD8052D11D03C
:1039B00008E0A07F20F00400A07703E0112D00D0E4
:1039C000FFDF0025BDF806007086052D04D02846CF
:1039D00004B0C7E5A6F832800020F9E770B50646C6
:1039E000FFF731FD054605F087FD040000D1FFDF3C
:1039F0006680207820F00F00801C20F0F00020303E
:103A000020700320207295F83E006072BDE870407F
:103A100005F075BD2DE9F04786B0040000D1FFDF49
:103A20002078AF4D20F00F00801C20F0F0007030A7
:103A3000207060680178491F1B2933D2DFE801F04C
:103A4000FE32323255FD320EFDFD42FC323232780A
:103A5000FCFCFBFA3232FCFCF9F8FC00C68830466C
:103A6000FFF7F1FC0546304607F03EF9E0B160682B
:103A7000007A85F83E0021212846FFF74BFB3046AF
:103A8000FEF753FB304603F05BFE3146012012F097
:103A9000D3FCA87F20F01000A877FFF726FF0028AE
:103AA00000D0FFDF06B05DE5207820F0F000203088
:103AB00020700320207266806068007A607205F0D2
:103AC0001EFDD8E7C5882846FFF7BDFC00B9FFDF1B
:103AD00060680079012800D0FFDF6068017A06B0D5
:103AE0002846BDE8F04707F0DEBCC6883046FFF741
:103AF000AAFC050000D1FFDF05F001FD606831463A
:103B00000089288160684089688160688089A8810F
:103B1000012012F091FC0020A875A87F00F003009E
:103B20000228BFD1FFF7E1FE0028BBD0FFDFB9E7D5
:103B300000790228B6D000B1FFDF05F0E0FC66682E
:103B4000B6F806A0307A361D012806D0687E814678
:103B500005F054FA070003D101E0E878F7E7FFDF4A
:103B60000022022150460EF03CFF040000D1FFDF8E
:103B700022212046FFF7CEFA3079012800D002201A
:103B8000A17F804668F30101A177308B2081708B83
:103B90006081B08BA08184F822908DF80880B8688D
:103BA0000090F86801906A46032150460EF019FF14
:103BB00000B9FFDFB888ADF81000B8788DF81200B2
:103BC00004AA052150460EF00CFF00B9FFDFB888AB
:103BD000ADF80C00F8788DF80E0003AA04215046C9
:103BE0000EF0FFFE00B9FFDF062106F1120001F022
:103BF0009FF940B37079800700D5FFDF7179E07DD0
:103C000061F34700E075D6F80600A0617089A083D3
:103C1000062106F10C0001F08BF9F0B195F82500B2
:103C20004108607861F347006070D5F8260006E02F
:103C30003EE036E06DE055E04AE02CE040E0C4F8BC
:103C40000200688D12E0E07D20F0FE00801CE0752F
:103C5000D6F81200A061F08AD9E7607820F0FE0063
:103C6000801C6070F068C4F80200308AE080B8F10F
:103C7000010F04D0B8F1020F05D0FFDF12E70320D7
:103C8000FFF7D4F90EE7287E122800D0FFDF1120BD
:103C9000FFF7E4F906E706B02046BDE8F04701F07B
:103CA00035BD05F02CFC15F8300F40F0020005E0A2
:103CB00005F025FC15F8300F40F004002870F1E6FF
:103CC000287E132809D01528D8D11620FFF7C6F969
:103CD00006B0BDE8F04705F012BC1420F6E700007E
:103CE000EC010020A978052909D00429C6D105F0E6
:103CF00006FC022006B0BDE8F047FFF797B900794F
:103D00000028BBD0E87801F0C6F805F0F8FB0320E6
:103D1000F0E7287E122802D1687E01F0BCF811205D
:103D2000D4E72DE9F047054600784FF00008000978
:103D3000DFF8C0A891460C464646012875D00228F7
:103D400074D007280AD00A2871D0FFDFA9F80060D4
:103D500014B1A4F800806680002003E4696801279C
:103D600004F108000A784FF0020C4FF6FF73172A8F
:103D70007ED00EDC142A32D006DC052A68D0092A4F
:103D800010D0102A75D120E0152A73D0162AF9D147
:103D9000F8E0183A082A6CD2DFE802F0F36B6B0AFD
:103DA000CAF2DFF1C8884FF01208102621468DE1D3
:103DB0004FF01C080A26BCB38888A0806868807908
:103DC00020726868C0796072C0E74FF01B08142643
:103DD00054B30320207268688088A080B6E70A790F
:103DE0003C2AB3D00D1D4FF010082C26E4B1698891
:103DF000A180298B6182298B2182698BA182A98B69
:103E0000E1826B790246A91D1846FFF7ECFA297981
:103E1000002001290CD084F80FC0FF212176E06139
:103E200020626062A06291E70FE02EE151E18CE137
:103E3000E77320760AF1040090E80E00DAF810002B
:103E4000C4E90930C4E9071280E7A9F8006083E7F4
:103E50002C264FF01D08002CF7D00546A380887B48
:103E60002A880F1D60F300022A80887B400802E048
:103E70009DE007E1BEE060F341022A80887B800874
:103E800060F382022A80887BB91CC00860F3C302F9
:103E90002A80B87A0011401C60F3041202F07F00FF
:103EA00028807878AA1CFFF79EFA387D05F1090270
:103EB00007F11501FFF797FA387B01F048F82874ED
:103EC000787B01F044F86874F87EA874787AE87416
:103ED000387F2875B87B6875388AE882DAF81C0064
:103EE000A861B87A524697F808A0C0F34111012999
:103EF00004D0108C504503D2824609E0FFDF10E069
:103F0000022903D0288820F0600009E0504504D140
:103F1000288820F06000403002E0288840F06000EF
:103F20002880A4F824A0524607F11D01A86996E054
:103F300011264FF02008002C87D0A380686804F178
:103F40000A02007920726868007B607269688B1DC4
:103F500048791946FFF747FAF8E60A264FF0210894
:103F6000002CE9D08888A080686880792072686811
:103F7000C07960729AF8301021F004019FE065E08A
:103F80004CE06FE00B264FF02208002CD4D0C888FC
:103F9000A0806868007920726868007A00F0D7FF16
:103FA00060726868407A00F0D2FFA072CEE61C26EC
:103FB0004FF02608002CBFD0A3806868407960725B
:103FC0006868007AA0720AF1040090E80E00DAF83E
:103FD0001000C4E90530C4E90312686800793C2880
:103FE00003D0432803D0FFDFB0E62772AEE684F8A3
:103FF00008C0ABE610264FF02408002C9CD088881F
:10400000A0806868807920816868807A60816868AB
:104010000089A08168688089E08197E610264FF0CA
:104020002308002C88D08888A0806868C0882081F8
:1040300068680089608168684089A08168688089B3
:10404000E0819AF8301021F0020138E030264FF07C
:104050002508002C85D0A38069682822496821F0B2
:104060008DFA73E614264FF01B08002C8ED0A38027
:10407000686800790128BAD02772DAE90710C4E924
:10408000031063E64A46214660E0287A012803D0FF
:10409000022817D0FFDF59E610264FF01F08002C2A
:1040A00089D06888A080A8892081E8896081288AD1
:1040B000A081688AE0819AF8301021F001018AF825
:1040C000301043E64FF012081026688800F01DFFFC
:1040D0003CE6287AC8B3012838D0022836D0032815
:1040E00001D0FFDF32E609264FF01108002C85D001
:1040F0006F883846FFF7A7F990F822A0A780687A62
:104100002072042138460EF087FC052138460EF057
:1041100083FC002138460EF07FFC012138460EF06A
:104120007BFC032138460EF077FC022138460EF066
:1041300073FC062138460EF06FFC072138460EF05E
:104140006BFC504600F0A7FE00E6FFE72846BDE8FE
:10415000F04701F065BC70B5012803D0052800D0F8
:10416000FFDF70BD8DB22846FFF76DF9040000D166
:10417000FFDF20782128F4D005F0BEF980B1017866
:1041800021F00F01891C21F0F00110310170022192
:10419000017245800020A075BDE8704005F0AFB900
:1041A00021462846BDE870401322FFF74FB92DE99C
:1041B000F04116460C00804600D1FFDF307820F039
:1041C0000F00801C20F0F0001030307020780128A3
:1041D00004D0022818D0FFDFBDE8F0814046FFF789
:1041E00032F9050000D1FFDF0320A87505F087F93B
:1041F00094E80F00083686E80F00FE4810F8301FDC
:1042000041F001010170E7E74046FFF71CF90500A6
:1042100000D1FFDFA1884FF6FF700027814202D155
:10422000E288824203D0814201D1E08840B105F0AA
:1042300066F994E80F00083686E80F00AF75CBE703
:10424000A87D0128C8D178230022414612F04AF8FF
:104250000220A875C0E738B505460C460846FDF7AC
:1042600032F818BB203D062D4AD2DFE805F0031BCB
:10427000373C42300021052012F0B4F808B111207B
:1042800038BDA01C0DF023F904F04CFF050038D117
:10429000002208231146052012F024F8052830D00A
:1042A000FFDF2EE06068FDF752F808B1102038BD3E
:1042B000618820886A460DF0C5FB04F033FF0500D5
:1042C0001FD16068E8B1BDF80010018019E0A07846
:1042D00000F0010120880DF0E6FB0EE0206801F0FF
:1042E0004BFE05460DE0207800F001000CF0EDF9E2
:1042F00003E0618820880DF020FB04F013FFF0E755
:104300000725284638BD70B505460C460846FDF71A
:1043100000F808B1102070BD202D07D0212D0DD040
:10432000222D0BD0252D09D0072070BD2088A11C7F
:104330000CF0A0FABDE8704004F0F4BE062070BD99
:10434000AC482530704708B53421AA4821F0B7F9A8
:104350000120FEF76BFE1120FEF780FEA54968469E
:10436000263105F05FF8A3489DF8002010F8251FBE
:1043700062F3470121F001010170002141724FF405
:104380006171A0F8071002218172FEF7B1FE00B141
:10439000FFDFFDF75DF801F084F908BD10B50C46AC
:1043A0004021204621F069F9A07F20F00300A0778A
:1043B000202020700020A07584F8230010BD7047D5
:1043C0002DE9FC410746FCF77EFF10B11020BDE847
:1043D000FC81884E06F12501D6F825000090B6F83C
:1043E0002950ADF8045096F82B408DF80640384619
:1043F000FEF7E2FF0028EAD1FEF77AFE0028E6D0B9
:10440000009946F8251FB580B471E0E710B5044661
:10441000FCF77FFF08B1102010BD76487549224691
:1044200090F8250026314008FEF7DDFF002010BD82
:104430003EB504460D460846FCF76BFF08B1102058
:104440003EBD14B143F204003EBD6A4880780528A1
:1044500003D0042801D008203EBD694602A80AF016
:10446000AEFA2A4669469DF80800FEF7BCFF002018
:104470003EBDFEB50D4604004FF0000711D00822E6
:10448000FEF7C2FE002811D1002608E054F82600ED
:104490006946FEF747FF002808D1761CF6B2AE4207
:1044A000F4D30CF059F810B143F20320FEBD514E85
:1044B00086F824700CB300271BE000BF54F82700D7
:1044C00002A9FEF72FFF00B1FFDF9DF808008DF86D
:1044D000000054F8270050F8011FCDF80110808823
:1044E000ADF8050068460CF05CF800B1FFDF7F1CFA
:1044F000FFB2AF42E2D386F824500020FEBD2DE982
:10450000F0478AB01546894604001ED00F4608229F
:104510002946FEF779FE002811D1002613E000BFDE
:1045200054F826006946103000F0DAFC002806D165
:104530003FB157F82600FCF7C6FE10B110200AB0B4
:104540000BE4761CF6B2AE42EAD30026A5F10108D0
:104550001CE000BF06F1010A0AF0FF0712E000BFED
:1045600054F82600017C4A0854F827100B7CB2EB63
:10457000530F05D106221130113120F0D3FF58B16D
:104580007F1CFFB2AF42EBD30AF0FF064645E1DBEA
:104590004E4624B1012003E043F20520CFE700207E
:1045A0000CF024F810B90CF02DF810B143F20420EF
:1045B000C5E774B300270DF1170828E054F8270069
:1045C0006946103000F08CFC00B1FFDF54F8270082
:1045D000102250F8111FCDF801108088ADF80500A9
:1045E00054F827100DF1070020F0C8FFAEB156F8BF
:1045F000271001E0EC0100201022404620F0BEFF11
:1046000068460BF0B3FF00B1FFDF7F1CFFB2AF4283
:10461000D4D3FEF733FF002091E7404601F0A0FC21
:10462000EEE730B585B00446FCF74DFE18B960687A
:10463000FCF796FE10B1102005B030BD60884AF23C
:10464000B811884206D82078F84D28B1012806D044
:10465000022804D00720EFE7FEF74AFD18E0607853
:10466000022804D0032802D043F20220E4E785F8B0
:104670002F00C1B200200090ADF8040002292CD018
:10468000032927D0FFDF68460CF055F804F04AFDF7
:104690000028D1D1606801F056FC207858B1012083
:1046A0008DF800000DF1010001F05AFC68460DF094
:1046B0005EFA00B1FFDF207885F82E00FEF7DEFEFF
:1046C000608860B1A88580B20BF088FF00B1FFDF81
:1046D0000020B1E78DF80500D5E74020FAE74FF458
:1046E0006170EFE710B50446FCF713FE20B960686F
:1046F00038B1FCF72CFE08B1102010BD606801F045
:104700002FFCCA4830F82C1F6180C1786170807816
:104710002070002010BD2DE9F84314468946064656
:10472000FCF7F7FDA0B94846FCF71AFE80B9204611
:10473000FCF716FE60B9BD4DA878012800D13CB148
:104740003178FF2906D049B143F20400BDE8F8836F
:104750001020FBE7012801D00420F7E7CCB305289F
:1047600011D004280FD069462046FEF7A0FE00288D
:10477000ECD1217D49B1012909D0022909D00329B1
:1047800009D00720E2E70820E0E7024604E0012222
:1047900002E0022200E00322804623461746002062
:1047A0000099FEF7BEFE0028D0D1A0892880A07B0A
:1047B000E875BDF80000A882AF75BDF800100907C4
:1047C00001D5A18931B1A1892980C00704D0032076
:1047D00003E006E08021F7E70220FEF727FC86F8D9
:1047E00000804946BDE8F8430020FEF749BF7CB58C
:1047F0008E4C05460E46A078022803D0032801D02F
:1048000008207CBD15B143F204007CBD07200EF0EA
:10481000A1F810B9A078032806D0FEF735FC28B11E
:10482000A078032804D009E012207CBD13207CBDB1
:10483000304600F013FB0028F9D1E670FEF79BFD2F
:1048400009F0FAFF01208DF800008DF801008DF8C5
:1048500002502088ADF80400E07D8DF8060068461F
:104860000DF02EF804F05EFC0028E0D1A0780328BB
:1048700004D00420FEF7DAFB00207CBDE07800F0D5
:10488000FDFA0520F6E71CB510B143F204001CBD8B
:10489000664CA078042803D0052801D008201CBD50
:1048A00000208DF8000001218DF801108DF8020024
:1048B00068460DF005F804F035FC0028EFD1A0782B
:1048C000052805D05FF00200FEF7B0FB00201CBDFC
:1048D000E07800F0E0FA0320F6E72DE9FC4180469D
:1048E0000E4603250846FCF73BFD002866D14046EE
:1048F000FEF7A9FD040004D02078222804D2082065
:1049000065E543F2020062E5A07F00F003073EB1D7
:10491000012F0CD000203146FEF751FC0500EFD1ED
:10492000012F06D0022F1AD0FFDF28464FE50120C5
:10493000F1E7A07D3146022801D011B107E0112036
:1049400045E56846FCF791FE0028D9D16946404606
:1049500006F06CFD0500E8D10120A075E5E7A07D1B
:10496000032804D1314890F83000C00701D02EB39D
:104970000EE026B1A07F40071ED4002100E00121F7
:10498000404606F073FD0500CFD1A075002ECCD0B7
:104990003146404600F0AEFA05461128C5D1A07F49
:1049A0004107C2D4316844F80E1F7168616040F05D
:1049B000040020740025B8E71125B6E7102006E5AD
:1049C00070B50C460546FEF73EFD010005D02246B7
:1049D0002846BDE87040FEF739BD43F2020070BDC5
:1049E00010B5012807D1114B9B78012B00D011B1D4
:1049F00043F2040010BD0BF023FEBDE8104004F0AC
:104A000091BB012300F051BA00231A46194600F069
:104A10004CBA70B506460C460846FCF754FC18B96B
:104A20002068FCF776FC18B1102070BDEC01002066
:104A3000F84D2A7E112A04D0132A00D33EB1082053
:104A4000F3E721463046FEF7A9FE60B1EDE7092005
:104A5000132A0DD0142A0BD0A188FF29E5D31520E5
:104A6000FEF7FCFA0020D4E90012C5E90712DCE7E2
:104A7000A1881F29D9D31320F2E71CB5E548007E91
:104A8000132801D208201CBD00208DF800006846C4
:104A90000CF01FFA04F046FB0028F4D11120FEF7B9
:104AA000DDFA00201CBD2DE9F04FDFF868A3814638
:104AB00091B09AF818009B4615460C46132803D36C
:104AC000FFF7DBFF00281FD12046FCF7FCFBE8BB0B
:104AD0002846FCF7F8FBC8BB20784FF00107C00759
:104AE0004FF0000102D08DF83A7001E08DF83A10D5
:104AF00020788846C0F3C1008DF8000060788DF8FA
:104B00000910C10803D0072011B0BDE8F08FB0B381
:104B1000C10701D08DF80970810705D59DF80910EE
:104B200041F002018DF80910400705D59DF80900F4
:104B300040F004008DF809009DF80900810703D5B5
:104B400040F001008DF80900002000E015E06E46FD
:104B500006EB400162884A81401CA288C0B20A82EA
:104B60000328F5D32078C0F3C100012825D00328FD
:104B700023D04846FCF7A7FB28B11020C4E7FFE785
:104B80008DF80970D8E799F80000400808D001288E
:104B900009D0022807D0032805D043F20220B3E74A
:104BA0008DF8028001E08DF80270484650F8011F30
:104BB000CDF803108088ADF80700FEF7DCFB8DF818
:104BC00001000021424606EB41002B88C3826B881E
:104BD0008383AB884384EB880385491CC285C9B2B3
:104BE00082860329EFD3E088ADF83C0068460CF0DC
:104BF000B5FA002887D19AF818005546112801D037
:104C0000082081E706200DF0A5FE38B12078C0F31A
:104C1000C100012804D0032802D006E0122073E767
:104C200095F8240000283FF46EAFFEF72DFA022815
:104C300001D2132068E7584600F010F900289DD1F2
:104C400085F819B068460CF0C9FB04F06BFA040053
:104C500094D1687E00F012F91220FEF7FFF9204689
:104C600052E770B56B4D287E122801D00820DCE693
:104C70000CF0B7FB04F056FA040005D1687E00F092
:104C80000AF91120FEF7EAF92046CEE670B506468D
:104C900015460C460846FCF73CFB18B92846FCF7BD
:104CA00038FB08B11020C0E62A46214630460CF0F9
:104CB000A9FE04F037FA0028F5D121787F29F2D136
:104CC0000520B2E67CB505460C460846FCF7FBFA23
:104CD00008B110207CBD2846FEF7B5FB20B1007856
:104CE000222804D208207CBD43F202007CBD494842
:104CF00090F83000400701D511207CBD2078C00815
:104D000002D16078C00801D007207CBDADF800500A
:104D100020788DF8020060788DF803000220ADF84D
:104D2000040068460BF0B6FF04F0FCF97CBD70B5DA
:104D300086B014460D460646FEF785FB28B100787E
:104D4000222805D2082006B06FE643F20200FAE7F7
:104D50002846FCF705FB20B944B12046FCF7F7FADA
:104D600008B11020EFE700202060A080294890F8CB
:104D70003000800701D51120E5E703A930460BF08C
:104D8000CCFD10B104F0CEF9DDE7ADF80060BDF860
:104D90001400ADF80200BDF81600ADF80400BDF82F
:104DA0001000BDF81210ADF80600ADF808107DB186
:104DB000298809B1ADF80610698809B1ADF802106B
:104DC000A98809B1ADF80810E98809B1ADF8041057
:104DD000DCB1BDF80610814201D9081A2080BDF867
:104DE0000210BDF81400814201D9081A6080BDF894
:104DF0000800BDF80410BDF816200144BDF81200EB
:104E00001044814201D9081AA08068460BF044FE84
:104E1000B8E70000EC0100201CB554490968CDE951
:104E2000001068460CF09CF904F07CF91CBD1CB520
:104E300000200090019068460CF092F904F072F99D
:104E40001CBD10800888508048889080C8881081D8
:104E50008888D080002050819081704710B504462A
:104E600004F0CCF830B1407830B1204604F0EBFBD0
:104E7000002010BD052010BD122010BD10B504F09B
:104E8000BDF8040000D1FFDF607800B9FFDF607873
:104E9000401E607010BD10B504F0B0F8040000D1E1
:104EA000FFDF6078401C607010BD1CB5ADF80000DD
:104EB0008DF802308DF803108DF8042068460CF050
:104EC00064FD04F02FF91CBD0CB529A2D2E9001233
:104ED000CDE900120079694601EB501000780CBD55
:104EE0000278520804D0012A02D043F2022070470F
:104EF000FEF718BA1FB56A46FFF7A3FF68460CF025
:104F0000A3FA04F00FF904B010BD70B50C0006460A
:104F10000DD0FEF798FA050000D1FFDFA6802889A2
:104F20002081288960816889A081A889E0817CE549
:104F300010B500231A4603E0845C2343521CD2B20E
:104F40008A42F9D30BB1002010BD012010BD00B57D
:104F500040B1012805D0022803D0032804D0FFDF88
:104F6000002000BDFF2000BD042000BD645A0200E7
:104F7000070605040302010010B50446FCF7A3F977
:104F800008B1102010BD2078C0F30210042807D803
:104F90006078072804D3A178102901D8814201D272
:104FA000072010BDE078410706D421794A0703D4D1
:104FB000000701D4080701D5062010BD002010BD50
:104FC00010B513785C08837F64F3C7138377137875
:104FD0009C08C37F64F30003C3771078C309487843
:104FE00063F34100487013781C090B7864F347138E
:104FF0000B701378DB0863F3000048705078487139
:1050000010BD10B5C4780B7864F300030B70C4783E
:10501000640864F341030B70C478A40864F382034A
:105020000B70C478E40864F3C3030B700379117840
:1050300063F30001117003795B0863F341011170A0
:1050400003799B0863F3820111700079C00860F353
:10505000C301117010BD70B514460D46064604F02C
:105060004BFA80B10178182221F00F01891C21F040
:10507000F001A03100F8081B214620F0C4FABDE879
:10508000704004F03CBA29463046BDE87040132217
:10509000FEF7DCB92DE9F047064608A8894690E8F6
:1050A00030041F4690461421284620F008FB0021BA
:1050B000CAF80010B8F1000F03D0B9F1000F03D106
:1050C00014E03878C00711D02068FCF722F9C0BB83
:1050D000B8F1000F07D12068123028602068143022
:1050E00068602068A8602168CAF8001038788007D6
:1050F00024D56068FCF72BF918BBB9F1000F21D05B
:10510000FFF71EF90168C6F868118188A6F86C11CE
:10511000807986F86E0101F0F8FCF94FEF60626863
:1051200062B196F8680106F2691140081032FEF784
:105130005AF910223946606820F020FA0020BDE8B4
:10514000F08706E0606820B1E8606068C6F8640136
:10515000F4E71020F3E730B5054608780C4620F058
:105160000F00401C20F0F001103121700020607011
:1051700095F8230030B104280FD0052811D0062857
:1051800014D0FFDF20780121B1EB101F04D295F875
:10519000200000F01F00607030BD21F0F0002030D2
:1051A00002E021F0F00030302070EBE721F0F00059
:1051B0004030F9E7F0B591B0022715460C46064697
:1051C0003A46ADF80870092103AB05F004F80490E5
:1051D000002810D004208DF804008DF80170E03410
:1051E000099605948DF818500AA968460FF0F2F850
:1051F00000B1FFDF012011B0F0BD10B588B00C4642
:105200000A99ADF80000C3B11868CDF802005868DB
:10521000CDF80600ADF80A20102203A820F0AEF960
:1052200068460CF081F903F07DFF002803D1A17FCF
:1052300041F01001A17708B010BD0020CDF80200A8
:10524000E6E72DE9F84F0646808A0D4680B2824691
:10525000FEF7F9F804463078DFF8A48200274FF013
:105260000209A8F120080F2870D2DFE800F06FF2E1
:105270003708387D8CC8F1F0EFF35FF3F300A07FBF
:1052800000F00300022809D05FF0000080F0010167
:1052900050460DF0AFFB050003D101E00120F5E71A
:1052A000FFDF98F85C10C90702D0D8F860000BE067
:1052B000032105F11D0010F0E0FDD5F81D00914916
:1052C000B0FBF1F201FB1200C5F81D0070686867C1
:1052D000B068A8672078252800D0FFDFCAE0A07F4B
:1052E00000F00300022809D05FF0000080F0010107
:1052F00050460DF07FFB060003D101E00120F5E7E9
:10530000FFDF3078810702D52178252904D040F0CD
:1053100001003070BDE8F88F85F80090307F28716B
:1053200006F11D002D36C5E90206F3E7A07F00F067
:105330000300022808D0002080F0010150460DF043
:1053400059FB040004D102E00120F5E7A7E1FFDFEB
:105350002078C10604D5072028703D346C60D9E759
:1053600040F008002070D5E7E07F000700D5FFDFA0
:10537000307CB28800F0010301B05046BDE8F04F28
:10538000092105F0B3BD04B9FFDF716821B1102216
:1053900004F1240020F0F2F828212046FDF7BAFE9F
:1053A000A07F00F0030002280ED104F124000023A6
:1053B00000901A4621465046FFF71FFF112807D0DC
:1053C00029212046FDF7A6FE307A84F82000A1E7C7
:1053D000A07F000700D5FFDF14F81E0F40F0080083
:1053E0002070E782A761E761C109607861F341003D
:1053F000014660F382016170307AE0708AE7A07F35
:1054000000F00300022809D05FF0000080F00101E5
:1054100050460DF0EFFA040003D101E00120F5E75A
:10542000FFDF022104F1850010F027FD0420287021
:1054300004F5B4706860B4F88500288230481038EC
:105440007C346C61C5E9028064E703E024E15BE041
:105450002DE015E0A07F00F00300022807D0002017
:1054600080F0010150460DF0C5FA18B901E00120A5
:10547000F6E7FFDF324621465046BDE8F84FEAE541
:1054800004B9FFDF20782128A1D93079012803D180
:10549000E07F40F00800E077324621465046FFF7B3
:1054A000DAFD2046BDE8F84F2321FDF733BE3279FF
:1054B000AA8005F108030921504604F08CFEE8603B
:1054C00010B10520287025E7A07F00F00300022816
:1054D00008D0002080F0010150460DF08BFA040046
:1054E00003D101E00120F5E7FFDF04F162010223AF
:1054F0001022081F0DF005F907703179417009E796
:105500004C02002040420F00A07F00F00300022860
:1055100008D0002080F0010150460DF06BFA050024
:1055200003D101E00120F5E7FFDF95F8840000F0EA
:10553000030001287AD1A07F00F00307E07F10F07C
:10554000010602D0022F04D133E095F8A000C00775
:105550002BD0D5F8601121B395F88320087C62F335
:1055600087000874A17FCA09D5F8601162F3410071
:105570000874D5F8601166F300000874AEB1D5F870
:105580006001102204F1240188351FF0F7FF287E06
:1055900040F001002876287820F0010005F88809FD
:1055A00000E016B1022F04D02DE095F88800C00766
:1055B00027D0D5F85C1121B395F88320087C62F3DD
:1055C00087000874A17FCA09D5F85C1162F3410015
:1055D0000874D5F85C1166F3000008748EB1D5F834
:1055E0005C01102204F1240188351FF0C7FF2878E0
:1055F00040F0010005F8180B287820F0010005F8AC
:10560000A009022F44D0002000EB400005EBC000B1
:1056100090F88800800709D595F87C00D5F86421BA
:10562000400805F17D011032FDF7DDFE8DF8009098
:1056300095F884006A4600F003008DF8010095F8A3
:1056400088108DF8021095F8A0008DF8030021460F
:10565000504601F043FA2078252805D0212807D0AC
:10566000FFDF2078222803D922212046FDF752FDB2
:10567000A07F00F0030002280CD0002080F0010180
:1056800050460DF0C9F900283FF44FAEFFDF41E668
:105690000120B9E70120F1E7706847703AE6FFDFC3
:1056A00038E670B5FE4C002584F85C5025660EF097
:1056B0005EFE04F11001204603F0DAFE84F830505B
:1056C00070BD70B50D46FDF7BEFE040000D1FFDFD2
:1056D0004FF4B87128461FF0F2FF04F1240028614E
:1056E000A07F00F00300022808D0012105F1E000AE
:1056F0000EF03EFE002800D0FFDF70BD0221F5E76E
:105700000A46014602F1E0000EF052BE70B50546B1
:10571000406886B001780A2906D00D2933D00E29B9
:105720002FD0FFDF06B070BD86883046FDF78BFEB8
:10573000040000D1FFDF20782128F3D028281BD1D6
:10574000686802210E3001F0BEF9A8B1686808212E
:10575000801D01F0B8F978B104F1240130460CF055
:10576000B1F803F0DFFC00B1FFDF06B02046BDE872
:1057700070402921FDF7CEBC06B0BDE8704003F0B3
:10578000BEBE012101726868C6883046FDF75BFE27
:10579000040000D1FFDFA07F00F00301022902D145
:1057A00020F01000A077207821280AD06868017ABC
:1057B00009B1007980B1A07F00F00300022862D017
:1057C000FFDFA07F00F003000228ABD1FEF78DF8C9
:1057D0000028A7D0FFDFA5E703F091FEA17F080610
:1057E0002BD5E07FC00705D094F8200000F01F0003
:1057F000102820D05FF0050084F8230020782928A5
:105800001DD02428DDD13146042010F015FE2221C0
:105810002046FDF77FFCA07F00F00300022830D077
:105820005FF0000080F0010130460DF0F5F800282F
:10583000C7D0FFDFC5E70620DEE70420DCE701F084
:105840000300022808D0002080F0010130460DF04E
:10585000D1F8050003D101E00120F5E7FFDF2521A4
:105860002046FDF757FC03208DF80000694605F13E
:10587000E0000EF094FD0228A3D00028A1D0FFDFA5
:105880009FE70120CEE703F03AFE9AE72DE9F043C7
:1058900087B09946164688460746FDF7D4FD0400B2
:1058A0004BD02078222848D3232846D0E07F000719
:1058B00043D4A07F00F00300022809D05FF000006D
:1058C00080F0010138460DF095F8050002D00CE09B
:1058D0000120F5E7A07F00F00300022805D0012198
:1058E000002238460DF07DF805466946284601F04D
:1058F0001CF9009800B9FFDF45B10098E03505615B
:105900002078222806D0242804D007E0009900201F
:10591000086103E025212046FDF7FCFB00980121EA
:1059200041704762868001A9C0E902890EF052FDEC
:10593000022802D0002800D0FFDF07B0BDE8F083C6
:1059400070B586B00546FDF77EFD017822291ED987
:10595000807F00F00300022808D0002080F00101C1
:1059600028460DF047F804002FD101E00120F5E7AB
:10597000FFDF2AE0B4F85E0004F1620630440178EB
:10598000427829B121462846FFF714FCB0B9C9E690
:10599000ADF804200921284602AB04F01CFC03905A
:1059A0000028F4D005208DF80000694604F1E000DD
:1059B0000EF0F5FC022801D000B1FFDF0223102217
:1059C000314604F15E000CF0D2FEB4F8600000280D
:1059D000D0D1A7E610B586B00446FDF734FD0178B6
:1059E00022291BD9807F00F00300022808D0002064
:1059F00080F0010120460CF0FDFF040003D101E01E
:105A00000120F5E7FFDF06208DF80000694604F16C
:105A1000E0000EF0C4FC002800D0FFDF06B010BD8F
:105A20002DE9F05F05460C460027007890460109F5
:105A30003E4604F1080BBA4602297DD0072902D060
:105A40000A2909D146E0686801780A2905D00D299C
:105A500030D00E292ED0FFDFBBE114271C26002CEE
:105A60006BD08088A080FDF7EEFC5FEA000900D1D2
:105A7000FFDF99F817005A46400809F11801FDF7B1
:105A8000B2FC6868C0892082696851F8060FC4F8C2
:105A900012004868C4F81600A07E20F0060001E05D
:105AA0002C02002040F00100A07699F81E0040F082
:105AB00020014DE01A270A26002CD1D0C088A080F2
:105AC000FDF7C1FC050000D1FFDF59462846FFF76E
:105AD00042FB7EE10CB1A88BA080287A0B287DD0F8
:105AE00006DC01287BD0022808D0032804D135E049
:105AF0000D2875D00E2874D0FFDF6AE11E27092615
:105B0000002CADD0A088FDF79EFC5FEA000900D113
:105B1000FFDF287B00F003000128207A1BD020F053
:105B200001002072297B890861F341002072297BE2
:105B3000C90861F3820001E041E1F2E02072297BB3
:105B4000090961F3C300207299F81E0040F040017A
:105B500089F81E103DE140F00100E2E713270D2611
:105B6000002CAAD0A088FDF76EFC8146807F00F053
:105B70000300022808D0002080F00101A0880CF06A
:105B800039FF050003D101E00120F5E7FFDF99F8B7
:105B90001E0000F00302022A50D0686F817801F0E5
:105BA00003010129217A4BD021F001012172837870
:105BB0009B0863F3410121728378DB0863F3820160
:105BC000217283781B0963F3C3012172037863F3A5
:105BD00006112172437863F3C71103E061E0A9E085
:105BE00090E0A1E0217284F809A0C178A172022A94
:105BF00029D00279E17A62F30001E1720279520858
:105C000062F34101E1720279920862F38201E1726A
:105C10000279D20862F3C301E1724279217B62F317
:105C2000000121734279520862F3410121734279E4
:105C3000920862F382012173407928E0A86FADE7F2
:105C400041F00101B2E74279E17A62F30001E172C9
:105C50004279520862F34101E1724279920862F39B
:105C60008201E1724279D20862F3C301E1720279E2
:105C7000217B62F3000121730279520862F3410132
:105C800021730279920862F3820121730079C008BE
:105C900060F3C301217399F80000232831D926212C
:105CA00040E018271026E4B3A088FDF7CCFB83461C
:105CB000807F00F00300022809D0002080F001015D
:105CC000A0880CF097FE5FEA000903D101E00120F3
:105CD000F4E7FFDFE868A06099F8000040F00401F5
:105CE00089F8001099F80100800708D50120207379
:105CF0009BF8000023286CD92721584651E084F8EE
:105D00000CA066E015270F265CB1A088FDF79BFB71
:105D1000814606225946E86808F0CBFA0120A073B4
:105D2000A0E041E048463CE016270926E4B3287B82
:105D300020724EE0287B19270E26ACB3C4F808A0C9
:105D4000A4F80CA0012807D0022805D0032805D00C
:105D5000042803D0FFDF0DE0207207E0697B0428F0
:105D600001F00F0141F0800121721ED0607A20F015
:105D700003006072A088FDF766FB054600782128C5
:105D800027D0232800D0FFDFA87F00F003000228DF
:105D900013D0002080F00101A0880CF03DFE2221EC
:105DA0002846FDF7B7F914E004E0607A20F003001C
:105DB000401CDEE7A8F8006010E00120EAE70CB123
:105DC0006888A080287A68B301280AD002284FD0BA
:105DD000FFDFA8F800600CB1278066800020BDE8D6
:105DE000F09F15270F26002CE4D0A088FDF72BFB91
:105DF000807F00F00300022808D0002080F001011D
:105E0000A0880CF0F7FD050003D101E00120F5E7C3
:105E1000FFDFD5F81D000622594608F04AFA84F83B
:105E20000EA0D6E717270926002CC3D0A088FDF7BF
:105E30000AFB8146807F00F00300022808D0002082
:105E400080F00101A0880CF0D5FD050003D101E030
:105E50000120F5E7FFDF6878800701D5022000E028
:105E60000120207299F800002328B2D9272159E790
:105E700019270E26002C9DD0A088FDF7E4FA5FEAD2
:105E8000000900D1FFDFC4F808A0A4F80CA084F832
:105E900008A0A07A40F00300A07299F81E10C9096A
:105EA00061F38200A07299F81F2099F81E1012EA7F
:105EB000D11F05D099F8201001F01F0110292BD017
:105EC00020F00800A07299F81F10607A61F3C300F7
:105ED0006072697A01F003010129A2D140F0040047
:105EE000607299F81E0000F003000228E87A16D0CC
:105EF000217B60F300012173AA7A607B62F30000CA
:105F00006073EA7A520862F341012173A97A490861
:105F100061F3410060735CE740F00800D2E7617B09
:105F200060F300016173AA7A207B62F300002073A2
:105F3000EA7A520862F341016173A97A490861F370
:105F40004100207345E710B5FE4C30B101461022E8
:105F500004F120001FF012FB012084F8300010BD76
:105F600010B5044600F0D1FDF64920461022BDE8E8
:105F7000104020311FF002BB70B5F24D06004FF00B
:105F8000000413D0FBF79FF908B110240CE00621A0
:105F9000304608F075F9411C05D028665FF0010015
:105FA00085F85C0000E00724204670BD0020F7E77C
:105FB000007810F00F0204D0012A05D0022A0CD17B
:105FC00010E0000909D10AE00009012807D00228E1
:105FD00005D0032803D0042801D00720704708709B
:105FE000002070470620704705282AD2DFE800F01D
:105FF00003070F171F00087820F0FF001EE0087845
:1060000020F00F00401C20F0F000103016E008785F
:1060100020F00F00401C20F0F00020300EE0087847
:1060200020F00F00401C20F0F000303006E008782F
:1060300020F00F00401C20F0F000403008700020DD
:106040007047072070472DE9F041804688B00D4623
:1060500000270846FBF784F9A8B94046FDF7F3F995
:10606000040003D02078222815D104E043F2020076
:1060700008B0BDE8F08145B9A07F410603D500F026
:106080000300022801D01020F2E7A07FC10601D44E
:10609000010702D50DB10820EAE7E17F090701D524
:1060A0000D20E5E700F00300022805D125B12846C0
:1060B000FEF762FF0700DBD1A07F00F0030002289B
:1060C00008D0002080F0010140460CF093FC06004F
:1060D00002D00FE00120F5E7A07F00F003000228C6
:1060E0000ED0002080F00101002240460CF079FC27
:1060F000060007D0A07F00F00300022804D009E0CA
:106100000120EFE70420B3E725B12A4631462046B7
:10611000FEF756FF6946304600F007FD009800B9CB
:10612000FFDF0099022006F1E0024870C1F82480E8
:106130004A6100220A81A27F02F00302022A1CD0D7
:1061400001200871287800F00102087E62F3010046
:1061500008762A78520862F3820008762A78920834
:1061600062F3C30008762A78D20862F30410087636
:1061700024212046FCF7CEFF33E035B30871301DF3
:1061800088613078400908777078C0F3400048771C
:10619000287800F00102887F62F301008877A27FEF
:1061A000D20962F382008877E27F62F3C3008877C6
:1061B000727862F304108877A878C87701F1210219
:1061C00028462031FEF71DFF03E00320087105205B
:1061D000087625212046FCF79DFFA07F20F0400097
:1061E000A07701A900980EF0F5F8022801D000B1BF
:1061F000FFDF38463CE72DE9FF4F534A0D4699B083
:106200009A4607CA0AAB002783E807001998FDF7EA
:106210001AF9060006D03078262806D008201DB0CE
:10622000BDE8F08F43F20200F9E7B07F00F0030908
:10623000B9F1020F0AD05DB91B98FEF79DFE002848
:10624000EDD1B07F00F00300022801D11B9890BB74
:10625000B07F00F00300022808D0002080F0010188
:1062600019980CF0C7FB040003D101E00120F5E709
:10627000FFDF852D28D007DCF5B1812D1ED0822DC2
:106280001ED0832D08D11DE0862D1FD0882D1FD054
:10629000892D1FD08A2D1FD00F2020710F281DD0CF
:1062A00003F02AF9E0B101208DF83C00201D109088
:1062B0002079B8B15BE111E00020EEE70120ECE7C6
:1062C0000220EAE70320E8E70520E6E70620E4E706
:1062D0000820E2E70920E0E70A20DEE707209EE742
:1062E00011209CE7B9F1020F03D0A56F03D1A06F75
:1062F00002E0656FFAE7606F804632D04FF0010030
:1063000001904FF002000090214630461B9AFEF7A4
:1063100057FE1B98007800F00101A87861F3010096
:10632000A870B17FC90961F38200A870F17F61F3A1
:10633000C300A870617861F30410A8702078400948
:10634000287003E02C0200206C5A02006078C0F331
:10635000400068701B988078E87000206871287190
:1063600003E00220019001200090A87898F8021024
:10637000C0F3C000C1F3C00108405FEA000B2DD09C
:106380005046FAF7A0FF78BBDAF80C00FAF79BFF4B
:1063900050BBDAF81C00FAF796FF28BBDAF80C00BD
:1063A000A060DAF81C00E060607898F8012042EA0A
:1063B000500100BF61F34100607098F80210C0B254
:1063C00000EA111161F3000060700020207700994D
:1063D00006F11700022908D0012107E0607898F83B
:1063E000012002EA5001E5E732E0002104EB8101DF
:1063F00048610199701C022901D0012100E00021AF
:1064000004EB81014861A87800F00300012857D10E
:1064100098F8020000F00300012851D1B9F1020FF1
:1064200004D02A1D691D1B98FEF7EBFD287998F80A
:10643000041008408DF83400697998F8052011405F
:106440008DF8381008433BD05046FAF73CFF08B1AE
:106450001020E4E60AF110010491B9F1020F17D0FF
:106460000846002104F18C03CDE9000304F5AE7267
:1064700002920DAB5A462046FEF70CFE0028E8D1EA
:10648000B9F1020F08D0504608D14FF0010107E0E2
:1064900050464FF00101E5E70498F5E74FF00001A1
:1064A00004F1A403CDE9000304F5B072029281F077
:1064B00001010EAB5A462046FEF7ECFD0028C8D17C
:1064C0006078800734D4A87898F80210C0F3800070
:1064D000C1F3800108432BD0297898F800000AAA5C
:1064E000B9F1020F06D032F811204300DA4002F071
:1064F00003070AE032F810204B00DA4012F00307DD
:1065000005D0012F0BD0022F0BD0032F07D0BBF1EA
:10651000000F0DD0012906D0042904D008E002277D
:10652000F5E70127F3E7012801D0042800D104276B
:10653000B07F40F08000B077F17F6BF30001F1771E
:106540006078800706D50320A071BBF1000F0ED143
:10655000002028E00220022F18D0012F18D0042F8D
:1065600029D00020A071B07F20F08000B0772521D5
:106570003046FCF7CFFD0FA904F1E0000DF00FFF4E
:1065800010B1022800D0FFDF002048E6A071DFE74D
:10659000A0710D2104F120001FF091F8207840F047
:1065A0000200207001208DF85C0017AA314619986E
:1065B00000F094FADBE70120A071D8E72DE9F04361
:1065C00087B09046894604460025FCF73CFF06004C
:1065D00006D03078272806D0082007B0BDE8F08321
:1065E00043F20200F9E7B07F00F00300022809D06F
:1065F0005FF0000080F0010120460CF0FBF9040080
:1066000003D101E00120F5E7FFDFA7795FEA090088
:1066100005D0012821D0B9F1020F26D110E0B8F140
:10662000000F22D1012F05D0022F05D0032F05D056
:10663000FFDF2DE00C252BE0012529E0022527E0D6
:106640004046FAF740FEB0B9032F0ED11022414662
:1066500004F11D001EF092FF1AE0012F02D0022F5C
:1066600003D104E0B8F1000F12D00720B5E740468F
:10667000FAF729FE08B11020AFE7102104F11D0040
:106680001EF0FBFF0621404607F0FAFDC4F81D008E
:106690002078252140F0020020703046FCF73AFDBA
:1066A0002078C10713D020F00100207002208DF85F
:1066B000000004F11D0002908DF804506946C330BB
:1066C0000DF06DFE022803D010B1FFDF00E025774A
:1066D000002082E730B587B00D460446FCF7B3FED4
:1066E000A0B1807F00F00300022812D05FF000000C
:1066F00080F0010120460CF07DF904000ED0284600
:10670000FAF7E1FD38B1102007B030BD43F20200C6
:10671000FAE70120ECE72078400701D40820F3E7EE
:10672000294604F13D00202205461EF027FF20786F
:1067300040F01000207001070FD520F008002070F5
:1067400007208DF80000694604F1E00001950DF086
:1067500026FE022801D000B1FFDF0020D4E770B58B
:106760000D460646FCF76FFE18B10178272921D1A6
:1067700002E043F2020070BD807F00F003000228B7
:1067800008D0002080F0010130460CF033F90400FD
:1067900003D101E00120F5E7FFDFA079022809D14C
:1067A0006078C00706D02A4621463046FEF702FD33
:1067B00010B10FE0082070BDB4F860000E280BD2B5
:1067C00004F1620102231022081F0BF09AFF01213D
:1067D00001704570002070BD112070BD70B5064677
:1067E00014460D460846FAF76EFD18B92046FAF72A
:1067F00090FD08B1102070BDA6F57F40FF380ED087
:106800003046FCF720FE38B1417822464B08811C07
:106810001846FCF7E8FD07E043F2020070BD204691
:10682000FDF7F4FD0028F9D11021E01D0FF025FB44
:10683000E21D294604F1170000F087F9002070BD21
:106840002DE9F04104468AB01546884600270846DF
:10685000FAF786FD18B92846FAF782FD10B1102024
:106860000AB006E42046FCF7EEFD060003D03078BF
:1068700027281AD102E043F20200F1E7B07F00F0CE
:106880000300022808D0002080F0010120460CF00F
:10689000B1F8040003D101E00120F5E7FFDF207823
:1068A000400702D56078800701D40820D8E7B07F80
:1068B00000F00300022803D0A06F03D1A16F02E013
:1068C000606FFAE7616F407800B19DB1487810B110
:1068D000B8F1000F0ED0ADB1EA1D06A8E16800F0D6
:1068E00034F9102206A905F117001EF01BFE18B19D
:1068F000042707E00720B3E71022E91D04F12D006B
:106900001EF03CFEB8F1000F06D0102208F107017E
:1069100004F11D001EF032FE2078252140F0020017
:1069200020703046FCF7F6FB2078C10715D020F028
:106930000100207002208DF8000004F11D0002907B
:10694000103003908DF804706946B3300DF027FDC8
:10695000022803D010B1FFDF00E0277700207FE797
:10696000F8B515460E460746FCF76DFD040004D049
:106970002078222804D00820F8BD43F20200F8BD98
:10698000A07F00F00300022802D043F20500F8BD0A
:106990003046FAF798FC18B92846FAF794FC08B183
:1069A0001020F8BD00953288B31C21463846FEF70A
:1069B00024FC112815D00028F3D1297C4A08A17F96
:1069C00062F3C711A177297CE27F61F30002E277CD
:1069D000297C890884F82010A17F21F04001A1774B
:1069E000F8BDA17F0907FBD4D6F80200C4F8360031
:1069F000D6F80600C4F83A003088A086102229464E
:106A000004F124001EF0BAFD287C4108E07F61F308
:106A10004100E077297C61F38200E077287C8008E0
:106A200084F82100A07F40F00800A0770020D3E781
:106A300070B50D4606460BB1072070BDFCF703FD8F
:106A4000040007D02078222802D3A07F800604D437
:106A5000082070BD43F2020070BDADB1294630463A
:106A60000AF030FF02F05EFB297C4A08A17F62F346
:106A7000C711A177297CE27F61F30002E277297CCC
:106A8000890884F8201004E030460AF03EFF02F046
:106A900049FBA17F21F02001A17770BD70B50D46A3
:106AA000FCF7D1FC040005D02846FAF732FC20B1EF
:106AB000102070BD43F2020070BD29462046FEF74B
:106AC0004AFB002070BD04E010F8012B0AB1002041
:106AD0007047491E89B2F7D20120704770B515463C
:106AE000064602F009FD040000D1FFDF207820F007
:106AF0000F00801C20F0F000203020706680286895
:106B0000A060BDE8704002F0FABC10B5134C94F8D8
:106B10003000002808D104F12001A1F110000DF08F
:106B200080FC012084F8300010BD10B190F8B9202D
:106B30002AB10A4890F8350018B1002003E0B830B7
:106B400001E0064834300860704708B50023009320
:106B500013460A460CF049F908BD00002C0200203B
:106B600018B18178012938D101E0102070470188DF
:106B700042F60112881A914231D018DC42F6010225
:106B8000A1EB020091422AD00CDC41B3B1F5C05F09
:106B900025D06FF4C050081821D0A0F57060FF38E0
:106BA0001BD11CE001281AD002280AD117E0B0F549
:106BB000807F14D008DC012811D002280FD00328D0
:106BC0000DD0FF2809D10AE0B0F5817F07D0A0F5EC
:106BD0008070033803D0012801D0002070470F20B7
:106BE00070470A281FD008DC0A2818D2DFE800F016
:106BF000191B1F1F171F231D1F21102815D008DC6C
:106C00000B2812D00C2810D00D2816D00F2806D132
:106C10000DE011280BD084280BD087280FD003203B
:106C200070470020704705207047072070470F20ED
:106C3000704704207047062070470C20704743F2CD
:106C40000200704738B50C46050041D06946FFF791
:106C5000AFF9002819D19DF80010607861F30200A7
:106C600060706946681CFFF7A3F900280DD19DF8F4
:106C70000010607861F3C5006070A978C1F341012C
:106C8000012903D0022905D0072038BD217821F041
:106C9000200102E0217841F020012170410704D059
:106CA000A978C90861F386106070607810F0380F19
:106CB00007D0A978090961F3C710607010F0380F88
:106CC00002D16078400603D5207840F04000207063
:106CD000002038BD70B50446002008801546606865
:106CE000FFF7B0FF002816D12089A189884211D86A
:106CF00060688078C0070AD0B1F5007F0AD840F2FA
:106D00000120B1FBF0F200FB1210288007E0B1F582
:106D1000FF7F01D90C2070BD01F2012129800020E4
:106D200070BD10B50478137864F300031370047811
:106D3000640864F3410313700478A40864F38203C5
:106D400013700478E40864F3C3031370047824090F
:106D500064F3041313700478640964F34513137027
:106D60000078800960F38613137031B10878C10789
:106D700001D1800701D5012000E0002060F3C71396
:106D8000137010BD4278530702D002F0070306E0EB
:106D900012F0380F02D0C2F3C20300E001234A7898
:106DA00063F302024A70407810F0380F02D0C0F34B
:106DB000C20005E0430702D000F0070000E0012018
:106DC00060F3C5024A7070472DE9F04F95B00D0091
:106DD000824612D0122128461EF04FFC4FF6FF7B50
:106DE00005AA0121584607F066F8002426463746D2
:106DF0004FF420586FF4205973E0102015B0BDE80F
:106E0000F08F00BF9DF81E0001280AD1BDF81C10AC
:106E100041450BD011EB09000AD001280CD0022803
:106E20000CD0042C0ED0052C0FD10DE0012400E075
:106E30000224BDF81A6008E0032406E00424BDF82B
:106E40001A7002E0052400E00624BDF81A1051452E
:106E500047D12C74BEB34FF0000810AA4FF0070AB8
:106E6000CDE90282CDE900A80DF13C091023CDF84F
:106E7000109042463146584607F0D0F808BBBDF89E
:106E80003C002A46C0B210A90DF041FBC8B9AE8142
:106E9000CFB1CDE900A80DF1080C0AAE40468CE850
:106EA0004102132300223946584607F0B7F840B98B
:106EB000BDF83C00F11CC01EC0B22A1D0DF027FB1E
:106EC00010B103209AE70AE0BDF82900E881062CFA
:106ED00005D19DF81E00A872BDF81C002881002075
:106EE0008CE705A806F0F3FF00288BD0FFF779FEAA
:106EF00084E72DE9F0471C46DDE90978DDF82090AC
:106F000015460E00824600D1FFDF0CB1208818B173
:106F1000D5B11120BDE8F087022D01D0012100E09C
:106F2000002106F1140005F0B5FEA8F800000246A5
:106F30003B462946504603F04EF9C9F8000008B90F
:106F4000A41C3C600020E5E71320E3E7F0B41446FE
:106F5000DDE904528DB1002314B1022C09D101E006
:106F6000012306E00D7CEE0703D025F00105012387
:106F70000D742146F0BC03F0B9BF1A80F0BC704715
:106F80002DE9FE4F91461A881C468A468046FAB182
:106F900002AB494603F01FF9050019D04046A61C74
:106FA00027880BF06BFE3246072629463B460096A3
:106FB0000BF079FA20882346CDE900504A46514625
:106FC0004046FFF7C3FF002020800120BDE8FE8F70
:106FD0000020FBE72DE9F04786B082460EA89046D8
:106FE00090E8B000894604AA05A903A88DE8070027
:106FF0001E462A4621465046FFF77BFF039901B102
:1070000001213970002818D1F94904F1140204ABA8
:107010000860039805998DE80700424649465046A6
:1070200006F0EFF9A8B1092811D2DFE800F0050851
:107030000510100A0C0C0E00002006B06AE71120A3
:10704000FBE70720F9E70820F7E70D20F5E7032025
:10705000F3E7BDF810100398CDE9000133462A4646
:1070600021465046FFF772FFE6E72DE9F04389B06D
:107070000D46DDE9108781461C461646142103A8FB
:107080001EF01DFB012002218DF810108DF80C0060
:107090008DF81170ADF8146064B1A278D20709D0F0
:1070A0008DF81600E088ADF81A00A088ADF8180039
:1070B000A068079008A80095CDE90110424603A9F1
:1070C00048466B68FFF786FF09B0BDE8F083F0B56E
:1070D0008BB000240646069407940727089405A859
:1070E0000994019400970294CDE903400D461023C2
:1070F0002246304606F092FF78B90AA806A9019404
:1071000000970294CDE90310BDF8143000222946FF
:10711000304606F059FD002801D0FFF762FD0BB0A4
:10712000F0BD06F0F9BB2DE9FC410C468046002677
:1071300002F0E2F9054620780D287DD2DFE800F064
:10714000BC0713B325BD49496383AF959B00A8488D
:10715000006820B1417841F010014170ADE0404637
:1071600002F0FAF9A9E0042140460BF043FC0700C5
:1071700000D1FFDF07F11401404605F01FFDA5BB5C
:1071800013214046FDF71CFC97E0042140460BF01C
:1071900031FC070000D1FFDFE088ADF800000020DF
:1071A000B8819DF80000010704D5C00602D5A0886B
:1071B000B88105E09DF8010040067ED5A088F881E1
:1071C00005B9FFDF22462946404601F0BDFC0226F4
:1071D00073E0E188ADF800109DF8011009060FD5A5
:1071E000072803D006280AD00AE024E004214046FC
:1071F0000BF000FC060000D1FFDFA088F081022622
:10720000CDB9FFDF17E0042140460BF0F3FB070088
:1072100000D1FFDF07F1140006F0B5FB90F0010F7D
:1072200002D1E079000648D5387C022640F0020001
:10723000387405B9FFDF00E03EE0224629464046AB
:1072400001F082FC39E0042140460BF0D3FB017CC5
:10725000002D01F00206C1F340016171017C21F0B3
:1072600002010174E7D1FFDFE5E702260121404674
:1072700002F0A4F921E0042140460BF0BBFB0546D7
:10728000606800902089ADF80400012269464046FC
:1072900002F0B5F9287C20F0020028740DE0002DE2
:1072A000C9D1FFDFC7E7022600214046FBF70CF9F2
:1072B000002DC0D1FFDFBEE7FFDF3046BDE8FC8117
:1072C0003EB50C0009D001466B4601AA002006F02D
:1072D00027FF20B1FFF785FC3EBD10203EBD0020FA
:1072E0002080A0709DF8050002A900F00700FEF7BD
:1072F0007BFE50B99DF8080020709DF8050002A99A
:10730000C0F3C200FEF770FE08B103203EBD9DF839
:10731000080060709DF80500C109A07861F30410B1
:10732000A0709DF80510890961F3C300A0709DF855
:107330000410890601D5022100E0012161F3420019
:107340009DF8001061F30000A07000203EBD70B5F4
:10735000144606460D4651EA040005D075B10846AC
:10736000F9F7F5FF78B901E0072070BD29463046EE
:1073700006F037FF10B1BDE8704032E454B120464A
:10738000F9F7E5FF08B1102070BD21463046BDE891
:10739000704095E7002070BD2DE9FC5F0C469046DB
:1073A0000546002701780822007A3E46B2EB111FFD
:1073B0007ED104F10A0100910A31821E4FF0020AC7
:1073C00004F1080B0191092A73D2DFE802F0ECDF27
:1073D00005F427277AA9CD00688804210BF00AFB61
:1073E000060000D1FFDFB08920B152270726C2E096
:1073F0009002002051271026002C7DD06888A080A4
:107400000120A071A88900220099FFF7A0FF0028A1
:1074100073D1A8892081288AE081D1E0B5F8129043
:10742000072824D1E87B000621D5512709F1140053
:1074300086B2002CE1D0A88900220099FFF787FFCF
:1074400000285AD16888A08084F806A0A8892081E5
:107450000120A073288A2082A4F81290A88A0090A4
:1074600068884B46A969019A01F04BFBA8E05027B8
:1074700009F1120086B2002C3ED0A889002259469C
:10748000FFF765FF002838D16888A080A889E080D0
:10749000287A072813D002202073288AE081E87B0D
:1074A000C0096073A4F81090A88A0090688801E071
:1074B00083E080E04B4604F11202A969D4E7012081
:1074C000EAE7B5F81290512709F1140086B2002CB2
:1074D00066D0688804210BF08DFA83466888A08006
:1074E000A88900220099FFF732FF00286ED184F8A6
:1074F00006A0A889208101E052E067E00420A07383
:10750000288A2082A4F81290A88A009068884B46A6
:10751000A969019A01F0F5FAA989ABF80E104FE0BC
:107520006888FBF790FF0746688804210BF062FA31
:10753000064607B9FFDF06B9FFDF687BC00702D048
:107540005127142601E0502712264CB36888A080EA
:10755000502F06D084F806A0287B594601F0E1FAA6
:107560002EE0287BA11DF9E7FE49A88949898142BF
:1075700005D1542706269CB16888A08020E05327B7
:107580000BE06888A080A889E08019E06888042161
:107590000BF030FA00B9FFDF55270826002CF0D198
:1075A000A8F8006011E056270726002CF8D068885C
:1075B000A080002013E0FFDF02E0012808D0FFDFF9
:1075C000A8F800600CB1278066800020BDE8FC9F11
:1075D00057270726002CE3D06888A080687AA0711E
:1075E000EEE7401D20F0030009B14143091D01EB06
:1075F0004000704713B5DB4A00201071009848B175
:10760000002468460BF013F8002C02D1D64A0099EA
:1076100011601CBD01240020F4E770B50D4606463C
:1076200086B014465C2128461EF049F804B9FFDFF5
:10763000A0786874A2782188284601F09CFA00207E
:10764000A881E881228805F11401304605F09BFAF3
:107650006A460121304606F02EFC19E09DF8030031
:10766000000715D5BDF806103046FFF730FD9DF830
:107670000300BDF8061040F010008DF80300BDF8BF
:107680000300ADF81400FF233046059A06F074FDA0
:10769000684606F01CFC0028E0D006B070BD10B5AE
:1076A0000C4601F1140005F0A5FA0146627C204663
:1076B000BDE8104001F094BA30B50446A94891B035
:1076C0004FF6FF75C18905AA284606F0F4FB30E0A5
:1076D0009DF81E00A0422AD001282AD1BDF81C0026
:1076E000B0F5205F03D042F60101884221D100208D
:1076F00002AB0AAA0CA9019083E8070007200090BA
:10770000BDF81A1010230022284606F087FC38B96D
:10771000BDF828000BAAC0B20CA90CF0F8FE10B1FD
:10772000032011B030BD9DF82E00A04201D10020F1
:10773000F7E705A806F0CBFB0028C9D00520F0E745
:1077400070B5054604210BF055F9040000D1FFDFA8
:1077500004F114010C46284605F030FA214628466B
:10776000BDE8704005F031BA70B58AB00C460646E7
:10777000FBF769FE050014D02878222827D30CB126
:10778000A08890B101208DF80C0003208DF8100026
:1077900000208DF8110054B1A088ADF818002068C1
:1077A00007E043F202000AB070BD0920FBE7ADF824
:1077B00018000590042130460BF01CF9040000D19C
:1077C000FFDF04F1140005F02CFA000701D40820B3
:1077D000E9E701F091FE60B108A802210094CDE92B
:1077E000011095F8232003A930466368FFF7F2FBE8
:1077F000D9E71120D7E72DE9F04FB2F802A0834670
:1078000089B0154689465046FBF71DFE0746042100
:1078100050460BF0EFF80026044605964FF002089C
:107820000696ADF81C6007B9FFDF04B9FFDF4146DB
:10783000504603F0C6FE50B907AA06A905A88DE870
:1078400007004246214650466368FFF752FB454811
:1078500007AB0660DDE9051204F11400CDF80090D5
:10786000CDE90320CDE9013197F823205946504650
:107870006B6805F01FFA06000AD0022E04D0032E12
:1078800014D0042E00D0FFDF09B03046BDE8F08FE1
:10789000BDF81C000028F7D00599CDE9001042463C
:1078A000214650466368FFF751FBEDE7687840F0EA
:1078B00008006870E8E72DE9F04F99B004464FF0F2
:1078C00000082848ADF81C80ADF82080ADF8248071
:1078D000A0F80880ADF81480ADF81880ADF82C80C1
:1078E000ADF82880007916460D464746012808D095
:1078F000022806D0032804D0042802D0082019B09A
:10790000C4E72046F9F7DFFC80BB2846F9F7DBFC2B
:1079100060BB6068F9F724FD40BB606848B16089CE
:107920002189884202D8B1F5007F01D90C20E6E711
:1079300080460EAA06A92846FFF7CCF90028DED11A
:1079400068688078C0F34100022808D19DF81900CA
:1079500010F0380F03D02869F9F7F9FC30B905A900
:10796000206904E0900200201400002020E0FFF7CE
:1079700069F90028C3D1206948B1607880079DF873
:10798000150000F0380001D5F0B300E0E0BB9DF831
:10799000140080060ED59DF8150010F0380F03D0A6
:1079A0006068F9F7D4FC18B96068F9F7D9FC08B138
:1079B0001020A4E70AA96069FFF744F900289ED1C6
:1079C000606940B19DF8290000F0070101293CD110
:1079D00010F0380F39D00BA9A069FFF733F9002850
:1079E0008DD19DF8280080062FD49DF82C008006AC
:1079F0002BD4A06950B19DF82D0000F0070101299A
:107A000023D110F0380F00E01FE01ED0E06818B15D
:107A10000078D0B11C2818D20FAA611C2046FFF7AD
:107A200080F90121384661F30F2082468DF852100B
:107A3000B94642F603000F46ADF850000DF13F0283
:107A400018A928680CF082FD08B1072057E79DF8B7
:107A5000600015A9CDF80090C01CCDE9019100F09F
:107A6000FF0B00230BF20122514614A806F066F921
:107A7000F0BBBDF854000C90FD492A89286900929A
:107A8000CDE901016B89BDF838202868069906F018
:107A900055F901007ED120784FF0020AC10601D4C9
:107AA00080062BD5ADF80C90606950B90AA906A8DC
:107AB000FFF768F99DF8290020F00700401C8DF8B9
:107AC00029009DF8280008A940F0C8008DF828007A
:107AD0008DF8527042F60210ADF8500003AACDF8AE
:107AE00000A0CDE90121002340F2032214A800E008
:107AF0001EE00A9906F022F901004BD1DC484D4600
:107B000008385B460089ADF83D000FA8CDE902902A
:107B1000CDF80490CDF810904FF007090022CDF871
:107B20000090BDF854104FF6FF7006F04DF810B1FC
:107B3000FFF757F8E3E69DF83C00000625D52946F7
:107B4000012060F30F218DF852704FF42450ADF8EE
:107B50005000ADF80C5062789DF80C00002362F3E1
:107B600000008DF80C006278CDF800A0520862F396
:107B700041008DF80C0003AACDE9012540F2032253
:107B800014A806F0DBF8010004D1606888B320690E
:107B9000A8B900E086E005A906A8FFF7F3F8607829
:107BA000800706D49DF8150020F038008DF81500E8
:107BB00005E09DF8140040F040008DF814008DF8A9
:107BC000527042F60110ADF85000208940F20121B8
:107BD000B0FBF1F201FB1202606809ABCDF8008046
:107BE000CDE90103002314A8059906F0A7F80100C8
:107BF00058D12078C00729D0ADF80C50A06950B9F1
:107C00000BA906A8FFF7BEF89DF82D0020F007008D
:107C1000401C8DF82D009DF82C008DF8527040F01E
:107C200040008DF82C0042F60310ADF8500007A973
:107C300003AACDF800A0CDE90121002340F20322E0
:107C400014A80B9906F07AF801002BD1E06868B30C
:107C50002946012060F30F218DF8527042F604107E
:107C6000ADF85000E068002302788DF85820407885
:107C70008DF85900E06816AA4088ADF85A00E0680F
:107C800000798DF85C00E068C088ADF85D00CDF843
:107C90000090CDE901254FF4027214A806F04EF8C9
:107CA000010003D00C9800F0C7FF28E670480321BC
:107CB0000838017156B100893080BDF82400708009
:107CC000BDF82000B080BDF81C00F080002016E652
:107CD00070B501258AB016460B46012802D002284D
:107CE00016D104E08DF80E504FF4205003E08DF8CB
:107CF0000E5042F60100ADF80C005BB10024601C90
:107D000060F30F2404AA08A918460CF01FFC18B150
:107D1000072048E5102046E504A99DF82020544896
:107D2000CDE90021801E02900023214603A802F223
:107D3000012206F003F810B1FEF753FF33E54C487B
:107D400008380EB1C1883180057100202BE5F0B5EF
:107D500093B0074601268DF83E6041F60100ADF86C
:107D60003C0012AA0FA93046FFF7B2FF002848D105
:107D70003F4C0025083CE7B31C2102A81DF09FFCE6
:107D80009DF808008DF83E6040F020008DF8080056
:107D900042F60520ADF83C000E959DF83A0011958D
:107DA00020F00600801C8DF83A009DF838006A46E5
:107DB00020F0FF008DF838009DF8390009A920F067
:107DC000FF008DF839000420ADF82C00ADF830002C
:107DD0000EA80A9011A80D900FA80990ADF82E508A
:107DE00002A8FFF768FD00280BD1BDF800006081F4
:107DF00000E008E0BDF80400A081401CE08125718E
:107E0000002013B0F0BD6581A581BDF84800F4E7FE
:107E10002DE9F74F1649A0B00024083917940A79C4
:107E2000A146012A04D0022A02D0082023B02DE561
:107E3000CA88824201D00620F8E721988A46824209
:107E400001D10720F2E701202146ADF848004FF6A6
:107E5000FF788DF86E0042F6020B60F30F21ADF84B
:107E60004A80ADF86CB006918DF8724002E00000D7
:107E7000980200201CA9ADF870401391ADF8508015
:107E800012A806F048F800252E462F460DAB072213
:107E900012A9404606F042F878B10A285DD195B3A0
:107EA0008EB3ADF86450ADF866609DF85E008DF855
:107EB000144019AC012864D06BE09DF83A001FB360
:107EC000012859D1BDF8381059451FD118A809A962
:107ED00001940294CDE9031007200090BDF83610FC
:107EE00010230022404606F099F8B0BBBDF86000B0
:107EF000042801D006284AD1BDF8241021988142D7
:107F00003AD10F2092E73AE0012835D1BDF8380088
:107F1000B0F5205F03D042F6010188422CD1BAF8B7
:107F20000600BDF83610884201D1012700E0002785
:107F300005B19EB1219881421ED118A809AA0194C9
:107F40000294CDE90320072000900D461023002263
:107F5000404606F063F800B902E02DE04E460BE023
:107F6000BDF86000022801D0102810D1C0B217AAB5
:107F700009A90CF0CCFA50B9BDF8369086E7052077
:107F800054E705A917A8221D0CF0E0FA08B1032058
:107F90004CE79DF814000023001DC2B28DF8142098
:107FA00022980092CDE901401BA8069905F0C6FE73
:107FB00010B902228AF80420FEF713FE36E710B546
:107FC0000B46401E88B084B205AA00211846FEF771
:107FD000A8FE00200DF1080C06AA05A901908CE866
:107FE0000700072000900123002221464FF6FF7072
:107FF00005F0EAFD0446BDF81800012800D0FFDFB7
:108000002046FEF7EEFD08B010BDF0B5F74F044670
:1080100087B038790E46032804D0042802D00820FF
:1080200007B0F0BD04AA03A92046FEF753FE0500E1
:10803000F6D160688078C0F3410002280AD19DF82B
:108040000D0010F0380F05D02069F9F780F908B15C
:108050001020E5E7208905AA21698DE807006389DA
:10806000BDF810202068039905F068FE10B1FEF7F6
:10807000B8FDD5E716B1BDF8140030800420387182
:108080002846CDE7F8B50C0006460CD001464FF661
:10809000FF7500236A46284606F042F828B100BF63
:1080A000FEF79FFDF8BD1020F8BD69462046FEF79B
:1080B000C9FD0028F8D1A078314600F00103284618
:1080C000009A06F059F8EBE730B587B01446002265
:1080D0000DF1080C05AD01928CE82C0007220092EE
:1080E0000A46014623884FF6FF7005F06DFDBDF886
:1080F00014102180FEF775FD07B030BD70B50D4638
:1081000004210AF077FC040000D1FFDF294604F1C6
:108110001400BDE8704004F07DBD70B50D4604212B
:108120000AF068FC040000D1FFDF294604F11400C6
:10813000BDE8704004F091BD70B50D4604210AF011
:1081400059FC040000D1FFDF294604F11400BDE80A
:10815000704004F0A9BD70B5054604210AF04AFC40
:10816000040000D1FFDF214628462368BDE87040A7
:108170000122FEF705BF70B5064604210AF03AFC5D
:10818000040000D1FFDF04F1140004F033FD401DB2
:1081900020F0030511E0011D00880022431821464C
:1081A0003046FEF7EDFE00280BD0607CABB2684392
:1081B00082B2A068011D0AF0DAFAA068418800299D
:1081C000E9D170BD70B5054604210AF013FC040026
:1081D00000D1FFDF214628466368BDE870400222D7
:1081E000FEF7CEBE70B50E46054601F085F90400D7
:1081F00000D1FFDF0120207266726580207820F0B8
:108200000F00001D20F0F00040302070BDE87040ED
:1082100001F075B910B50446012900D0FFDF2046F2
:10822000BDE810400121FAF74FB92DE9F04F97B0A2
:108230004FF0000A0C008346ADF814A0D04619D0C8
:10824000E06830B1A068A8B10188ADF81410A0F8BA
:1082500000A05846FBF7F7F8070043F2020961D087
:10826000387822285CD3042158460AF0C3FB050065
:1082700005D103E0102017B0BDE8F08FFFDF05F156
:10828000140004F0B7FC401D20F00306A07801287C
:1082900003D0022801D00720EDE7218807AA58461D
:1082A00005F009FE30BB07A805F011FE10BB07A8BA
:1082B00005F00DFE48B99DF82600012805D1BDF84E
:1082C0002400A0F52451023902D04FF45050D2E7D7
:1082D000E068B0B1CDE902A00720009005AACDF872
:1082E00004A00492A2882188BDF81430584605F0F5
:1082F0006BFC10B1FEF775FCBDE7A168BDF814007A
:1083000008809DF81F00C00602D543F20140B2E785
:108310000B9838B1A1780078012905D080071AD4CC
:108320000820A8E74846A6E7C007F9D002208DF844
:108330003C00A8684FF00009A0B1697C42887143F5
:1083400091420FD98AB2B3B2011D0AF0C6F9804634
:10835000A0F800A006E003208DF83C00D5F80080CE
:108360004FF001099DF8200010F0380F00D1FFDF19
:108370009DF820001E49C0F3C200084497F823105E
:1083800010F8010C884201D90F2074E72088ADF85D
:10839000400014A90095CDE90191434607220FA999
:1083A0005846FEF717FE002891D19DF8500050B9AD
:1083B000A078012807D1687CB3B2704382B2A86864
:1083C000011D0AF09EF9002055E770B506461546D6
:1083D0000C460846FEF7C4FB002805D12A46214674
:1083E0003046BDE8704073E470BD11E59002002096
:1083F000765A020070B51E4614460D0009D044B1ED
:10840000616831B138B1FC49C988814203D0072085
:1084100070BD102070BD2068FEF7A2FB0028F9D1C6
:10842000324621462846BDE87040FFF744BA70B591
:1084300015460C0006D038B1EF490989814203D0B6
:10844000072070BD102070BD2068FEF789FB002852
:10845000F9D129462046BDE87040D6E570B50646FC
:1084600086B00D4614461046F8F753FFD0BB60683F
:10847000F8F776FFB0BBA6F57F40FF3803D0304653
:10848000FAF7E1FF80B128466946FEF79DFC002817
:108490000CD19DF810100F2008293DD2DFE801F023
:1084A00008060606060A0A0843F2020006B070BD76
:1084B0000320FBE79DF80210012908D1BDF8001048
:1084C000B1F5C05FF2D06FF4C052D142EED09DF84A
:1084D000061001290DD1BDF80410A1F52851062977
:1084E00007D200E029E0DFE801F0030304030303FF
:1084F000DCE79DF80A1001290FD1BDF80810B1F58D
:10850000245FD3D0A1F60211B1F50051CED00129DC
:10851000CCD0022901D1C9E7FFDF606878B9002318
:1085200005AA2946304605F0FBFD10B1FEF759FBC0
:10853000BCE79DF81400800601D41020B6E76188DE
:10854000224628466368FFF7BFFDAFE72DE9F043F9
:10855000814687B0884614461046F8F7DAFE18B10F
:10856000102007B0BDE8F083002306AA4146484624
:1085700005F0D6FD18B100BFFEF733FBF1E79DF81B
:108580001800C00602D543F20140EAE7002507279C
:1085900005A8019500970295CDE9035062884FF632
:1085A000FF734146484605F039FD060013D1606867
:1085B000F8F7AFFE60B960680195CDE90250009709
:1085C0000495238862884146484605F027FD064603
:1085D000BDF8140020803046CEE739B1864B0A88BA
:1085E0009B899A4202D843F2030070471DE610B5FA
:1085F00086B0814C0423ADF81430638943B1A4895B
:108600008C4201D2914205D943F2030006B010BD5D
:108610000620FBE7ADF81010002100910191ADF8A4
:10862000003002218DF8021005A9029104A90391DE
:10863000ADF812206946FFF7F8FDE7E72DE9FC47A2
:1086400081460D460846F8F73EFE88BB4846FAF7D5
:10865000FAFE5FEA00080AD098F80000222829D321
:10866000042148460AF0C6F9070005D103E043F2A9
:108670000200BDE8FC87FFDF07F1140004F0D1FA27
:1086800006462878012803D0022804D00720F0E706
:10869000B0070FD502E016F01C0F0BD0A8792C1DE7
:1086A000C00709D0E08838B1A068F8F70CFE18B10F
:1086B0001020DEE70820DCE721882A780720B1F5C2
:1086C000847F35D01EDC40F20315A1F20313A942CA
:1086D00026D00EDCB1F5807FCBD003DCF9B10129C7
:1086E00026D1C6E7A1F58073013BC2D0012B1FD173
:1086F00013E0012BBDD0022B1AD0032BB9D0042BD1
:1087000016D112E0A1F20912082A11D2DFE802F014
:108710000B04041010101004ABE7022AA9D007E0E4
:10872000012AA6D004E0320700E0F206002AA0DA0F
:10873000CDB200F0E1FE50B198F82300CDE900057C
:10874000FA89234639464846FEF78FFC91E7112007
:108750008FE72DE9F04F8BB01F4615460C46834638
:108760000026FAF770FE28B10078222805D20820EA
:108770000BB081E543F20200FAE7B80801D0072008
:10878000F6E7032F00D100274FF6FF79CCB1022D79
:1087900073D32046F8F7E4FD30B904EB0508A8F1DF
:1087A0000100F8F7DDFD08B11020E1E7AD1EAAB227
:1087B0002146484605F08FFD38F8021C88425CD1FE
:1087C000ADB20D49B80702D58889401C00E00120F0
:1087D0001FFA80F8F80701D08F8900E04F4605AAFC
:1087E0004146584605F067FB4FF0070A4FF0000975
:1087F000DCB320460BE000009002002040881028E7
:108800003BD8361D304486B2AE4236D2A01902881B
:108810004245F3D351E000BF9DF8170002074CD545
:1088200094B304EB0608361DB8F80230B6B2102B2C
:1088300023D89A19AA4220D8B8F8002091421CD116
:10884000C0061CD5CDE900A90DF1080C0AAAA11992
:1088500048468CE80700B8F800100022584605F09A
:10886000B3F920B1FEF7BDF982E726E005E0B8F8DC
:108870000200BDF82810884201D00B2078E7B8F834
:108880000200304486B207E0FFE7C00604D5584630
:10889000FEF71DFC002888D19DF81700BDF81A10BE
:1088A00020F010008DF81700BDF81700ADF800009B
:1088B000FF235846009A05F05FFC05A805F007FB6A
:1088C00018B9BDF81A10B942A6D9042158460AF0C1
:1088D00091F8040000D1FFDFA2895AB1CDE900A9C7
:1088E0004D46002321465846FEF7BFFB0028BBD16A
:1088F000A5813DE700203BE72DE9FF4F8BB01E46E9
:1089000017000D464FF0000412D0B00802D0072027
:108910000FB0B1E4032E00D100265DB10846F8F790
:1089200016FD28B93888691E0844F8F710FD08B10B
:108930001020EDE7C64AB00701D5D18900E001213A
:10894000F0074FF6FF7802D0D089401E00E0404685
:1089500086B206AA0B9805F0AEFA4FF000094FF068
:10896000070B0DF1140A38E09DF81B00000734D501
:10897000CDF80490CDF800B0CDF80890CDE9039A79
:10898000434600220B9805F049FB60BB05B3BDF8D8
:1089900014103A8821442819091D8A4230D3BDF8A1
:1089A0001E2020F8022BBDF8142020F8022BCDE960
:1089B00000B9CDE90290CDF810A0BDF81E10BDF8A9
:1089C000143000220B9805F029FB08B103209FE723
:1089D000BDF814002044001D84B206A805F077FA03
:1089E00020B10A2806D0FEF7FCF891E7BDF81E106A
:1089F000B142B9D934B17DB13888A11C884203D2C3
:108A00000C2085E7052083E722462946404605F0ED
:108A100062FC014628190180A41C3C80002077E7F5
:108A200010B50446F8F775FC08B1102010BD884851
:108A3000C0892080002010BDF0B58BB00D460646E1
:108A4000142103A81CF03BFE01208DF80C008DF8CA
:108A5000100000208DF81100ADF814503046FAF7E0
:108A6000F2FC48B10078222812D30421304609F0E4
:108A7000C1FF040005D103E043F202000BB0F0BDDA
:108A8000FFDF04F11400074604F0CBF8800601D4A0
:108A90000820F3E7207C022140F00100207409A89F
:108AA0000094CDE90110072203A930466368FEF760
:108AB00091FA20B1217C21F001012174DEE72946E1
:108AC0003046F9F7F2FC08A9384604F099F800B1ED
:108AD000FFDFBDF82040172C01D2172000E0204610
:108AE000A84201D92C4602E0172C00D217242146B7
:108AF0003046FFF712FB21463046F9F7FCF900201B
:108B0000BCE7F8B51C4615460E46069F0AF0A4F8C9
:108B10002346FF1DBCB231462A46009409F08FFC63
:108B2000F8BD70B50C4605460E2120461CF0A5FD8B
:108B3000002020802DB1012D01D0FFDF70BD062067
:108B400000E00520A07170BD10B54880087813467C
:108B500020F00F00001D20F0F00080300C4608705F
:108B60001422194604F108001CF04DFD00F0C7FC6A
:108B70003748046010BD2DE9F047DFF8D890491D53
:108B8000064621F0030117460C46D9F8000009F00B
:108B90006CFD050000D1FFDF4FF000083560A5F83F
:108BA00000802146D9F8000009F05FFD050000D1E2
:108BB000FFDF7560A5F800807FB104FB07F1091D98
:108BC0000BD0D9F8000009F050FD040000D1FFDF00
:108BD000B460C4F80080BDE8F087C6F80880FAE702
:108BE0002DE9F0411746491D21F00302194D0646B3
:108BF00001681446286809F063FD224671682868F8
:108C000009F05EFD3FB104FB07F2121D03D0B1680D
:108C1000286809F055FD042009F094FE044604205C
:108C200009F098FE201A012804D12868BDE8F04117
:108C300009F010BDBDE8F08110B50C4605F007F94C
:108C400000B1FFDF2046BDE81040FDF7CABF0000BD
:108C5000900200201400002038B50C468288817BE9
:108C600019B14189914200D90A462280C188121D5A
:108C700090B26A4608F04FFFBDF80000032800D309
:108C80000320C1B2208801F011F838BD38B50C4678
:108C90008288817B19B10189914200D90A462280DC
:108CA000C188121D90B26A4608F035FFBDF8000079
:108CB000022800D30220C1B2208800F0F7FF401C38
:108CC000C0B238BD2DE9FE4F82468B46F9481446A6
:108CD0000BF10302D0E90010CDE9011022F00302EC
:108CE00068464FF49071009209F0A1FCF24E002CFE
:108CF00002D1F24A00999160009901440091357FB8
:108D000005F1010504D1E8B20BF09AFB00B1FFDFD9
:108D1000009800EB0510C01C20F0030100915CB925
:108D2000707AB27A1044C2B200200870308C80B2DF
:108D300004F015FF00B1FFDF0098316A084400908D
:108D40002146684600F075FF80460098C01C20F060
:108D500003000090B37AF27A717A04B1002009F02E
:108D60005CFD0099084400902146684600F0A9FF88
:108D7000D14800273D4690F801900CE0284600F0CD
:108D80003BFF064681788088F9F74CF971786D1CB5
:108D900000FB0177EDB24D45F0D10098C01C20F0EA
:108DA0000300009004B100203946F9F746F9009914
:108DB000002708440090C0483D4690F801900CE020
:108DC000284600F019FF0646C1788088FEF709FCA6
:108DD00071786D1C00FB0177EDB24D45F0D1009824
:108DE000C01C20F00300009004B100203946FEF7BB
:108DF00001FC00994FF0000908440090AE484D4630
:108E000047780EE0284600F0F7FE0646807B30B13A
:108E100006F1080001F019FF727800FB02996D1C41
:108E2000EDB2BD42EED10098C01C20F003000090CE
:108E300004B10020494601F00CFF0099084400905D
:108E40002146684600F0AFFE0098C01D20F00700E4
:108E50000090DAF80010814204D3A0EB0B01B1F5C9
:108E6000803F04DB4FF00408CAF8000004E0CAF8B1
:108E70000000B8F1000F02D04046BDE8FE8F34BBC1
:108E80008F490020009A03F083F8FBF75CFA8A48C8
:108E900001AA00211030F8F7E1FA00B1FFDF86489F
:108EA000407FFEF754FF00B1FFDF83484FF4F671B7
:108EB00040301CF004FC80480421403080F8E91167
:108EC00080F8EA11062180F8EB11032101710020DE
:108ED000D3E770B5784C06464034207804EB401553
:108EE000E078083590B9A01990F8E80100280ED074
:108EF000A0780F2800D3FFDF202128461CF0DFFBDD
:108F0000687866F3020068700120E070284670BD42
:108F10002DE9F04105460C460027007805219046D2
:108F20003E46B1EB101F00D0FFDF287A50B1012878
:108F30000ED0FFDFA8F800600CB12780668000200B
:108F4000BDE8F0810127092674B16888A08008E097
:108F50000227142644B16888A0802869E060A88AA6
:108F60002082287B2072E5E7A8F80060E7E730B5AB
:108F7000514C012000212070617020726072032228
:108F8000A272E07221732174052121831F21618364
:108F900060744CA161610A2121776077474D4FF4DD
:108FA000B06020626868C11C21F00301814200D0DA
:108FB000FFDF6868606030BD30B5404C156863689D
:108FC00010339D4202D20420136030BD3A4B5D78CD
:108FD0005A6802EB0512107051700320D0801720E0
:108FE00090800120D0709070002090735878401CC1
:108FF0005870606810306060002030BD70B5064663
:109000002D480024457807E0204600F0F5FD017862
:10901000B14204D0641CE4B2AC42F5D1002070BD72
:10902000F7B5074608780C4610B3FFF7E7FF05468B
:10903000A7F12006202F06D0052E19D2DFE806F072
:109040000F2B2B151A0000F0E2FD0DB1697800E03E
:109050000021401AA17880B20844FF2808D8A078DF
:1090600030B1A088022831D202E0608817282DD2C2
:109070000720FEBD207AE0B161881729F8D3A188C6
:109080001729F5D3A1790029F2D0E1790029EFD091
:10909000402804D9ECE7242F18D1207A48B1618800
:1090A0004FF6FB70814202D8A18881420ED904207C
:1090B000FEBD0BE07C5A0200AC030020180000202B
:1090C000000000206E5246357800000065B9207817
:1090D00002AA0121FFF770FF0028E9D12078FFF7ED
:1090E0008DFF050000D1FFDF052E18D2DFE806F066
:1090F000030B0E081100A0786870A088E8800FE0CC
:109100006088A8800CE0A078A87009E0A078E870DA
:1091100006E054F8020FA8606068E86000E0FFDF36
:109120000020C5E71A2835D00DDC132832D2DFE83D
:1091300000F01B31203131272723252D31312931F2
:109140003131312F0F00302802D003DC1E2821D10D
:10915000072070473A3809281CD2DFE800F0151BB9
:109160000F1B1B1B1B1B07000020704743F2040052
:10917000704743F202007047042070470D2070478B
:109180000F20704708207047112070471320704748
:10919000062070470320704710B5007800F00100EA
:1091A00008F0ABFCBDE81040BCE710B5007818B182
:1091B000012801D0072010BD08F0EFFCBDE81040E9
:1091C000B0E710B5007800F0010008F09FFCBDE8A2
:1091D0001040A7E70EB5017801F001018DF80010ED
:1091E000417801F001018DF801100178C1F34001CF
:1091F0008DF802104178C1F340018DF80310017819
:1092000089088DF80410417889088DF80510817857
:109210008DF80610C1788DF8071000798DF80800D8
:10922000684607F095FAFFF77DFF0EBD2DE9F84F70
:10923000DFF8F883FE4C00264FF490771FE0012002
:1092400000F082FD0120FFF744FE05463946D8F8BC
:10925000080009F00AFA686000B9FFDF686807F0E3
:1092600006F9B0B12846FAF7D5FB284600F072FDA2
:1092700028B93A466968D8F8080009F021FA94F943
:10928000E9010428DBDA022009F05CFB074600252F
:10929000A5E03A466968D8F8080009F011FAF2E743
:1092A000B8F802104046491C89B2A8F80210B94229
:1092B00001D3002141800221B8F8020009F09AFB95
:1092C000002864D0B8F80200694608F088FBFFF770
:1092D00029FF00B1FFDF9DF8000078B1B8F8020067
:1092E00009F0CCFC5FEA000900D1FFDF484608F036
:1092F0003AFF18B1B8F8020002F052F9B8F80200CB
:1093000009F0AAFC5FEA000900D1FFDF484608F037
:1093100022FFE0BB0321B8F8020009F06BFB5FEA13
:10932000000B47D1FFDF45E0DBF8100010B10078FB
:10933000FF2849D0022000F007FD0220FFF7C9FDF9
:109340008246484609F013F8CAF8040000B9FFDF66
:10935000DAF8040009F0DBF8002100900170B8F899
:1093600002105046AAF8021001F01CFE484609F00F
:10937000D0F800B9FFDF504600F0ECFC18B99AF8BD
:109380000100000704D50098CBF8100012E024E09B
:10939000DBF8100038B10178491C11F0FF010170B1
:1093A00008D1FFDF06E000221146484600F0F9FB35
:1093B00000B9FFDF94F9EA01022805DBB8F80200E2
:1093C00001F0B5FD0028AFD194F9E901042804DBD0
:1093D000484609F002F900B101266D1CEDB2BD420C
:1093E00004D294F9EA010228BFF65AAF002E7FF4A6
:1093F00022AFBDE8F84F032000F0A6BC10B58B4C9F
:10940000E06008682061AFF2DB10F9F766FD60707C
:1094100010BD87480021403801708448017085499B
:109420004160704770B505464FF080500C46D0F84B
:10943000A410491C05D1D0F8A810C9430904090C8F
:109440000BD050F8A01F01F0010129704168216084
:109450008068A080287830B970BD062120460CF0C5
:109460000CFD01202870607940F0C000607170BD73
:1094700070B54FF080540D46D4F88010491C0BD1C4
:10948000D4F88410491C07D1D4F88810491C03D1A2
:10949000D4F88C10491C0CD0D4F880100160D4F89A
:1094A00084104160D4F888108160D4F88C10C160B9
:1094B00002E010210CF0E1FCD4F89000401C0BD12C
:1094C000D4F89400401C07D1D4F89800401C03D174
:1094D000D4F89C00401C09D054F8900F28606068B4
:1094E0006860A068A860E068E86070BD2846BDE8D4
:1094F000704010210CF0C1BC4D480079E9E470B512
:109500004B4CE07830B3207804EB4010407A00F008
:109510000700204490F9E801002800DCFFDF2078F4
:10952000002504EB4010407A00F00700011991F883
:10953000E801401E81F8E8012078401CC0B220708C
:109540000F2800D12570A078401CA0700CF08CFB77
:10955000E57070BDFFDF70BD3EB50546032109F023
:1095600049FA0446284609F077FB054604B9FFDFAF
:10957000206918B10078FF2800D1FFDF01AA6946F1
:10958000284600F00EFB60B9FFDF0AE0002202A9C6
:10959000284600F006FB00B9FFDF9DF8080000B187
:1095A000FFDF9DF80000411E8DF80010EED220690B
:1095B0000199884201D1002020613EBD70B5054669
:1095C000A0F57F400C46FF3800D1FFDF012C01D011
:1095D000FFDF70BDFFF790FF040000D1FFDF2078B0
:1095E00020F00F00401D20F0F0005030207065800A
:1095F0000020207201202073BDE870407FE72DE934
:10960000F04116460D460746FFF776FF040000D1ED
:10961000FFDF207820F00F00401D20F0F0005030D8
:109620002070678001202072286805E01800002063
:10963000EC030020F81300202061A888A082267384
:10964000BDE8F0415BE77FB5FFF7D8FC040000D12F
:10965000FFDF02A92046FFF7FFFA054603A92046CF
:10966000FFF714FB8DF800508DF80100BDF80800DD
:10967000001DADF80200BDF80C00001DADF804009F
:10968000E088ADF80600684608F01FFA002800D010
:10969000FFDF7FBD2DE9F05FF94E8146307810B1D4
:1096A0000820BDE8F09F4846F7F733FE08B11020C8
:1096B000F7E7F44C207808B9FFF759FCA17A607AF3
:1096C0004D460844C4B200F0A2FAA04207D2201AC4
:1096D000C1B22A460020FFF76FFC0028E1D1716873
:1096E000E848C91C002721F003017160B3463E46DB
:1096F0003D46BA463C4690F801800AE0204600F01C
:109700007BFA4178807B0E4410FB0155641CE4B267
:109710007F1C4445F2D1C6EBC601DA4E0AEB870046
:1097200000EB8100F17A00EB850000EB8100DBF8B3
:1097300004105C464518012229464846FFF7C2FA44
:10974000070012D00020FFF759FC05000BD005F1EF
:109750001300616820F00300884200D0FFDF7078BA
:10976000401E7070656038469BE7002229464846D7
:10977000FFF7A8FA00B1FFDFD9F8000060604FF6EC
:10978000FF7060800120207000208AE72DE9F04101
:109790000446BB4817460E46007810B10820BDE8C5
:1097A000F0810846F7F78FFD08B11020F7E7B54DB7
:1097B000287808B9FFF7DBFB601E1E2807D8012CAC
:1097C00022D13078FE281FD828770020E7E7A4F1BF
:1097D00020001F2805D8E0B23A463146BDE8F041E6
:1097E0001EE4A4F140001F2805D831462046BDE8FC
:1097F000F04100F0D7BAA4F1A0001F2804D800203F
:10980000A02C03D0A12C06D00720C8E7317801F0A6
:1098100001016977C3E731680922F82901D38B0771
:1098200001D01046BBE76B7C03F00303012B04D18E
:109830006B8BD7339CB28C42F3D82962AFE72DE90A
:10984000F04781460E460846F7F763FD48B948469B
:10985000F7F77DFD28B909F1030020F00301494520
:1098600002D01020BDE8F08786484FF0000A403053
:10987000817869B14178804600EB4114083437881B
:1098800032460021204600F073FA050004D027E09C
:10989000A6F800A00520E5E7B9F1000F24D0308834
:1098A000B84201D90C251FE0607800F00705284672
:1098B00000F04AFA08EB0507324697F8E8014946F6
:1098C000401C87F8E801204607F5F47700F050FACD
:1098D00005463878401E3870032000F035FA2DB167
:1098E0000C2D01D0A6F800A02846BBE76078644E96
:1098F00000F00701012923D002290CD0032934D01C
:10990000FFDF98F801104046491CC9B288F80110E1
:109910000F2935D036E0616821B1000702D4608894
:10992000FFF71AFE98F8EA014746012802D170783D
:10993000F9F7F2FA97F9EA010428E2DBFFDFE0E742
:10994000616821B14FF49072B06808F0B9FE98F8E0
:10995000E9014746032802D17078F9F7DDFA97F953
:10996000E9010428CDDBFFDFCBE7C00602D5608824
:10997000FFF7F2FD98F9EB010628C2DBFFDFC0E735
:1099800080F801A08178491E8170617801F007019B
:1099900001EB080090F8E811491C80F8E811A3E7F2
:1099A00070B50D460446F7F78EFC18B92846F7F750
:1099B000B0FC08B1102070BD29462046BDE87040BB
:1099C0000AF075BD70B505460AF094FDC4B228468C
:1099D000F7F7BDFC08B1102070BD35B128782C70A8
:1099E00018B1A04201D0072070BD2046FDF764FEEB
:1099F000052805D10AF082FD012801D0002070BDA4
:109A00000F2070BD70B5044615460E460846F7F7A0
:109A10005AFC18B92846F7F77CFC08B1102070BD35
:109A2000022C03D0102C01D0092070BD2A463146EB
:109A300020460AF06CFD0028F7D0052070BD70B5F7
:109A400014460D460646F7F73EFC38B92846F7F7A8
:109A500060FC18B92046F7F77AFC08B1102070BDF9
:109A60002246294630460AF071FD0028F7D007202B
:109A700070BD3EB50446F7F74CFC28B110203EBD42
:109A800018000020AC030020684606F0C8FDFFF770
:109A900049FB0028F3D19DF806002070BDF80800AE
:109AA0006080BDF80A00A0800020E8E770B5054698
:109AB0000C460846F7F74BFC20B93CB12068F7F795
:109AC00028FC08B1102070BDA08828B12146284686
:109AD000BDE87040FDF748BE092070BD70B5054671
:109AE0000C460846F7F7EFFB30B9681E1E2814D85D
:109AF0002046F7F7E8FB08B1102070BD042D01D90E
:109B0000072070BD05B9FFDFF84800EB850050F86D
:109B1000041C2046BDE870400847A5F120001F281E
:109B200005D821462846BDE87040FAF794BBF02DD1
:109B300008D0F12DE4D1207808F05CF8BDE8704041
:109B4000FFF7F0BAA068F7F7BEFB0028D4D1204693
:109B500008F028F8F2E770B504460D460846F7F716
:109B6000D8FB30B9601E1E2811D82846F7F7ABFB8A
:109B700008B1102070BD012C05D0022C03D0032C9D
:109B800001D0042C01D1062070BD072070BDA4F1C6
:109B900020001F28F9D829462046BDE87040FAF772
:109BA000B2BB08F0A7BA38B50446D148007B00F034
:109BB0000105D9B904F034FB0DB1226800E00022A0
:109BC000CC484178C06806F018FCCA481030C0780C
:109BD0008DF8000010B1012802D004E0012000E05F
:109BE00000208DF80000684606F093FD002D02D09D
:109BF00020682830206038BD30B5BD4D04466878F7
:109C0000A04200D8FFDF686800EB041030BD70B5DB
:109C1000B74800252C46467807E02046FFF7ECFFC2
:109C20004078641C2844C5B2E4B2B442F5D1284659
:109C300070BD2DE9F0410C4607464FF0000800F0DA
:109C4000DEF80646FF2801D94FF013083868C01C1B
:109C500020F003023A6054EA080421D1A448F3B288
:109C6000072124300CF00EFB09E0072C10D2DFE8AE
:109C700004F0060408080A0406009F4804E09F4810
:109C800002E09F4800E09F480CF01CFB054600E006
:109C9000FFDFA54200D0FFDF641CE4B2072CE4D351
:109CA000386800EB06103860404678E5021D5143E5
:109CB000452900D245210844C01CB0FBF2F0C0B2D7
:109CC00070472DE9FC5F064689484FF000088B4637
:109CD0004746444690F8019022E02046FFF78CFF6B
:109CE000050000D1FFDF687869463844C7B22846CE
:109CF000FEF7B2FF824601A92846FEF7C7FF0346DA
:109D0000BDF804005246001D81B2BDF80000001DE0
:109D100080B208F0EDFE6A78641C00FB0288E4B2B1
:109D20004C45DAD13068C01C20F003003060BBF134
:109D3000000F00D000204246394608F0E7FE3168A7
:109D400008443060BDE8FC9F69494031087100203B
:109D5000C870704766494031CA782AB10A7801EB69
:109D600042110831814201D0012070470020704724
:109D70002DE9F04106460078154600F00F0400205A
:109D80001080601E0F46052800D3FFDF57482A4683
:109D9000183800EB8400394650F8043C3046BDE8E2
:109DA000F041184770B50C46402802D0412806D132
:109DB00020E0A07861780D18E178814201D9072070
:109DC00070BD2078012801D9132070BDFF2D08D85F
:109DD0000AF026FD06460BF0FFFE301A801EA84250
:109DE00001DA122070BD4248216881602179017337
:109DF000002070BDBDE87040084600F02BB82DE98A
:109E0000F047DFF8EC900026344699F8090099F8FD
:109E10000A2099F801700244D5B299F80B20104439
:109E200000F0FF0808E02046FFF7E6FE817B40785F
:109E300011FB0066641CE4B2BC42F4D199F809102D
:109E400099F80A0029442944414400B101200844FA
:109E5000304407E538B50446407800F00300012897
:109E600003D002280BD0072038BD606858B1F7F73F
:109E700077FAD0B96068F7F76AFA20B915E0606838
:109E8000F7F721FA88B969462046FCF791F80028CF
:109E9000EAD1607800F00300022808D19DF80000A4
:109EA00028B16068F7F753FA08B1102038BD61890E
:109EB000F8290DD8208988420AD8607800F003027A
:109EC0000B48012A06D1D731026A89B28A4201D2EF
:109ED000092038BD94E80E0000F1100585E80E0059
:109EE0000AB900210183002038BD00009C5A0200FD
:109EF000AC03002018000020574100001FAD0000F7
:109F0000E92F0000334201002DE9F04107461446D5
:109F10008846084601F022FD064608EB88001C2210
:109F2000796802EBC0000D18688C58B1414638467C
:109F300001F01CFD014678680078C200082305F195
:109F400020000CE0E88CA8B14146384601F015FD30
:109F50000146786808234078C20005F1240008F023
:109F600006FC38B1062121726681D0E90010C4E9EF
:109F7000031009E0287809280BD00520207266819B
:109F80006868E060002028702046BDE8F04101F0DC
:109F9000DBBC072020726681F4E72DE9F04116460C
:109FA0000D460746406801EB85011C2202EBC1010A
:109FB0004418204601F003FD40B10021708865F38C
:109FC0000F2160F31F4106200CF036FA09202070A3
:109FD000324629463846BDE8F04195E72DE9F04183
:109FE0000E46074600241C21F07816E004EB84039B
:109FF000726801EBC303D25C6AB1FFF77DFA05001A
:10A0000000D1FFDF6F802A4621463046FFF7C5FFAB
:10A010000120BDE8F081641CE4B2A042E6D8002033
:10A02000F7E770B5064600241C21C0780AE000BF9F
:10A0300004EB8403726801EBC303D5182A782AB1B4
:10A04000641CE4B2A042F3D8402070BD2821284609
:10A050001BF013FB706880892881204670BD70B5A5
:10A06000034600201C25DC780DE000BF00EB8006D5
:10A070005A6805EBC6063244167816B1128A8A422F
:10A0800004D0401CC0B28442F0D8402070BDF0B56E
:10A09000044600201C26E5780EE000BF00EB800798
:10A0A000636806EBC7073B441F788F4202D15B7899
:10A0B000934204D0401CC0B28542EFD84020F0BD8E
:10A0C0000078032801D000207047012070470078F5
:10A0D000022801D00020704701207047007807282F
:10A0E00001D000207047012070472DE9F04106465D
:10A0F00088461078F1781546884200D3FFDF2C7827
:10A100001C27641CF078E4B2A04201D8201AC4B223
:10A1100004EB8401706807EBC1010844017821B1A8
:10A120004146884708B12C7073E72878A042E8D1EF
:10A13000402028706DE770B514460B880122A240BC
:10A14000134207D113430B8001230A22011D08F09B
:10A15000D8FA047070BD2DE9FF4F81B00878DDE9B1
:10A160000E7B9A4691460E4640072CD4019808F083
:10A1700085FD040000D1FFDF07F1040820461FFA27
:10A1800088F107F0C4FE050000D1FFDF2046294614
:10A190006A4608F00EF90098A0F80370A0F805A030
:10A1A000284608F0B4F9017869F306016BF3C7118A
:10A1B000017020461FFA88F107F0ECFE00B9FFDFBE
:10A1C000019806F08CF806EB0900017F491C017725
:10A1D00005B0BDE8F08F2DE9F84F0E469A4691463E
:10A1E0000746032108F006FC0446008DDFF8B88519
:10A1F000002518B198F80000B0421ED1384608F08A
:10A200003DFD070000D1FFDF09F10401384689B2A6
:10A2100007F07DFE050010D0384629466A4608F052
:10A22000C8F8009800210A460180817006F010F9F4
:10A230000098C01DCAF8000021E098F80000B04264
:10A2400016D104F1260734F8341F012000FA06F96C
:10A2500011EA090F00D0FFDF2088012340EA09003E
:10A2600020800A22391D384608F066FA067006E09A
:10A27000324604F1340104F12600FFF75CFF0A21A5
:10A2800088F800102846BDE8F88FFEB515460C4644
:10A29000064602AB0C220621FFF79DFF002827D0BF
:10A2A0000299607812220A70801C487008224A8045
:10A2B000A07002982988052381806988C180A988B7
:10A2C0000181E988418100250C20CDE900050622A5
:10A2D00021463046FFF73FFF2946002266F31F4123
:10A2E000F02310460BF0FEFF6078801C60700120A8
:10A2F000FEBDFEB514460D460622064602AB1146CB
:10A30000FFF769FF002812D0029B1320002118706C
:10A31000A8785870022058809C800620CDE9000162
:10A320000246052329463046FFF715FF0120FEBDF2
:10A330002DE9FE430C46804644E002AB0E22072185
:10A340004046FFF748FF002841D060681C2267782C
:10A350008678BF1C06EB860102EBC1014518029806
:10A360001421017047700A214180698A0181E98ABC
:10A370004181A9888180A9898181304601F0EEFA66
:10A38000029905230722C8806F70042028700025D9
:10A390000E20CDE9000521464046FFF7DCFE2946A8
:10A3A00066F30F2168F31F41F023002206200BF013
:10A3B00099FF6078FD49801C607062682046921C9D
:10A3C000FFF793FE606880784028B6D10120BDE891
:10A3D000FE83FEB50D46064638E002AB0E2207218D
:10A3E0003046FFF7F8FE002835D068681C23C17896
:10A3F00001EB810203EBC20284180298152202705D
:10A40000627842700A224280A2894281A2888281B7
:10A41000084601F0A3FA014602988180618AC18052
:10A42000E18A0181A088B8B10020207000210E20AF
:10A43000CDE900010523072229463046FFF78BFEB0
:10A440006A68DB492846D21CFFF74FFE6868C0786F
:10A450004028C2D10120FEBD0620E6E72DE9FE43DB
:10A460000C46814644E0204601F093FAD0B302AB9B
:10A47000082207214846FFF7AEFE0028A7D06068F3
:10A480001C2265780679AD1C06EB860102EBC10142
:10A4900047180298B7F81080062101704570042112
:10A4A0004180304601F05AFA0146029805230722FE
:10A4B000C180A0F804807D70082038700025CDE9A7
:10A4C000000521464846FFF746FE294666F30F2160
:10A4D00069F31F41F023002206200BF003FF607890
:10A4E000801C60706268B3492046121DFFF7FDFDB5
:10A4F000606801794029B6D1012068E72DE9F34F62
:10A5000083B00E4680E0304601F043FA002875D053
:10A5100071681C2091F8068008EB880200EBC200ED
:10A520000C184146304601F028FA0146A078C300D5
:10A5300070684078C20004F1240008F034F907463E
:10A540008088E18B401A80B2002581B3AA46218B16
:10A55000814200D808468146024602AB0721039893
:10A56000FFF739FE010028D0BAF1000F03D0029A9C
:10A57000B888022510808B46E28B3968A9EB05006C
:10A580001FFA80FA0A440398009208F077FBED1D49
:10A59000009A59465346009507F085FFE08B5044DA
:10A5A00080B2E083B988884209D1012508E0FFE73D
:10A5B000801C4FF0010A80B2C9E7002008E60025A0
:10A5C000CDE90095238A072231460398FFF7C3FDA2
:10A5D000E089401EE0818DB1A078401CA0707068B9
:10A5E000F178427811FB02F1CAB2816901230E3081
:10A5F00008F087F880F800800020E08372686E49D8
:10A600003046921DFFF771FD7068817940297FF413
:10A610007AAF0120DCE570B5064648680D46144661
:10A620008179402910D104EB84011C2202EBC10185
:10A63000084401F0E5F9002806D0686829468471CD
:10A640003046BDE8704059E770BDFEB50C46074680
:10A65000002645E0204601F09CF9D8B360681C2232
:10A66000417901EB810102EBC1014518688900B90C
:10A67000FFDF02AB082207213846FFF7ACFD0028B8
:10A6800033D00299607816220A70801C487004202A
:10A6900048806068407901F061F90146029805231D
:10A6A000072281806989C1800820CDE90006214602
:10A6B0003846FFF750FD6078801C6070A889698972
:10A6C0000844B0F5803F00D3FFDFA88969890844BA
:10A6D000A8816E81626839492046521DFFF705FD49
:10A6E000606841794029B5D10120FEBD30B5438C69
:10A6F000458BC3F3C704002345B1838B641EED1A59
:10A70000C38A6D1E1D4495FBF3F3E4B22CB100899E
:10A7100018B1A04200D8204603444FF6FF70834290
:10A7200000D3034613800C7030BD2DE9FC41074671
:10A7300016460D46486802EB86011C2202EBC10159
:10A7400044186A4601A92046FFF7D0FFA089618915
:10A7500001448AB2BDF80010914212D0081A00D507
:10A76000002060816868407940280AD1204601F0C5
:10A770003DF9002805D06868294646713846FFF73C
:10A7800064FFBDE8FC812DE9FE4F894680461546F1
:10A790005088032108F02EF98346B8F802004028BB
:10A7A0000ED240200DE000002C000020C1A00000CF
:10A7B000CFA00000DDA0000001BA0000EDB900004C
:10A7C000403880B282460146584601F0E2F800283F
:10A7D0007ED00AEB8A001C22DBF8041002EBC000DA
:10A7E0000C18204601F0EBF8002877D1B8F80000EB
:10A7F000E18A88423CD8A189D1B348456ED1002670
:10A800005146584601F0B2F8218C0F18608B48B9B8
:10A81000B9F1020F62D3B8F804006083618A8842FC
:10A8200026D80226A9EB06001FFA80F9B888A28B69
:10A83000801A002814DD4946814500DA084683B2B3
:10A8400068886968029139680A44CDE9003208F0E5
:10A8500003FADDE90121F61D009B009607F0EFFDEC
:10A86000A18B01EB090080B2A083618B884207D9DC
:10A87000688803B052465946BDE8F04F01F0DDB894
:10A880001FD14FF009002872B8F802006881D7E99B
:10A890000001C5E90401608BA881284601F054F845
:10A8A0005146584601F062F80146DBF804000823DF
:10A8B0000078C20004F1200007F059FF0020A083B7
:10A8C0006083A0890AF0FF02401EA081688800E032
:10A8D00004E003B05946BDE8F04F26E7BDE8FE8F1F
:10A8E0002DE9F041064615460F461C461846F6F778
:10A8F000EAFC18B92068F6F70CFD08B1102013E443
:10A900007168688C0978B0EBC10F01D313200BE498
:10A910003946304601F02AF801467068082300786D
:10A92000C20005F1200007F0ECFED4E90012C0E9F6
:10A9300000120020E3E710B50446032108F05AF89E
:10A940000146007800F00300022805D02046BDE84B
:10A95000104001F1140298E48A8A2046BDE81040B4
:10A96000C7E470B50446032108F044F805460146E3
:10A970002046FFF773FD002816D029462046FFF732
:10A9800064FE002810D029462046FFF722FD00284B
:10A990000AD029462046FFF7CBFC002804D02946E0
:10A9A0002046BDE87040A9E570BD2DE9F0410C4698
:10A9B00080461EE0E178427811FB02F1CAB281695B
:10A9C00001230E3007F0D3FE077860681C22C1799E
:10A9D000491EC17107EB8701606802EBC10146188F
:10A9E0003946204600F0D5FF18B1304600F0E0FFB0
:10A9F00020B16068C1790029DCD180E7FEF77CFDD9
:10AA0000050000D1FFDF0A202872384600F0A6FFBB
:10AA100068813946204600F0B0FF0146606808238F
:10AA20004078C20006F1240007F0A1FED0E9001032
:10AA3000C5E90310A5F80280284600F085FFB0782C
:10AA400000B9FFDFB078401EB07058E770B50C4613
:10AA50000546032107F0CEFF01464068C279224433
:10AA6000C2712846BDE870409FE72DE9FE4F82463F
:10AA7000507814460F464FF0000800284FD00128A8
:10AA800007D0022822D0FFDF2068B8606068F86035
:10AA900024E702AB0E2208215046FFF79CFB00285A
:10AAA000F2D00298152105230170217841700A2106
:10AAB0004180C0F80480C0F80880A0F80C8062884B
:10AAC00082810E20CDE90008082221E0A6783046D8
:10AAD00000F044FF054606EB86012C22786802EB65
:10AAE000C1010822465A02AB11465046FFF773FBDC
:10AAF0000028C9D0029807210170217841700421F3
:10AB0000418008218580C680CDE9001805230A46CA
:10AB100039465046FFF71FFB87F80880DEE6A67827
:10AB2000022516B1022E13D0FFDF2A1D914602AB7B
:10AB300008215046FFF74FFB0028A5D002980121BD
:10AB4000022E0170217841704580868002D005E098
:10AB50000625EAE7A188C180E1880181CDE9009856
:10AB60000523082239465046D4E710B50446032190
:10AB700007F040FF014600F108022046BDE8104002
:10AB800073E72DE9F05F0C4601281DD0957992F806
:10AB90000480567905EB85011F2202EBC10121F0EB
:10ABA000030B08EB060111FB05F14FF6FF7202EAF9
:10ABB000C10909F1030115FB0611F94F21F0031A30
:10ABC00040B101283DD124E06168E57891F800802A
:10ABD0004E78DFE75946786807F047FD606000B9B6
:10ABE000FFDF594660681AF06AFDE57051467868E3
:10ABF00007F03BFD6168486100B9FFDF60684269AA
:10AC000002EB09018161606880F80080606846702D
:10AC100017E0606852464169786807F051FD5A466E
:10AC20006168786807F04CFD032007F08BFE04464E
:10AC3000032007F08FFE201A012802D1786807F060
:10AC400009FD0BEB0A00BDE8F09F0246002102203F
:10AC500097E773B5D24D0A202870009848B10024B8
:10AC60004FEA0D0007F0E3FC002C01D10099696068
:10AC70007CBD01240020F5E770B50C46154638214F
:10AC800020461AF01CFD012666700A2104F11C0002
:10AC90001AF015FD05B9FFDF297A207861F301006C
:10ACA0002070A879002817D02A4621460020FFF7F7
:10ACB00068FF6168402088706168C87061680871C9
:10ACC0006168487161688871616828880881616875
:10ACD000688848816068868170BDC878002802D085
:10ACE000002201204DE7704770B50546002165F34D
:10ACF0001F4100200BF0A0FB0321284607F07AFE3D
:10AD0000040000D1FFDF21462846FFF767F900283D
:10AD100004D0207840F010002070012070BD2DE993
:10AD2000FF4180460E460F0CFEF7E6FB050007D0FC
:10AD30006F800321384607F05DFE040008D106E06D
:10AD400004B03846BDE8F0411321F9F739BEFFDF02
:10AD50005FEA080005D0B8F1060F18D0FFDFBDE8A4
:10AD6000FF8120782A4620F0080020700020ADF8EE
:10AD7000020002208DF800004FF6FF70ADF80400CD
:10AD8000ADF8060069463846F9F711FAE7E7C6F369
:10AD9000072101EB81021C23606803EBC202805C87
:10ADA000042803D008280AD0FFDFD8E7012000904C
:10ADB0004FF440432A46204600F008FECFE704B097
:10ADC0002A462046BDE8F041FFF7E7B82DE9F05FDD
:10ADD0000027B0F80A9090460C4605463E46B9F169
:10ADE000400F01D2402001E0A9F140001FFA80FA93
:10ADF000287AC01E08286BD2DFE800F00D04192065
:10AE000058363C4772271026002C6CD0D5E9030138
:10AE1000C4E902015CE070271226002C63D00A22EC
:10AE200005F10C0104F108001AF0EDFB50E0712768
:10AE30000C26002C57D0E868A06049E07427102643
:10AE40009CB3D5E90301C4E902016888032107F036
:10AE5000D1FD8346FEF750FB02466888508051467C
:10AE60005846FFF751F833E075270A26ECB1A88958
:10AE700020812DE076271426BCB105F10C0004F1E9
:10AE8000080307C883E8070022E07727102664B18B
:10AE9000D5E90301C4E902016888032107F0AAFD8E
:10AEA00001466888FFF781FD12E01CE07327082641
:10AEB000CCB16888032107F09DFD01460078C006EB
:10AEC00006D56888FFF78AF810B96888F8F786FD14
:10AED000A8F800602CB12780A4F8069066806888E6
:10AEE000A0800020AFE6A8F80060FAE72DE9FC4159
:10AEF0000C461E4617468046032107F07BFD05469B
:10AF00000A2C0AD2DFE804F0050505050505090944
:10AF10000907042303E0062301E0FFDF0023CDE956
:10AF20000076224629464046FFF715F929E438B550
:10AF30000546A0F57F40FF3830D0284607F08CFE4C
:10AF4000040000D1FFDF204607F011FA002815D0D9
:10AF500001466A46204607F02CFA00980321B0F813
:10AF60000540284607F046FD0546052C03D0402C39
:10AF700005D2402404E0007A80B1002038BD403C76
:10AF8000A4B2214600F005FD40B1686804EB8401DD
:10AF90003E2202EBC101405A0028EFD0012038BD0B
:10AFA0002C0000202DE9F04F054689B0408807F0BD
:10AFB00053FE040000D1FFDF06AA2046696800F0B6
:10AFC000C1FC069C001F34F8031F21806388638046
:10AFD000228881B28A4205D1042B0AD0052B1DD0CC
:10AFE000062B15D02A462046FFF7CDFB09B0BDE859
:10AFF000F08F1646241D2A4621463046F7F73FFAC1
:10B000000828F3D12A4621463046FCF7F4FBEDE749
:10B010006888211D6B68FAF739FCE7E717466888EE
:10B02000032107F0E7FC4FF000088DF80480064686
:10B03000ADF80680042FD9D36279002AD6D02079C2
:10B040004FF6FF794FF01C0A13282CD008DC01289A
:10B0500078D0062847D0072875D0122874D106E08A
:10B06000142872D0152871D016286DD1ACE10C2FA0
:10B070006AD1307800F00301022965D140F0080060
:10B0800030706079B07001208DF804002089ADF82F
:10B0900008006089ADF80A00A089ADF80C00E089CD
:10B0A000ADF80E0019E0B07890429FD130780107DA
:10B0B0009CD5062F9AD120F0080030706888414650
:10B0C00060F31F4100200BF0B7F902208DF8040057
:10B0D000ADF808902089ADF80A0068882A4601A9D1
:10B0E000F9F765F882E7082F80D12789B4F80A902C
:10B0F000402F01D2402001E0A7F1400080B28046FD
:10B100000146304600F045FC08B3716808EB880042
:10B110002C2202EBC000095A4945E3D1FE4807AA98
:10B12000D0E90210CDE9071060798DF81C0008F015
:10B13000FF048DF81E4068883146FFF796FC2A46CA
:10B14000214639E0B6E014E03CE039E0E6E0F248C0
:10B15000D0E90010CDE907106079ADF820708DF8C6
:10B160001C00ADF82290688807AA3146FFF77DFCE5
:10B170003CE7082FB6D16089B4F80880402801D296
:10B18000402000E0403887B23946304600F001FCEC
:10B190000028A7D007EB870271680AEBC2000844B9
:10B1A000028A42459ED1017808299BD14078617975
:10B1B000884297D1F9B22A463046FEF7EEFE15E7EF
:10B1C0000E2F07D0CDF81C80CDF8208060798DF847
:10B1D0001C00C8E76189E7898B46B4F80C903046BB
:10B1E000FEF73DFFABF14001402901D309204AE0C1
:10B1F000B9F1170F01D3172F01D20B2043E04028DC
:10B200000ED000EB800271680AEBC200084401789E
:10B21000012903D1407861798842A9D00A2032E01F
:10B220003046FEF7FEFE014640282BD001EB81039D
:10B2300072680AEBC30002EB0008012288F80020C4
:10B24000627988F80120706822894089B84200D963
:10B250003846248A03232B72AA82EF812882A5F81C
:10B260000C906C82084600F079FB6881A8F8149075
:10B27000A8F81870A8F80E40A8F810B0284600F0FA
:10B2800063FBB3E6042005212972A5F80A80E88152
:10B2900001212973A049D1E90421CDE90721617970
:10B2A0008DF81C10ADF81E00688807AA3146FFF71C
:10B2B000DCFBE3E7062FE4D3B078904215D1307879
:10B2C000010712D520F0080030706888414660F30D
:10B2D0001F4100200BF0B0F802208DF804002089F7
:10B2E000ADF80800ADF80A90F7E604213046FEF705
:10B2F000CEFE04464028C4D00220830300902A4694
:10B300002146304600F062FB4146688864F30F2115
:10B3100060F31F4106200BF08FF867E60E2FB0D1C7
:10B3200004213046FEF7B3FE81464028A9D04146AD
:10B33000688869F30F2160F31F4106200BF07CF849
:10B34000208A0790E08900907068A7894089B842F8
:10B3500000D938468346B4F80A80208905904846CB
:10B3600000F0FCFA6881079840B10220079B00902A
:10B370002A464946304600F029FB37E6B8F1170F58
:10B380001ED3172F1CD30420287200986882EF81E7
:10B39000A5F810B0A5F80C8009EB89020AEBC200F1
:10B3A0007168009A0C180598A4F81480A4F818B0D5
:10B3B000E2812082284600F0C7FA0620207015E6B8
:10B3C00001200B230090D3E7082FA6D12189304616
:10B3D000FEF745FE074640289FD007EB87027168BD
:10B3E0000AEBC2000844804600F0E9FA002894D134
:10B3F0006489B8F80E002044B0F5803F05D3688812
:10B400003A46314600F019FBF0E5002C85D0A8F84B
:10B410000E0068883A463146FFF7FDF8082028728A
:10B42000384600F09BFA6881AC8127E770B50D467D
:10B430000646032107F0DEFA040004D02078000756
:10B4400004D5112070BD43F2020070BD2A4621468A
:10B450003046FEF71AFF18B9286860616868A06175
:10B46000207840F008002070002070BD70B50D46B7
:10B470000646032107F0BEFA040004D02078000736
:10B4800004D4082070BD43F2020070BD2A46214654
:10B490003046FEF72EFF00B9A582207820F0080084
:10B4A0002070002070BD2DE9F04F0E4691B080460F
:10B4B000032107F09FFA0446404607F0DFFB0746EA
:10B4C0000020079008900990ADF830000A90029093
:10B4D0000390049004B9FFDF0DF108091FBBFFDFE3
:10B4E00021E038460BA9002206F004FE9DF82C004E
:10B4F00000F07F050A2D00D3FFDF6019017F491E90
:10B5000001779DF82C0000060DD52A460CA907A846
:10B51000FEF711FE02E00000AC5A020019F8051017
:10B52000491C09F80510761EF6B2DAD204F134008F
:10B53000FA4D04F1260BDFF8E8A304F12A07069080
:10B5400010E05846069900F06AFA064628700A2864
:10B5500000D3FFDF5AF8261040468847E08CC05DD4
:10B56000B04202D0208D0028EBD10A202870EC4D8B
:10B570004E4628350EE00CA907A800F050FA044604
:10B58000375D55F8240000B9FFDF55F8242039460F
:10B5900040469047BDF81E000028ECD111B026E5CA
:10B5A00010B5032107F026FA040000D1FFDF0A21BD
:10B5B00004F11C001AF083F8207840F00400207099
:10B5C00010BD10B50C46032107F014FA2044007F8B
:10B5D000002800D0012010BD2DE9F84F89461546FE
:10B5E0008246032107F006FA070004D02846F5F743
:10B5F0006AFE40B903E043F20200BDE8F88F484616
:10B60000F5F787FE08B11020F7E7786828B1698858
:10B610000089814201D90920EFE7B9F800001C2414
:10B6200018B1402809D2402008E03846FEF7F9FC5E
:10B630008046402819D11320DFE7403880B2804689
:10B640000146384600F0A5F948B108EB8800796852
:10B6500004EBC000085C012803D00820CDE70520DA
:10B66000CBE7FDF749FF06000BD008EB88007968AF
:10B6700004EBC0000C18B9F8000020B1E88910B143
:10B6800013E01120B9E72888172802D36888172803
:10B6900001D20720B1E7686838B12B1D2246414628
:10B6A0003846FFF71DF90028A7D104F10C026946BE
:10B6B0002046FFF71BF8288860826888E082B9F886
:10B6C000000030B102202070E889A080E889A0B194
:10B6D0002BE003202070A889A08078688178402919
:10B6E00005D180F8028039465046FEF721FE4046DB
:10B6F00000F034F9A9F8000021E07868218B408936
:10B70000884200D908462083A6F802A0042030729F
:10B71000B9F800007081E0897082F181208B30825D
:10B72000A08AB081304600F00FF97868C1784029CE
:10B7300005D180F8038039465046FEF74AFE0020C6
:10B740005BE770B50D460646032107F053F9040088
:10B7500003D0402D04D2402503E043F2020070BD27
:10B76000403DADB2294600F014F958B105EB850112
:10B770001C22606802EBC101084400F020F918B1F6
:10B78000082070BD052070BD2A462146304600F0D5
:10B7900054F9002070BD2DE9F0410D461646804653
:10B7A000032107F027F90446402D01D2402500E08F
:10B7B000403DADB28CB1294600F0EBF880B105EB0D
:10B7C00085011C22606802EBC1014718384600F071
:10B7D000F6F838B10820BDE8F08143F20200FAE73C
:10B7E0000520F8E733463A4629462046FFF778F821
:10B7F0000028F0D1EAB221464046FEF796FF00202D
:10B80000E9E72DE9F0410D4616468046032107F091
:10B81000F1F80446402D01D2402500E0403DAFB292
:10B8200024B13046F5F74FFD38B902E043F202008B
:10B83000D1E73068F5F747FD08B11020CBE739466E
:10B84000204600F0A6F860B107EB87011C22606873
:10B8500002EBC1014518284600F0B1F818B10820E4
:10B86000B9E70520B7E7B088A98A884201D90C203A
:10B87000B1E76168E88C4978B0EBC10F01D31320C0
:10B88000A9E73946204600F078F8014660680823A9
:10B890004078C20005F1240006F033FFD6E900121B
:10B8A000C0E90012FAB221464046FEF7B4FE00207D
:10B8B00091E72DE9F0470D461F469046814603214A
:10B8C00007F098F80446402D01D2402001E0A5F190
:10B8D000400086B23CB14DB13846F5F738FD50B165
:10B8E0001020BDE8F08743F20200FAE76068C8B1B3
:10B8F000A0F80C8024E03146204600F04AF888B1D8
:10B9000006EB86011C22606802EBC101451828463F
:10B9100000F055F840B10820E3E700002C000020BB
:10B92000C45A02000520DCE7A5F80880F2B22146DF
:10B930004846FEF7FAFE1FB1A88969890844388095
:10B940000020CEE706F035BD017821F00F01491C3B
:10B9500021F0F00110310170FDF7D1BD10B50446A2
:10B96000402800D9FFDF4034A0B210BD40684269D2
:10B970000078484302EBC0007047C2784068037803
:10B9800012FB03F24378406901FB032100EBC10085
:10B990007047C2788A4209D9406801EB81011C22B4
:10B9A00002EBC101405C08B10120704700207047E4
:10B9B0000078062801D901207047002070470078E0
:10B9C000062801D00120704700207047F0B401EB39
:10B9D00081061C27446807EBC6063444049D0526EF
:10B9E0002670E3802571F0BCFEF78EBA10B5418950
:10B9F00011B1FFF7DDFF08B1002010BD012010BD1F
:10BA000010B5C18C8278B1EBC20F04D9C18911B1D4
:10BA1000FFF7CEFF08B1002010BD012010BD10B50A
:10BA20000C4601230A22011D06F0A1FE00782188A0
:10BA3000012282409143218010BDF0B402EB8205C7
:10BA40001C264C6806EBC505072363554B681C791B
:10BA5000402C03D11A71F0BCFEF700BDF0BC70475A
:10BA600010B5EFF3108000F0010472B6F948417888
:10BA7000491C41704078012801D10AF01DF9002CC1
:10BA800000D162B610BD70B5F24CA07848B901255E
:10BA9000A570FFF7E5FF0AF020F920B100200AF0B9
:10BAA000EAF8002070BD4FF08040E570C0F8045304
:10BAB000F7E770B5EFF3108000F0010572B6E54CC2
:10BAC000607800B9FFDF6078401E6070607808B968
:10BAD0000AF0F6F8002D00D162B670BDDD4810B551
:10BAE000817821B10021C1708170FFF7E2FF002051
:10BAF00010BD10B504460AF0F0F8D6498978084020
:10BB000000D001202060002010BD10B5FFF7A8FF75
:10BB10000AF0E3F802220123CE49540728B1CE48A7
:10BB2000026023610320087202E00A72C4F8043341
:10BB30000020887110BD2DE9F05FDFF8189342787E
:10BB4000817889F80420002689F80510074689F8CD
:10BB500006600078DFF804B3354620B1012811D023
:10BB6000022811D0FFDF0AF0CAF84FF0804498B1E4
:10BB70000AF0CCF8B0420FD130460AF0CBF80028DA
:10BB8000FAD041E00126EEE7FFF76AFF5846016868
:10BB9000C907FCD00226E6E70120E060C4F80451A2
:10BBA000AF490E600107D1F84412AD4AC1F34231EA
:10BBB00024321160AA49343108604FF0020AC4F8F7
:10BBC00004A3A060A7480168C94341F3001101F133
:10BBD0000108016841F01001016000E020BFD4F8C5
:10BBE00004010028FAD030460AF094F80028FAD070
:10BBF000B8F1000F04D19B48016821F010010160E9
:10BC0000C4F808A3C4F8045199F805004E4688B159
:10BC1000387878B90AF061F880460AF0F5F90146FB
:10BC20006FF00042B8F1000F02D0C6E9032101E035
:10BC3000C6E90312DBF80000C00701D00AF049F89A
:10BC4000387810B13572BDE8F09F4FF01808C4F88D
:10BC50000883C4F82C510127C4F81870D4F82C01BB
:10BC60000028FBD0C4F80C51C4F810517948C01D0D
:10BC70000AF062F83570FFF748FF6761784930795C
:10BC800020310860C4F80483DDE770B5050000D1F9
:10BC9000FFDF4FF080424FF0FF30C2F80803002171
:10BCA000C2F80011C2F80411C2F80C11C2F8101148
:10BCB000684C61700AF01DF810B10120A07060702E
:10BCC00066480068C00701D00AF003F82846BDE8BE
:10BCD000704030E75F48007A002800D001207047AC
:10BCE0002DE9FF5F6048D0F800805F4A5F49083265
:10BCF00011608406D4F8080100B10120D4F82411A1
:10BD000001B101218A46D4F81C1101B101218946F3
:10BD1000D4F8201109B1012700E00027D4F8001160
:10BD200001B101218B46D4F8041101B10121039125
:10BD3000D4F80C1101B101210291D4F8101101B114
:10BD40000121444D019129780026009120B1C4F8C9
:10BD50000861012009F08FFFBAF1000F04D0C4F888
:10BD60002461092009F087FFB9F1000F04D0C4F85D
:10BD70001C610A2009F07FFF27B1C4F820610B2065
:10BD800009F079FF3348C01D09F0DEFF00B1FFDF85
:10BD9000DFF8C4900127BBF1000F10D0C4F808737E
:10BDA000E87818B1EE70002009F065FF287A0228C3
:10BDB00005D1032028720221C9F8001027610398D9
:10BDC00008B1C4F80461029850B1C4F80C61287A33
:10BDD000032800D0FFDFC9F800602F72FFF769FE6B
:10BDE000019838B1C4F81061287A012801D100F017
:10BDF0005DF86761009838B12E70287A012801D16A
:10BE0000FFF783FEFFF755FE1248C01D09F0B2FF91
:10BE10001549091DC1F80080BDE8FF9F0D4810B508
:10BE2000C01D09F091FF0B4940B1012008704FF08F
:10BE3000E021C1F80002BDE8104011E6087A0128AF
:10BE400001D1FFF762FE0348BDE81040C01D09F0B4
:10BE500091BF00003C000020340C00400C04004066
:10BE60001805004010ED00E010050240010000013F
:10BE700070B5224CA07808B909F022FF012085078F
:10BE8000A861207A002603280AD100BFD5F80C014A
:10BE900020B9002009F03EFF0028F7D1C5F80C6159
:10BEA00026724FF0FF30C5F8080370BD70B5134C13
:10BEB0006079F0B1012803D0A179401E814218DADF
:10BEC00009F00BFF05460AF09FF86179012902D9B4
:10BED000A179491CA1710DB1216900E0E168411A05
:10BEE000022902DA11F1020F06DC0DB1206100E037
:10BEF000E060BDE8704008E670BD00003C00002036
:10BF000010B5202000F07FF8202000F08DF84D497A
:10BF1000202081F80004F5F771FA4B4908604B487E
:10BF2000D0F8041341F00101C0F80413D0F8041351
:10BF300041F08071C0F80413424901201C39C1F856
:10BF4000000110BD10B5202000F05DF83E48002132
:10BF5000C8380160001D01603D4A481E10603B4A20
:10BF6000C2F80803384B1960C2F80001C2F860013A
:10BF700038490860BDE81040202000F055B8344929
:10BF80003548091F086070473149334808607047D9
:10BF90002D48C8380160001D521E026070472C49B0
:10BFA00001200860BFF34F8F70472DE9F041284909
:10BFB000D0F8188028480860244CD4F800010025E7
:10BFC000244E6F1E28B14046F5F776F940B900219E
:10BFD00011E0D4F8600198B14046F5F76DF948B129
:10BFE000C4F80051C4F860513760BDE8F04120202A
:10BFF00000F01AB831684046BDE8F04119F08ABB3C
:10C00000FFDFBDE8F08100280DDB00F01F020121F9
:10C0100091404009800000F1E020C0F88011BFF39A
:10C020004F8FBFF36F8F7047002809DB00F01F02AE
:10C03000012191404009800000F1E020C0F8801209
:10C040007047000020E000E0C80602400000024007
:10C050001805024000040240010000010F4A126866
:10C060000D498A420CD118470C4A12680A4B9A4271
:10C0700006D101B509F09AFFFFF781FFBDE8014045
:10C08000074909680958084706480749054A064B01
:10C090007047000000000000BEBAFECA5400002035
:10C0A000040000208013002080130020F8B51D46F6
:10C0B000DDE906470E000AD006F0E0FD2346FF1D2D
:10C0C000BCB231462A46009406F0EDF9F8BDD0190D
:10C0D0002246194619F052FA2046F8BD70B50D46B1
:10C0E0000446102119F0C9FA258117206081A07B30
:10C0F00040F00A00A07370BD4FF6FF720A8001463F
:10C1000002200AF099B9704700897047827BD307F3
:10C1100001D1920703D48089088000207047052050
:10C120007047827B920700D58181704701460020CD
:10C13000098841F6FE52114200D00120704700B537
:10C140000346807BC00701D0052000BD59811846F9
:10C15000FFF7ECFFC00703D0987B40F00400987312
:10C16000987B40F001009873002000BD827B52074D
:10C1700000D509B14089704717207047827B61F371
:10C18000C302827370472DE9FC5F0E4604460178B6
:10C190009646012000FA01F14DF6FF5201EA02092C
:10C1A00062684FF6FF7B1188594502D10920BDE82E
:10C1B000FC9FB9F1000F05D041F6FE55294201D090
:10C1C0000120F4E741EA090111801D0014D0002389
:10C1D0002B7094F800C0052103221F464FF0020A7D
:10C1E000BCF10E0F76D2DFE80CF0F909252F476479
:10C1F0006B77479193B4D1D80420D8E76168208940
:10C200008B7B9B0767D517284AD30B89834247D37B
:10C210008989172901D3814242D185F800A0A5F868
:10C2200001003280616888816068817B21F00201B1
:10C230008173C6E0042028702089A5F80100608978
:10C24000A5F803003180BCE0208A3188C01D1FFAA8
:10C2500080F8414524D3062028702089A5F80100E4
:10C260006089A5F80300A089A5F805000721208AA8
:10C27000CDE90001636941E00CF0FF00082810D00F
:10C28000082028702089A5F801006089A5F803001E
:10C2900031806A1D694604F10C0008F057F910B1AD
:10C2A0005EE01020EDE730889DF8001008443080F3
:10C2B00087E00A2028702089A5F80100328044E038
:10C2C0000C2028702089A5F801006089A5F80300DA
:10C2D00031803AE082E064E02189338800EB41025A
:10C2E0001FFA82F843453BD3B8F1050F38D30E222D
:10C2F0002A700BEA4101CDE90010E36860882A4604
:10C300007146FFF7D3FEA6F800805AE0402028705F
:10C3100060893188C01C1FFA80F8414520D32878F5
:10C32000714620F03F00123028702089A5F80100E6
:10C330006089CDE9000260882A46E368FFF7B6FE0F
:10C34000A6F80080287840063BD461682089888060
:10C3500037E0A0893288401D1FFA80F8424501D29B
:10C3600004273DE0162028702089A5F80100608987
:10C37000A5F80300A089CDE9000160882A4671462E
:10C380002369FFF793FEA6F80080DEE718202870E7
:10C39000207A6870A6F800A013E061680A88920409
:10C3A00001D405271CE0C9882289914201D00627C3
:10C3B00016E01E21297030806068018821F4005148
:10C3C0000180B9F1000F0BD0618878230022022090
:10C3D00009F088FF61682078887006E033800327C1
:10C3E0006068018821EA090101803846DFE62DE90D
:10C3F000FF4F85B01746129C0D001E461CD03078AA
:10C40000C10703D000F03F00192801D9012100E045
:10C4100000212046FFF7AAFEA8420DD32088A0F5F0
:10C420007F41FF3908D03078410601D4000605D598
:10C43000082009B0BDE8F08F0720FAE700208DF84A
:10C4400000008DF8010030786B1E00F03F0C0121D8
:10C45000A81E4FF0050A4FF002094FF0030B9AB2E5
:10C46000BCF1200F75D2DFE80CF08B10745E74689D
:10C47000748C749C74B674BB74C974D574E274748F
:10C4800074F274F074EF74EE748B052D78D18DF81E
:10C490000090A0788DF804007088ADF8060030791F
:10C4A0008DF80100707800F03F000C2829D00ADCDC
:10C4B000A0F10200092863D2DFE800F012621562E1
:10C4C0001A621D622000122824D004DC0E281BD022
:10C4D0001028DBD11BE016281FD01828D6D11FE06A
:10C4E0002078800701E020784007002848DAEFE054
:10C4F00020780007F9E72078C006F6E72078800664
:10C50000F3E720784006F0E720780006EDE7208882
:10C51000C005EAE720884005E7E720880005E4E752
:10C520002088C004E1E72078800729D5032D27D192
:10C530008DF800B0B6F8010082E0217849071FD5D8
:10C54000062D1DD381B27078012803D0022817D19F
:10C5500002E0CAE0022000E0102004228DF8002052
:10C5600072788DF80420801CB1FBF0F2ADF8062043
:10C5700092B242438A4203D10397ADF80890A7E0F4
:10C580007AE02078000777D598B282088DF800A06D
:10C59000ADF80420B0EB820F6ED10297ADF8061013
:10C5A00096E02178C90667D5022D65D381B20620B1
:10C5B0008DF80000707802285ED300BFB1FBF0F266
:10C5C0008DF80400ADF8062092B242438A4253D15E
:10C5D000ADF808907BE0207880064DD5072003E079
:10C5E000207840067FD508208DF80000A088ADF89F
:10C5F0000400ADF80620ADF8081068E020780006C9
:10C6000071D50920ADF804208DF80000ADF80610B2
:10C6100002975DE02188C90565D5022D63D381B2FB
:10C620000A208DF80000707804285CD3C6E72088C3
:10C63000400558D5012D56D10B208DF80000A0885B
:10C64000ADF8040044E021E026E016E0FFE7208892
:10C65000000548D5052D46D30C208DF80000A08894
:10C66000ADF80400B6F803006D1FADF80850ADF842
:10C670000600ADF80AA02AE035E02088C00432D5D3
:10C68000012D30D10D208DF8000021E0208880049C
:10C6900029D4B6F80100E080A07B000723D5032D44
:10C6A00021D3307800F03F001B2818D00F208DF8E0
:10C6B0000000208840F40050A4F80000B6F8010003
:10C6C000ADF80400ED1EADF80650ADF808B00397C4
:10C6D00069460598F5F71EFC050008D016E00E2007
:10C6E0008DF80000EAE7072510E008250EE0307815
:10C6F00000F03F001B2809D01D2807D00220059913
:10C7000009F09AFE208800F400502080A07B4007AA
:10C7100008D52046FFF70AFDC00703D1A07B20F013
:10C720000400A073284684E61FB5022806D1012024
:10C730008DF8000088B26946F5F7ECFB1FBD0000DC
:10C74000F8B51D46DDE906470E000AD006F096FA58
:10C750002346FF1DBCB231462A46009405F0A3FED5
:10C76000F8BDD0192246194618F008FF2046F8BD3A
:10C770002DE9FF4F8DB09B46DDE91B57DDF87CA00E
:10C780000C46082B05D0E06901F002F950B11020E9
:10C79000D2E02888092140F0100028808AF8001093
:10C7A000022617E0E16901208871E2694FF4205107
:10C7B0009180E1698872E06942F601010181E069D6
:10C7C000002181732888112140F0200028808AF8F8
:10C7D0000010042638780A900A2038704FF00209B9
:10C7E00004F118004D460C9001F095FBB04681E035
:10C7F000BBF1100F0ED1022D0CD0A9EB0800801C4C
:10C8000080B20221CDE9001005AB52461E990D9869
:10C81000FFF796FFBDF816101A98814203D9F74822
:10C8200000790F9004E003D10A9808B138702FE026
:10C830004FF00201CDE900190DF1160352461E9981
:10C840000D98FFF77DFF1D980088401B801B83B269
:10C85000C6F1FF00984200D203461E990BA8D9B139
:10C860005FF00002DDF878C0CDE9032009EB060196
:10C8700089B2CDE901C10F980090BDF816100022D1
:10C880000D9801F0CBFB387070B1C0B2832807D08F
:10C89000BDF8160020833AE00AEB09018A19E1E7A6
:10C8A000022011B0BDE8F08FBDF82C00811901F015
:10C8B000FF08022D0DD09AF80120424506D1BDF89F
:10C8C0002010814207D0B8F1FF0F04D09AF8018000
:10C8D0001FE08AF80180C94800680178052902D163
:10C8E000BDF81610818009EB08001FFA80F905EBEE
:10C8F000080085B2DDE90C1005AB0F9A01F00EFBC4
:10C9000028B91D980088411B4145BFF671AF022D23
:10C9100013D0BBF1100F0CD1A9EB0800801C81B221
:10C920000220CDE9000105AB52461E990D98FFF794
:10C9300007FF1D980580002038700020B1E72DE921
:10C94000F8439C46089E13460027B26B9AB3491FD2
:10C950008CB2F18FA1F57F45FF3D05D05518AD880C
:10C960002944891D8DB200E000252919B6F83C80C4
:10C970000831414520D82A44BCF8011022F8021B96
:10C98000BCF8031022F8021B984622F8024B91468D
:10C9900006F062F94FF00C0C41464A462346CDF8AA
:10C9A00000C005F04CFDF587B16B00202944A41DA3
:10C9B0002144088003E001E0092700E0832738468E
:10C9C000BDE8F88310B50B88848F9C420CD9846B2A
:10C9D000E018048844B1848824F40044A41D23444E
:10C9E0000B801060002010BD0A2010BD2DE9F0471B
:10C9F0008AB00025904689468246ADF81850072730
:10CA00004BE0059806888088000446D4A8F80060AA
:10CA100007A8019500970295CDE903504FF40073E4
:10CA200000223146504601F0F9FA04003CD1BDF82D
:10CA30001800ADF82000059804888188B44216D10A
:10CA40000A0414D401950295039521F4004100973E
:10CA5000049541F4804342882146504601F0B4F8E1
:10CA600004000BD10598818841F40041818005AA1A
:10CA700008A94846FFF7A6FF0400DCD000970598F8
:10CA800002950195039504950188BDF81C3000229C
:10CA9000504601F099F80A2C06D105AA06A9484685
:10CAA000FFF790FF0400ACD0ADF8185004E00598F3
:10CAB000818821F40041818005AA06A94846FFF734
:10CAC00081FF0028F3D00A2C03D020460AB0BDE82D
:10CAD000F0870020FAE710B50C46896B86B051B19B
:10CAE0000C218DF80010A18FADF80810A16B0191F9
:10CAF0006946FAF718FB00204FF6FF71A063E18743
:10CB0000A08706B010BD2DE9F0410D460746896BA0
:10CB10000020069E1446002911D0012B0FD1324669
:10CB200029463846FFF762FF002808D1002C06D0BE
:10CB3000324629463846BDE8F04100F038BFBDE82E
:10CB4000F0812DE9FC411446DDE9087C0E46DDE963
:10CB50000A15521DBCF800E092B2964502D2072099
:10CB6000BDE8FC81ACF8002017222A70A5F801600E
:10CB7000A5F803300522CDE900423B462A46FFF7DF
:10CB8000DFFD0020ECE770B50C4615464821204635
:10CB900018F095FD04F1080044F81C0F00204FF632
:10CBA000FF71E06161842084A5841720E08494F8FB
:10CBB0002A0040F00A0084F82A0070BD4FF6FF7288
:10CBC0000A800146032009F037BC30B585B00C4619
:10CBD0000546FFF780FFA18E284629B101218DF877
:10CBE00000106946FAF79FFA0020E0622063606354
:10CBF00005B030BDB0F8400070470000580000207C
:10CC000090F84620920703D4408808800020F3E77C
:10CC10000620F1E790F846209207EDD5A0F84410E1
:10CC2000EAE70146002009880A0700D5012011F033
:10CC3000F00F01D040F00200CA0501D540F0040019
:10CC40008A0501D540F008004A0501D540F01000E2
:10CC50000905D1D540F02000CEE700B5034690F895
:10CC60004600C00701D0062000BDA3F842101846B8
:10CC7000FFF7D7FF10F03E0F05D093F8460040F0C5
:10CC8000040083F8460013F8460F40F001001870C6
:10CC9000002000BD90F84620520700D511B1B0F831
:10CCA0004200A9E71720A7E710F8462F61F3C30257
:10CCB0000270A1E72DE9FF4F9BB00E00DDE92B3498
:10CCC000DDE92978289D24D02878C10703D000F019
:10CCD0003F00192801D9012100E000212046FFF77B
:10CCE000D9FFB04215D32878410600F03F010CD49B
:10CCF0001E290CD0218811F47F6F0AD13A8842B1E5
:10CD0000A1F57F42FF3A04D001E0122901D10006CB
:10CD100002D504201FB0C5E5F9491D984FF0000A5F
:10CD200008718DF818A08DF83CA00FAA0A60ADF824
:10CD30001CA0ADF850A02978994601F03F02701F61
:10CD40005B1C04F1180C4FF0060E4FF0040BCDF8ED
:10CD500058C01F2A7ED2DFE802F07D7D107D267D3F
:10CD6000AC7DF47DF37DF27DF17DF47DF07D7D7D04
:10CD7000EF7DEE7D7D7D7D7DED0094F84610B5F86C
:10CD80000100890701D5032E02D08DF818B022E3E7
:10CD90004FF40061ADF85010608003218DF83C1015
:10CDA000ADF84000D8E2052EEFD1B5F801002083A0
:10CDB000ADF81C00B5F80310618308B1884201D9B1
:10CDC00001207FE10020A07220814FF6FF702084B7
:10CDD000169801F0A0F8052089F8000002200290C2
:10CDE00083460AAB1D9A16991B9801F097F890BBE1
:10CDF0009DF82E00012804D0022089F8010010209F
:10CE000003E0012089F8010002200590002203A917
:10CE10000BA807F09BFBE8BB9DF80C00059981422D
:10CE20003DD13A88801CA2EB0B01814237DB02998D
:10CE30000220CDE900010DF12A034A4641461B9824
:10CE4000FFF77EFC02980BF1020B801C80B217AA40
:10CE500003A901E0A0E228E002900BA807F076FB0E
:10CE600002999DF80C00CDE9000117AB4A464146F6
:10CE70001B98FFF765FC9DF80C100AAB0BEB01004B
:10CE80001FFA80FB02981D9A084480B202901699FE
:10CE90001B9800E003E001F041F80028B6D0BBF198
:10CEA000020F02D0A7F800B053E20A208DF8180054
:10CEB0004FE200210391072EFFF467AFB5F80100A0
:10CEC0002083ADF81C00B5F80320628300283FF4EE
:10CED00077AF90423FF674AF0120A072B5F805001D
:10CEE00020810020A073E06900F052FD78B9E1696B
:10CEF00001208871E2694FF420519180E1698872C4
:10CF0000E06942F601010181E06900218173F01FAF
:10CF100020841E98606207206084169800F0FBFF52
:10CF2000072089F800000120049002900020ADF84D
:10CF30002A0028E01DE2A3E13AE1EAE016E2AEE0D1
:10CF400086E049E00298012814D0E0698079012840
:10CF500003D1BDF82800ADF80E00049803ABCDE96D
:10CF600000B04A4641461B98FFF7EAFB0498001DB3
:10CF700080B20490BDF82A00ADF80C00ADF80E00A8
:10CF8000059880B202900AAB1D9A16991B9800F082
:10CF9000C5FF28B902983988001D05908142D1D279
:10CFA0000298012881D0E0698079012805D0BDF878
:10CFB0002810A1F57F40FF3803D1BDF82800ADF857
:10CFC0000E00049803ABCDE900B04A4641461B98D9
:10CFD000FFF7B6FB0298BBE1072E02D0152E7FF4B7
:10CFE000D4AEB5F801102183ADF81C10B5F80320BC
:10CFF000628300293FF4E4AE91423FF6E1AE0121A5
:10D00000A1724FF0000BA4F808B084F80EB0052E02
:10D0100007D0C0B2691DE26907F079FA00287FF4F1
:10D0200044AF4FF6FF70208401A906AA14A8CDF8DA
:10D0300000B081E885032878214600F03F031D9A5F
:10D040001B98FFF795FB8246208BADF81C0080E112
:10D050000120032EC3D14021ADF85010B5F80110C6
:10D060002183ADF81C100AAAB8F1000F00D00023EC
:10D07000CDE9020304921D98CDF804800090388811
:10D080000022401E83B21B9800F0C8FF8DF81800E4
:10D0900090BB0B2089F80000BDF8280037E04FF066
:10D0A000010C052E9BD18020ADF85000B5F8011081
:10D0B0002183B5F803002084ADF81C10B0F5007F83
:10D0C00003D907208DF8180085E140F47C422284C2
:10D0D0000CA8B8F1000F00D00023CDE90330CDE952
:10D0E000018C1D9800903888401E83B21B9800F078
:10D0F00095FF8DF8180028B18328A8D10220BDE043
:10D10000580000200D2189F80010BDF83000401CA7
:10D110001EE1032E04D248067FF537AE002017E14A
:10D12000B5F80110ADF81C102878400602D58DF82E
:10D130003CE002E007208DF83C004FF0000803209F
:10D14000CDE902081E9BCDF810801D980193A6F131
:10D15000030B00901FFA8BF342461B9800F034FD3E
:10D160008DF818008DF83C80297849060DD5208867
:10D17000C00506D5208BBDF81C10884201D1C4F82B
:10D18000248040468DF81880E2E0832801D14FF0DA
:10D19000020A4FF48070ADF85000BDF81C002083E7
:10D1A000A4F820B01E986062032060841321CCE0B4
:10D1B000052EFFF4EAADB5F80110ADF81C10A28FF2
:10D1C00062B3A2F57F43FE3B28D008228DF83C20B5
:10D1D0004FF0000B0523CDE9023BDDF878C0CDF818
:10D1E00010B01D9A80B2CDF804C040F40043009204
:10D1F000B5F803201B9800F0E7FC8DF83CB04FF425
:10D2000000718DF81800ADF85010832810D0F8B1D7
:10D21000A18FA1F57F40FE3807D0DCE00B228DF80E
:10D220003C204FF6FE72A287D2E7A4F83CB0D2E0D1
:10D2300000942B4631461E9A1B98FFF780FB8DF811
:10D24000180008B183284BD1BDF81C00208355E796
:10D2500000942B4631461E9A1B98FFF770FB8DF801
:10D260001800E8BBE18FA06B0844811D8DE88203A4
:10D270004388828801881B98FFF763FC824668E038
:10D2800095F80180022E70D15FEA080002D0B8F153
:10D29000010F6AD109208DF83C0007A800908DF895
:10D2A00040804346002221461B98FFF72CFC8DF856
:10D2B00042004FF0000B8DF843B050B9B8F1010FA8
:10D2C00012D0B8F1000F04D1A18FA1F57F40FF3833
:10D2D0000AD0A08F40B18DF83CB04FF4806000E0E0
:10D2E00037E0ADF850000DE00FA91B98F9F71BFFD0
:10D2F00082468DF83CB04FF48060ADF85000BAF132
:10D30000020F06D0FC480068C07928B18DF81800DB
:10D3100027E0A4F8188044E0BAF1000F03D0812080
:10D320008DF818003DE007A80090434601222146F1
:10D330001B98FFF7E8FB8DF8180021461B98FFF7B4
:10D34000CAFB9DF8180020B9192189F800100120A6
:10D3500038809DF83C0020B10FA91B98F9F7E3FE37
:10D360008246BAF1000F33D01BE018E08DF818E0C8
:10D3700031E02078000712D5012E10D10A208DF857
:10D380003C00E088ADF8400003201B9909F054F8F8
:10D390000820ADF85000C1E648067FF5F6AC4FF026
:10D3A000040A2088BDF8501008432080BDF85000C2
:10D3B00080050BD5A18FA1F57F40FE3806D11E98C0
:10D3C000E06228982063A6864FF0030A5046A1E445
:10D3D0009DF8180078B1012089F80000297889F8B3
:10D3E0000110BDF81C10A9F802109DF8181089F85A
:10D3F0000410052038802088BDF850108843208014
:10D40000E4E72DE9FF4F8846087895B00121814077
:10D410004FF20900249C0140ADF820102088DDF86F
:10D420008890A0F57F424FF0000AFF3A06D039B14C
:10D43000000705D5012019B0BDE8F08F0820FAE7F4
:10D44000239E4FF0000B0EA886F800B018995D4699
:10D450000988ADF83410A8498DF81CB0179A0A71E4
:10D460008DF838B0086098F8000001283BD00228F9
:10D4700009D003286FD1307820F03F001D30307084
:10D48000B8F80400E08098F800100320022904D1C5
:10D49000317821F03F011B31317094F846100907B3
:10D4A00059D505ABB9F1000F13D0002102AA82E8CB
:10D4B0000B000720CDE90009BDF83400B8F80410CE
:10D4C000C01E83B20022159800F0A8FD0028D1D11B
:10D4D00001E0F11CEAE7B8F80400A6F80100BDF885
:10D4E0001400C01C04E198F805108DF81C1098F881
:10D4F0000400012806D04FF4007A02282CD003281B
:10D50000B8D16CE12188B8F8080011F40061ADF8D9
:10D51000201020D017281CD3B4F84010814218D313
:10D52000B4F84410172901D3814212D1317821F087
:10D530003F01C91C3170A6F801000321ADF8341079
:10D54000A4F8440094F8460020F0020084F8460055
:10D5500065E105257EE177E1208808F1080700F400
:10D56000FE60ADF8200010F0F00F1BD010F0C00FDF
:10D5700003D03888228B9042EBD199B9B878C00794
:10D5800010D0B9680720CDE902B1CDF804B0009001
:10D59000CDF810B0FB88BA883988159800F014FBD4
:10D5A0000028D6D12398BDF82010401C80294ED0E9
:10D5B00006DC10290DD020290BD0402987D124E08A
:10D5C000B1F5807F6ED051457ED0B1F5806F97D197
:10D5D000DEE0C80601D5082000E0102082460DA933
:10D5E00007AA0520CDE902218DF83800ADF83CB03E
:10D5F000CDE9049608A93888CDE9000153460722F1
:10D6000021461598FFF7B4F8A8E09DF81C200121E9
:10D610004FF00A0A002A9BD105ABB9F1000F00D0E8
:10D620000020CDE902100720CDE90009BDF8340043
:10D630000493401E83B2218B0022159800F0EEFC6B
:10D640008DF81C000B203070BDF8140020E09DF810
:10D650001C2001214FF00C0A002A22D113ABB9F192
:10D66000000F00D00020CDE902100720CDE900090D
:10D670000493BDF83400228C401E83B2218B159890
:10D6800000F0CCFC8DF81C000D203070BDF84C0073
:10D69000401CADF8340005208DF83800208BADF823
:10D6A0003C00BCE03888218B88427FF452AF9DF863
:10D6B0001C004FF0120A00281CD1606AA8B1B8788B
:10D6C000C0073FF446AF00E018E0BA680720CDE994
:10D6D00002B2CDF804B00090CDF810B0FB88BA8843
:10D6E000159800F071FA8DF81C001320307001209D
:10D6F000ADF8340093E00000580000203988208BFA
:10D700008142D2D19DF81C004FF0160A0028A06B70
:10D7100008D0E0B34FF6FF7000215F46ADF808B0C7
:10D72000019027E068B1B978C907BED1E18F0DAB90
:10D730000844821D03968DE80C0243888288018884
:10D7400009E0B878C007BCD0BA680DAB03968DE885
:10D750000C02BB88FA881598FFF7F3F905005ED034
:10D76000072D72D076E0019005AA02A92046FFF7A6
:10D7700029F90146E28FBDF80800824201D0002954
:10D78000F1D0E08FA16B084407800198E08746E064
:10D790009DF81C004FF0180A40B1208BC8B13888A2
:10D7A000208321461598FFF796F938E004F1180018
:10D7B0000090237E012221461598FFF7A4F98DF8E9
:10D7C0001C000028EDD1192030700120ADF8340084
:10D7D000E7E7052521461598FFF77DF93AE020880F
:10D7E00000F40070ADF8200050452DD1A08FA0F5B9
:10D7F0007F41FE3901D006252CE0D8F808004FF013
:10D80000160A48B1A063B8F80C10A1874FF6FF7153
:10D81000E187A0F800B002E04FF6FF70A087BDF8E6
:10D82000200030F47F611AD078230022032015995C
:10D8300008F058FD98F8000020712088BDF82010ED
:10D84000084320800EE000E007252088BDF8201066
:10D8500088432080208810F47F6F1CD03AE0218814
:10D86000814321809DF8380020B10EA91598F9F761
:10D870005AFC05469DF81C000028EBD086F801A054
:10D8800001203070208B70809DF81C0030710520C5
:10D89000ADF83400DEE7A18EE1B118980DAB008839
:10D8A000ADF834002398CDE90304CDE90139206BAC
:10D8B0000090E36A179A1598FFF7FCF905460120D6
:10D8C0008DF838000EA91598F9F72DFC00B1054622
:10D8D000A4F834B094F8460040070AD52046FFF774
:10D8E000A0F910F03E0F04D114F8460F20F0040008
:10D8F00020701898BDF83410018028469BE500B5CB
:10D9000085B0032806D102208DF8000088B2694650
:10D91000F9F709FC05B000BD10B5384C0B7822684A
:10D92000012B02D0022B2AD111E013780BB1052B69
:10D9300001D10423137023688A889A802268CB88D7
:10D94000D38022680B891381498951810DE08B882E
:10D9500093802268CB88D38022680B8913814B89FE
:10D9600053818B899381096911612168F9F7DBFB88
:10D97000226800210228117003D0002800D08120E5
:10D9800010BD832010BD806B002800D0012070479F
:10D990008178012909D10088B0F5205F03D042F6D3
:10D9A0000101884201D10020704707207047F0B57F
:10D9B00087B0002415460E460746ADF8184011E022
:10D9C00005980088288005980194811DCDE90241C1
:10D9D000072104940091838842880188384600F02A
:10D9E000F3F830B905AA06A93046FEF7EBFF002888
:10D9F000E6D00A2800D1002007B0F0BD5800002072
:10DA000010B58B7883B102789A4205D10B885BB14F
:10DA100002E08B79091D4BB18B789A42F9D1B0F8AD
:10DA200001300C88A342F4D1002010BD812010BD2C
:10DA3000072826D012B1012A27D103E0497801F046
:10DA4000070102E04978C1F3C20105291DD2DFE8D0
:10DA500001F00318080C12000AB1032070470220DD
:10DA6000704704280DD250B10DE0052809D2801E60
:10DA7000022808D303E0062803D0032803D005209A
:10DA80007047002070470F20704781207047C0B258
:10DA900082060BD4000607D5FE48807A4143C01D9C
:10DAA00001EBD00080B270470846704700207047F5
:10DAB00070B513880B800B781C0625D5F54CA47A1D
:10DAC000844204D843F010000870002070BD9568AF
:10DAD00000F0070605EBD0052D78F54065F304133B
:10DAE0000B701378D17803F0030341EA032140F26D
:10DAF0000123B1FBF3F503FB15119268E41D00FB54
:10DB0000012000EBD40070BD906870BD37B514469D
:10DB1000BDF8041011809DF804100A061ED5C1F34B
:10DB20000013DC49A568897A814208D8FE2811D102
:10DB3000C91DC9085A42284617F097FD0AE005EBAF
:10DB4000D00100F00702012508789540A8439340D2
:10DB500018430870207820F0100020703EBD2DE999
:10DB6000F0410746C81C0E4620F00300B04202D028
:10DB70008620BDE8F081C74D002034462E60AF807E
:10DB80002881AA72E8801AE0E988491CE9808106A8
:10DB900014D4E17800F0030041EA002040F20121B2
:10DBA000B0FBF1F201FB12012068FFF770FF298939
:10DBB000084480B22881381A3044A0600C342078A0
:10DBC0004107E1D40020D4E72DE9FF4F89B0164684
:10DBD000DDE9168A0F46994623F44045084600F0D1
:10DBE0000DFB04000FD0099804F0CAFE02902078C3
:10DBF00000060AD5A748817A0298814205D8872075
:10DC00000DB0BDE8F08F0120FAE7224601A9029885
:10DC1000FFF74EFF834600208DF80C004046B8F118
:10DC2000070F1AD001222146FFF702FF0028E7D193
:10DC30002078400611D502208DF80C00ADF8107048
:10DC4000BDF80400ADF81200ADF814601898ADF8F6
:10DC50001650CDF81CA0ADF818005FEA094004D5B5
:10DC600000252E46A84601270CE02178E07801F037
:10DC7000030140EA012040F20121B0FBF1F28046AD
:10DC800001FB12875FEA494009D5B84507D1A17861
:10DC9000207901F0030140EA0120B04201D3BE42E5
:10DCA00001D90720ACE7A8191FFA80F9B94501D9B5
:10DCB0000D20A5E79DF80C0028B103A90998F9F7F4
:10DCC00030FA00289CD1B84507D1A0784FEA192135
:10DCD00061F30100A07084F804901A9800B10580E7
:10DCE000199850EA0A0027D0199830B10BEB0600BA
:10DCF0002A46199917F042FC0EE00BEB060857462E
:10DD0000189E099804F0A8FF2B46F61DB5B23946B7
:10DD10004246009504F093FB224601A90298FFF7C2
:10DD2000C7FE9DF80400224620F010008DF8040084
:10DD3000DDE90110FFF7EAFE002061E72DE9FF4F62
:10DD4000DFF8509182461746B9F80610D9F800005E
:10DD500001EB410100EB810440F20120B2FBF0F144
:10DD600085B000FB11764D46DDF84C8031460698B3
:10DD7000FFF78DFE29682A898B46611A0C31014410
:10DD80001144AB8889B28B4202D8842009B038E7AD
:10DD90000699CDB2290603D5A90601D50620F5E7D7
:10DDA000B9F806C00CF1010C1FFA8CFCA9F806C0EA
:10DDB000149909B1A1F800C0A90602D5C4F80880D9
:10DDC00007E0104480B2A9F80800191A01EB0B0013
:10DDD000A0602246FE200699FFF798FEE7702671A4
:10DDE0002078390A61F30100320AA17840F004007A
:10DDF00062F30101A17020709AF802006071BAF814
:10DE00000000E08000262673280602D599F80A70E3
:10DE100000E00127A80601D54FF000084D46002478
:10DE20004FF007090FE0CDE902680196CDF80090A8
:10DE30000496E9882046129B089AFFF7C5FE002841
:10DE4000A4D1641CE4B2BC42EDD300209EE72DE9CE
:10DE5000F047804600F0D2F9070005D0002644467E
:10DE60000C4D40F2012919E00120BDE8F087204661
:10DE700000F0C4F90278C17802F0030241EA0222FC
:10DE8000B2FBF9F309FB13210068FFF700FE3044F1
:10DE900086B201E0F8050020641CA4B2E988601E87
:10DEA0008142E4DCA8F10100E8802889801B2881F8
:10DEB00000203870D9E710B5144631B1491E2180D1
:10DEC00004F05EFDA070002010BD012010BD10B553
:10DED000D24904460088CA88904201D30A2010BD66
:10DEE000096800EB400001EB80025079A072D088F5
:10DEF00020819178107901F0030140EA0120A0818E
:10DF0000A078E11CFFF7D4FD20612088401C208010
:10DF1000E080002010BD0121018270472DE9FF4FF4
:10DF200085B04FF6FF788246A3F8008048681F4608
:10DF30000D4680788DF8060048680088ADF804002A
:10DF400000208DF80A00088A0C88A04200D30446FD
:10DF50002C8241E0288A401C2882701D6968FFF7E6
:10DF60004FFDB8BB3988414501D1601E38806888B3
:10DF7000A04236D3B178307901F0030140EA01299B
:10DF800001A9701DFFF73CFD20BB298941452CD01C
:10DF9000002231460798FFF74BFDD8B9298949453A
:10DFA00018D1E9680391B5F80AC0D6F808B0504610
:10DFB000CDF800C004F050FEDDF800C05A460CF168
:10DFC000070C1FFA8CFC4B460399CDF800C004F0F7
:10DFD00000FA50B1641CA4B2204600F00FF906000C
:10DFE000B8D1641E2C820A20D0E67C807079B8718A
:10DFF000F088B8803178F07801F0030140EA012020
:10E000007881A7F80C90504604F0BAFC324607F12C
:10E010000801FFF74DFD38610020B7E62DE9FF4FFD
:10E0200087B081461C469246DDF860B0DDF854802A
:10E03000089800F0E3F805000CD0484604F0A0FC76
:10E040002978090608D57549897A814204D887203C
:10E050000BB0D6E50120FBE7CAF309062A4601A961
:10E06000FFF726FD0746149807281CD000222946F2
:10E07000FFF7DEFC0028EBD12878400613D50120FD
:10E080008DF808000898ADF80C00BDF80400ADF854
:10E090000E00ADF81060ADF8124002A94846F9F73D
:10E0A00040F80028D4D12978E87801F0030140EA4B
:10E0B0000121AA78287902F0030240EA022056459D
:10E0C00007D0B1F5007F04D9611E814201DD0B202C
:10E0D000BEE7864201D90720BAE7801B85B2A54278
:10E0E00000D92546BBF1000F01D0ABF800501798BE
:10E0F00018B1B9192A4617F041FAB8F1000F0DD03E
:10E100003E4448464446169F04F0B8FD2146FF1D94
:10E11000BCB232462B46009404F0C5F9002097E7C4
:10E120002DE9F04107461D461646084600F066F800
:10E1300004000BD0384604F023FC2178090607D5EB
:10E140003649897A814203D8872012E5012010E5FB
:10E1500022463146FFF7ACFC65B12178E07801F04A
:10E16000030140EA0120B0F5007F01D8012000E062
:10E17000002028700020FCE42DE9F04107461D46F0
:10E180001646084600F03AF804000BD0384604F072
:10E19000F7FB2178090607D52049897A814203D8FF
:10E1A0008720E6E40120E4E422463146FFF7AEFC96
:10E1B000FF2D14D02178E07801F0030240EA02201C
:10E1C00040F20122B0FBF2F302FB130015B900F29A
:10E1D000012080B2E070000A60F30101217000208C
:10E1E000C7E410B50C4600F009F828B1C1882180B9
:10E1F0004079A070002010BD012010BD0749CA88D9
:10E20000824209D340B1096800EB40006FF00B0275
:10E2100002EB80000844704700207047F80500209A
:10E2200010B508F0EFFAF4F741FB08F051F9BDE83A
:10E23000104008F019BA302834BF01200020704780
:10E24000202834BF4FF0A0420C4A012300F01F00E9
:10E2500003FA00F0002914BFC2F80C05C2F8080543
:10E260007047202834BF4FF0A041044900F01F0040
:10E27000012202FA00F0C1F81805704700030050AF
:10E2800070B50346002002466FF02F050EE09C5C3F
:10E29000A4F130060A2E02D34FF0FF3070BD00EB20
:10E2A000800005EB4000521C2044D2B28A42EED3DB
:10E2B00070BD30B50A230BE0B0FBF3F403FB14048C
:10E2C000B0FBF3F08D183034521E05F8014CD2B279
:10E2D000002AF1D130BD30B500234FF6FF7510E0B4
:10E2E000040A44EA002084B2C85C6040C0F303140E
:10E2F000604005EA00344440E0B25B1C84EA401010
:10E300009BB29342ECD330BD2DE9F041FA4B00268D
:10E31000012793F860501C7893F864C0B8B183F873
:10E320008D40A3F88E1083F88C2083F88A70BCF19E
:10E33000000F0CBF83F8906083F89050EF4880681E
:10E34000008804F089FCBDE8F04104F01FB94FF6E5
:10E35000FF7083F88D40A3F88E0083F88C2083F83B
:10E360008A70BCF1000F14BF83F8905083F890605E
:10E37000BDE8F08170B5E14E0446306890F8981021
:10E380000025012919D090F89210012924D090F885
:10E39000681001292AD090F88A1001291CBF00209A
:10E3A00070BD657017212170D0F88C106160B0F8D5
:10E3B0009010218180F88A5016E065701C21217030
:10E3C000D0F899106160D0F89D10A16090F8A1106C
:10E3D000217380F8985007E0657007212170D0F80C
:10E3E0009410616080F89250012070BD6570142116
:10E3F000217000F16A012022201D17F0BFF80121D1
:10E400002172306880F86850BB48B0F86C20A0F8E2
:10E410009420B268537B80F8963080F89210108870
:10E4200004F01AFC04F0C1F8DEE7B448006890F884
:10E430006810002914BFB0F86C004FF6FF707047E9
:10E4400070B5AE4C06462068002808BFFFDF0025E7
:10E45000206845706660002808BFFFDF20684178AB
:10E4600000291CBFFFDF70BDA42117F028F9206828
:10E47000FF2101707F2180F836101321418428216B
:10E4800080F86510012180F8581080F85D5008F080
:10E4900082FEBDE8704008F048B8984909680978DC
:10E4A00081420CBF0120002070479448006890F81A
:10E4B0002200C0F3400070479048006890F82200A6
:10E4C00000F0010070478D48006890F82200C0F30A
:10E4D000001070472DE9F04388480024016891F846
:10E4E0002400B1F822C0C0F38002C0F340031A44F4
:10E4F00000F001000244CCF3001060B3BCF1130F34
:10E5000021D00BDCBCF1100F02BF7D4830F81200A7
:10E51000BDE8F083BCF1120F15D008E0BCF1150F77
:10E5200009D0BCF11D0F04BF7648BDE8F083FFDFC2
:10E530002046BDE8F0837449002031F8121012FB28
:10E540000010BDE8F0837149002031F8121012FB71
:10E550000010BDE8F08391F85A3091F85B002E2648
:10E560004FF47A774FF014084FF04009022B04BFA4
:10E570004AF2D745B5FBF7F510D0012B04BF4AF29C
:10E580002F75B5FBF7F510D04AF62315B5FBF7F557
:10E59000082B08BF4E4613D0042B18D02646082B54
:10E5A0000ED0042B13D0022B49D004F12806042BE3
:10E5B0000FD0082B1CBF4FF01908082304D00AE025
:10E5C0004FF0140806F5A8764FF0400303E006F577
:10E5D000A8764FF0100318FB036313FB0253C2EB42
:10E5E00002124B4D02EB820205EB82021A441CF030
:10E5F000010F4FF4C8734FF4BF7504BFCCF340064E
:10E60000002E77D0CCF3400602F5A572EEB10828B3
:10E6100004BF1E4640270CD0042804BF2E461027F6
:10E6200007D0022807BF04F11806042704F12806C2
:10E63000082707EB870808EB87173E441BE004F127
:10E6400018064FF019080423C5E7082804BF1E4622
:10E6500040270CD0042804BF2E46102707D00228DC
:10E6600007BF04F11806042704F12806082707EB62
:10E67000871706EB8706324402F19C0691F8652065
:10E6800010F00C0F08BF00223244082804BF1E46B9
:10E6900040270CD0042804BF2E46102707D002289C
:10E6A00007BF04F11806042704F128060827C7EB62
:10E6B000C70707EB470706EB4706324498321CF0C2
:10E6C000010F27D0082808BF40200CD0042804BF21
:10E6D0002B46102007D0022807BF04F1180304209E
:10E6E00004F12803082000EB400101EB001018445E
:10E6F00002444AE04DE000000406002060000020D3
:10E70000285B02008E891300305B0200205B020050
:10E71000D4FEFFFF082804BF9C4640260CD00428E6
:10E7200004BFAC46102607D0022807BF04F1180C1E
:10E73000042604F1280C082606EB8616898F0CEBBC
:10E74000860C6244EB2920D944F2552C0B3101FB95
:10E750000CF1890D082807D0042802D0022805D022
:10E7600008E02B46102008E0402006E004F11803E2
:10E77000042002E004F12803082000EB801003EBE2
:10E78000800000F5A57001FB002202F26510BDE8D3
:10E79000F08302F5A572082804BF9C4640260CD0E1
:10E7A000042804BFAC46102607D0022807BF04F196
:10E7B000180C042604F1280C082606EB8616B1F87E
:10E7C00044100CEB860C6244EB29DED944F2552C44
:10E7D0000B3101FB0CF1890D0828C5D00428C0D0ED
:10E7E0000228C7D1C2E7FE4840F271210068806A62
:10E7F00048437047FA48006890F83500002818BF71
:10E800000120704710B5F74C207B022818BF032861
:10E8100008D1207D04F115010DF0A1FC08281CBFD2
:10E82000012010BD207B002816BF022800200120F7
:10E83000BDE8104009F0C0B9EA4908737047E849DB
:10E84000096881F8300070472DE9F047E44C2168F1
:10E85000087B002816BF022800200120487301F120
:10E860000E0109F093F92168087B022816BF0328DE
:10E870000122002281F82F204FF0080081F82D009E
:10E88000487B01F10E034FF001064FF0000701280D
:10E8900004BF5B7913F0C00F0AD001F10E03012809
:10E8A00004D1587900F0C000402801D0002000E0D9
:10E8B000012081F82E00002A04BF91F8220010F0F8
:10E8C000040F07D0087D01F115010DF048FC216807
:10E8D00081F82D002068476006F0CEF92168C14D0F
:10E8E0004FF00009886095F82D000DF054FC80462B
:10E8F00095F82F00002818BFB8F1000F04D095F844
:10E900002D000DF00FFA68B195F8300000281CBFFB
:10E9100095F82E0000281DD0697B05F10E00012915
:10E920000ED012E06E734A4605F10E01404609F022
:10E9300082F995F82D1005F10E000DF023FD09E088
:10E94000407900F0C000402831D0394605F10E0072
:10E9500009F0A8F92068C77690F8220010F0040F9B
:10E9600008BFBDE8F087002795F82D000DF08EFA5E
:10E97000050008BFBDE8F08710210EF04CFA002812
:10E9800018BFBDE8F08720683A4600F11C01C67642
:10E99000284609F050F9206800F11C0160680EF06B
:10E9A00093FE6068BDE8F04701210EF0A8BE0DF0AF
:10E9B00026FD4A4605F10E0109F03DF9CAE7884AED
:10E9C0001268137B0370D2F80E000860508A8880AA
:10E9D000704778B583490446814D407B08732A68A7
:10E9E000207810706088ADF8000080B200F001015E
:10E9F000C0F3400341EA4301C0F3800341EA8301CD
:10EA0000C0F3C00341EAC301C0F3001341EA03119C
:10EA1000C0F3401341EA4311C0F3801041EA801073
:10EA20005084E07D012808BF012607D0022808BFD6
:10EA3000022603D0032814BFFFDF0826286880F8C9
:10EA40005A60607E012808BF012607D0022808BF4F
:10EA5000022603D0032814BFFFDF0826286880F8A9
:10EA60005B60217B80F82410418C1D290CBF0021A4
:10EA700061688162617D80F83510A17B002916BF35
:10EA80000229002101210175D4F80F10C0F81510DA
:10EA9000B4F81310A0F81910A17EB0F8662061F345
:10EAA0000302A0F86620E17E012918BF002180F84A
:10EAB0003410002078BD4A480068408CC0F3001133
:10EAC00031B1C0F38000002804BF1F20704702E06E
:10EAD000C0F3400109B10020704710F0010F14BFCE
:10EAE000EE20FF2070473E480068408CC0F30011C4
:10EAF00019B1C0F3800028B102E0C0F3400008B1B2
:10EB000000207047012070473549002209680A66D5
:10EB10004B8C1D2B0CBF81F8642081F8640070477A
:10EB200000232F4A126882F859309164A2F84C00F1
:10EB3000012082F859007047294A0023126882F8A0
:10EB40005830A2F854000120116582F8580070472F
:10EB50002349096881F85D0070472148006890F9F1
:10EB60005D0070471E48006890F82200C0F3401016
:10EB700070471B48006890F82200C0F3C00070473F
:10EB8000012070471648006890F85B00704770B528
:10EB900008F0EBFA08F0CAFA08F0A2F908F020FA37
:10EBA0000F4C2068016E491C016690F83300002567
:10EBB00030B108F0F0FA07F0B8FC206880F8335064
:10EBC0002068457090F8371021B1BDE870400420EE
:10EBD00009F0D7BC90F8641001B3006E814203E0E5
:10EBE000600000200406002018D8042009F0C9FCA9
:10EBF000206890F8220010F0010F07D0A06843228F
:10EC00000188BDE870400120FFF77EBBBDE8704081
:10EC100043224FF6FF710020FFF776BBBDE870403E
:10EC2000002009F0AEBC2DE9F04782B00F468146C6
:10EC3000FE4E4FF000083068458C15F0030F10D0E1
:10EC400015F0010F05F0020005D0002808BF4FF0B5
:10EC5000010806D004E0002818BF4FF0020800D1D8
:10EC6000FFDF4FF0000A544615F0010F05F00200D7
:10EC70000DD080B915F0040F0DD04AF00800002F18
:10EC80001CBF40F0010040F0020440D08FE010B102
:10EC900015F0040F0DD015F0070F10D015F0010F6F
:10ECA00005F0020036D0002808BF15F0040F27D069
:10ECB0003DE0002F18BF4AF0090478D134E02FB1AD
:10ECC0004AF0080415F0200F14D070E0316805F008
:10ECD0002002B1F84400104308BF4AF0010466D096
:10ECE0004AF0180415F0200F61D191F85A10082944
:10ECF00059D155E0316891F85A10082950D152E0A5
:10ED00004AF00800002F18BF40F001044FD140F036
:10ED100010044CE0002818BF15F0040F07D0002F96
:10ED200018BF4AF00B0442D14AF018043FE015F036
:10ED3000030F3BD115F0040F38D077B131684AF09A
:10ED4000080091F85A1008290CBF40F0020420F086
:10ED5000020415F0200F21D029E0316805F02002CF
:10ED6000B1F84400104308BF4AF003041FD04AF032
:10ED7000180015F0200F08D091F85A10082914BF78
:10ED800040F0020420F0020411E091F85A20082A11
:10ED900014BF40F0010020F00100EDE7082902D087
:10EDA00024F0010403E044F0010400E0FFDF15F06B
:10EDB000400F1BD0C7B93168B1F84400002804BF28
:10EDC000488C10F0010F0BD110F0020F08BF10F0AB
:10EDD000200F05D115F0010F08BF15F0020F03D069
:10EDE00091F85A00082801D044F040047068A0F857
:10EDF00000A0017821F02001017007210EF030FC05
:10EE0000414670680EF023FE214670680EF02BFE1E
:10EE100014F0010F0AD006230022854970680EF015
:10EE2000FCFD3068417B70680EF05CFC14F0020F52
:10EE300018D0D6E90010B9F1000F4FF006034FF0DB
:10EE4000010207D01C310EF0E8FD012170680EF0C0
:10EE500056FC07E015310EF0E0FD3068017D70686A
:10EE60000EF04DFC14F0040F18BFFFDF14F0080F74
:10EE700017D0CDF800A03068BDF800100223B0F81C
:10EE80006600020962F30B01ADF800109DF8011055
:10EE9000032260F307118DF80110694670680EF0C7
:10EEA000BCFD012F61D13068B0F84410E9B390F88F
:10EEB0002200C0F34000C0BB70680EF0C4FD401CCF
:10EEC000C7B23068B0F84420B0F85610551AC7F1F0
:10EED000FF018D42A8BF0D46AA423AD990F8220000
:10EEE00010F0010F35D144F01004214670680EF087
:10EEF000BAFDF81CC0B2ED1E284482B23068B0F8EA
:10EF00006610036E090951FA83F190F85C30494F9D
:10EF10001944BC460023E1FB07C31B096FF0240C16
:10EF200003FB0C1180F85C1000E01EE090F85B0021
:10EF3000012101F037F80090BDF800009DF80210A3
:10EF4000032340EA01400190042201A970680EF0F9
:10EF500064FD3068AAB2016C70680EF0B2FD3068D2
:10EF6000B0F856102944A0F8561014F0400F06D0FF
:10EF7000D6E90010012306225D310EF04EFD14F09B
:10EF8000200F18BFFFDF0020002818BFFFDF02B0EE
:10EF9000BDE8F0872DE9F843244C2068002808BF1D
:10EFA000FFDF2068417839BB0178FF2924D0002693
:10EFB00080F83160A0F85660867080F8376030467F
:10EFC00008F022F807F0E2FC206890F95D0007F0F5
:10EFD00082FD194807F085FD184807F0FBFF6068BF
:10EFE00008F015F8206890F8240010F0010F06D002
:10EFF000252007F07EFD09E00C20BDE8F88310F025
:10F00000020F18BF262075D007F073FD206890F816
:10F010005A10252007F078FC206880F82C6007F053
:10F02000EDFF206890F85A10002009E060000020F1
:10F030001206002053E4B36E1C5B0200195B020051
:10F0400007F04BFE0F21052007F019FD206890F80E
:10F050002E10002901BF90F82F10002990F82200EF
:10F0600010F0040F75D005F007FE0546206829460C
:10F07000806806F01AFBDFF83084074690FBF8F052
:10F0800008FB10704142284605F0F7FA21688860B5
:10F0900097FBF8F04A68104448600DF05DF80146AF
:10F0A0002068426891426FD8C0E90165FF4D4FF07A
:10F0B000010895F82D000DF06EF8814695F82F00A7
:10F0C0000127002818BFB9F1000F04D095F82D00D2
:10F0D0000CF028FEA8B195F8300000281CBF95F868
:10F0E0002E00002825D0697B05F10E00012916D0DD
:10F0F0001AE0FFE710F0040F14BF2720FFDF83D1D1
:10F1000084E73A466F7305F10E01484608F093FD17
:10F1100095F82D1005F10E000DF034F909E0407955
:10F1200000F0C000402815D0414605F10E0008F05F
:10F13000B9FD206890F8220010F0040F24D095F853
:10F140002D000CF0A3FE05001ED010210DF063FE73
:10F1500040B119E00DF053F93A4605F10E0108F0FF
:10F160006AFDE6E720683A4600F11C01C7762846AA
:10F1700008F061FD206800F11C0160680EF0A4FA3F
:10F18000012160680EF0BBFA2068417B0E3007F069
:10F190005AFC206890F8581059B3B0F85410A0F8F1
:10F1A0004410016D016490F82210C1F30011E9B917
:10F1B000B0F8660002210509ADF80050684606F077
:10F1C0003DFE28B1BDF80000C0F30B00A84204D1F9
:10F1D000BDF80000401CADF800002168BDF800003B
:10F1E000B1F8662060F30F12A1F86620206880F85D
:10F1F0005860206890F8591031B1B0F84C108187F0
:10F20000816C816380F85960B0F86610026E09095C
:10F2100051FA82F190F85C20DFF894C21144634601
:10F220000022E1FB0C3212096FF0240302FB0311F0
:10F2300080F85C100DF013F8032160680DF092F86F
:10F24000216881F833000020BDE8F883994988607F
:10F2500070472DE9F043974C83B0226892F8313023
:10F260003BB1508C1D2808BFFFDF03B0BDE8F04361
:10F270008DE401260027F1B1054692F85C0007F005
:10F2800038FC206890F85B10FF2007F03DFB2068F9
:10F290004FF4A57190F85B20002007F0E4FD206892
:10F2A00090F8221011F0030F00F02E81002D00F0D5
:10F2B000258100F029B992F822108046D07EC1F352
:10F2C0000011002956D0054660680780017821F0BA
:10F2D00020010170518C132937D01FDC102908BF81
:10F2E000022144D0122908BF062140D0FFDF6F4D14
:10F2F000606805F10E010EF0D9F9697B60680EF0C7
:10F30000F1F92068418C1D2918BF152965D0B0F886
:10F310004420016C60680EF0FEF95EE0152918BF0C
:10F320001D29E3D14FF001010EF09AF960680178D0
:10F3300041F020010170216885B11C310EF0C4F943
:10F34000012160680EF0DBF9D1E700210EF088F9A9
:10F350006068017841F020010170C8E715310EF0B6
:10F36000B3F92068017D60680EF0C9F9BFE70EF0BF
:10F3700077F9BCE70021FFF756FC6068C17811F00F
:10F380003F0F2AD0017911F0100F26D00EF066F948
:10F390002368024693F82410C1F38000C1F3400CA7
:10F3A000604401F0010100EB010C93F82C10C1F353
:10F3B0008000C1F34005284401F001010844ACEB92
:10F3C0000000C1B293F85A0000F0ECFD0090032356
:10F3D0000422694660680EF020FB2068002590F842
:10F3E000241090F82C0021EA000212F0010F18BF3F
:10F3F00001250ED111F0020F04D010F0020F08BF4A
:10F40000022506D011F0040F03D010F0040F08BF3E
:10F410000425B8F1000F2BD0012D1BD0022D08BF01
:10F4200026201BD0042D14BFFFDF272016D0206814
:10F4300090F85A10252007F067FA206890F82210FB
:10F44000C1F3001169B101224FF49671002007F059
:10F450000AFD0DE0252007F04CFBE8E707F049FB2B
:10F46000E5E790F85A204FF49671002007F0FBFC76
:10F47000206890F82C10294380F82C1090F8242054
:10F4800032EA01011DD04670418C13292CD027DCB3
:10F49000102904BF03B0BDE8F083122924D000BFB7
:10F4A000C1F30010002807E040420F0004060020CE
:10F4B00053E4B36E6000002018BFFFDF03B0BDE867
:10F4C000F083418C1D2908BF80F82C70DBD0C1F37C
:10F4D0000011002914BF80F8316080F83170D2E744
:10F4E000152918BF1D29DBD190F85A2003B04FF021
:10F4F0000101BDE8F043084607F092BE90F85B209A
:10F500000121084607F08CFE2168002DC87E7CD0C2
:10F510004A8C3D46C2F34000002808BF47F008056A
:10F5200012F0400F18BF45F04005002819BFD1F870
:10F530003890B1F83C80D1F84090B1F844806068D0
:10F54000072107800EF08CF8002160680EF07FFA2A
:10F55000294660680EF087FA15F0080F15D020686C
:10F56000BDF800100223B0F86600020962F30B0137
:10F57000ADF800109DF80110032260F307118DF81B
:10F580000110694660680EF048FA60680EF024F9D0
:10F590002168C0F1FE00B1F85620A8EB02018142BB
:10F5A000A8BF0146CFB2D019404542D245F0100164
:10F5B00060680EF058FA60680EF00EF92168C0F12C
:10F5C000FE00B1F85610A8EB01018142A8BF014628
:10F5D000CFB260680EF037FA3844421C2068B0F8A9
:10F5E0006610036E090951FA83F190F85C30FF4D03
:10F5F0001944AC460023E1FB05C31B096FF0240C42
:10F6000003FB0C1180F85C1000E038E090F85B0020
:10F61000012100F0C7FC0090BDF800009DF8021029
:10F62000032340EA01400190042201A960680EF022
:10F63000F4F9216891F8220010F0400F05D0012361
:10F6400006225D3160680EF0E8F920683A46B0F8AD
:10F65000560000EB090160680EF033FA2068B0F83C
:10F6600056103944A0F8561008F0C1F9002818BF08
:10F67000FFDF20684670867003B0BDE8F08301218B
:10F68000FFF7D1FAF0E7DA4810B50068417841B9E0
:10F690000078FF2805D000210846FFF7DAFD00209A
:10F6A00010BD07F062FD07F041FD07F019FC07F0FF
:10F6B00097FC0C2010BD10B5CD4C206890F82200AE
:10F6C00010F0010F1CBFA06801884FF03C0212BF70
:10F6D00001204FF6FF710020FEF716FE2168012081
:10F6E00081F8370010BDC249096881F832007047BF
:10F6F0002DE9F041002508F010FF002800F00581F9
:10F70000BB4C2068417801270026012906D0022938
:10F7100001D003297ED0FFDFBDE8F0818178022689
:10F720000029418C46D0C1F34002002A08BF11F0E5
:10F73000010F70D090F85B204FF001014FF00000F6
:10F7400007F06EFD216891F82200C0F34000002808
:10F7500014BF0C20222091F85B1007F0D5F8206828
:10F76000467090F8330058B106F0CBFE206890F850
:10F770005B0010F00C0F0CBF4020452007F001FD8E
:10F78000206890F83400002818BF07F019FD2168A0
:10F7900091F85B0091F8651010F00C0F08BF002184
:10F7A000962007F055FC08F019F9002818BFFFDF74
:10F7B000BDE8F081C1F3001282B110293FD090F86A
:10F7C000330020B106F09DFE402007F0DAFC2068EF
:10F7D00090F8221011F0040F36D043E090F8242066
:10F7E00090F82C309A422AD1B0F84400002808BF83
:10F7F00011F0010F05D111F0020F08BF11F0200F19
:10F800007ED04FF001014FF00000FFF722FD20688D
:10F81000418C01E040E034E011F0010F04BFC1F37E
:10F820004001002907D1B0F85610B0F844209142A9
:10F8300018BFBDE8F08180F83170BDE8F081BDE807
:10F84000F0410021012004E590F83510012914BF92
:10F850000329102545F00E0190F85A204FF00000C2
:10F8600007F0DEFC206890F83400002818BF07F08D
:10F87000A7FC0021962007F0EBFB20684670BDE84E
:10F88000F081B0F85610B0F8440081423DD0BDE898
:10F89000F04101210846DCE48178D9B1418C11F0B6
:10F8A000010F1CD080F8687090F86A20B0F86C10D6
:10F8B0000120FEF729FD2068467007F056FC07F08E
:10F8C00035FC07F00DFB07F08BFBBDE8F041032092
:10F8D00008F057BE8178BDE8F0410120B9E411F08D
:10F8E000020F04BFFFDFBDE8F081B0F85610808F33
:10F8F00081420AD001210846FFF7ABFC032000E05B
:10F9000003E021684870BDE8F081BDE8F041FFF7F1
:10F910003EB9FFF73CB910B5354C206890F834106B
:10F9200049B1363007F05BFC18B921687F2081F8B7
:10F93000360007F03BFC206890F8330018B107F060
:10F940002AFC06F0F2FD08F0E8FDA8B1206890F866
:10F950002210C1F3001179B14078022818BFFFDFEF
:10F9600000210120FFF775FC2068417800291EBFA7
:10F9700040780128FFDF10BDBDE81040FFF707B950
:10F980002DE9F0471A4C0F4680462168B8F1030F65
:10F99000488C08BFC0F3400508D000F0010591F87D
:10F9A0003200002818BF4FF0010901D14FF00009C3
:10F9B00007F093F80646B8F1030F0CBF4FF00208AA
:10F9C0004FF0010835EA090008BFBDE8F08720685C
:10F9D00090F8330090B10CF025FC38700146FF28F8
:10F9E0000CD06068C01C0CF0F6FB03E053E4B36E6F
:10F9F0006000002038780CF022FC06436068017833
:10FA0000C1F3801221680B7D9A4208D10622C01CE6
:10FA1000153115F087FD002808BF012000D0002017
:10FA20003978FF2906D0C8B9206890F82D0088429F
:10FA300016D113E0A0B1616811F8030BC0F3801078
:10FA40000CF08DFB05460CF0EDFC38B128460CF0AF
:10FA50001DFA18B110210DF0DEF908B1012000E007
:10FA60000020216891F8221011F0040F01D0F0B1AC
:10FA70001AE0CEB9FE4890F83500002818BF40457E
:10FA800015D1616811F8030BC0F380100CF067FB0F
:10FA900004460CF0C7FC38B120460CF0F7F918B159
:10FAA00010210DF0B8F910B10120BDE8F087002059
:10FAB000BDE8F0872DE9F04FEE4D074683B028688A
:10FAC00000264078022818BFFFDF28684FF07F0922
:10FAD00090F8341049B1363007F081FB002804BF9C
:10FAE000286880F8369007F061FB68680DF0DAFD51
:10FAF0000446002F00F0048268680DF05EFF0028C5
:10FB000000F0FE8106F0B7FF002800F0F981FF2029
:10FB1000DFF864B3DFF8588300274FF0010A062CA2
:10FB200080F00082DFE804F0EFEFEF03EFF78DF8ED
:10FB3000000069460320FFF723FF002800F0E4805F
:10FB4000296891F8340010B191F89800D0B1286874
:10FB5000817801294CD06868042107800DF080FD70
:10FB600008F10E0168680DF0A1FD98F80D106868A5
:10FB70000DF0B8FD2868828F816B68680DF0EFFD8D
:10FB800000F04DB99DF8000081F898A00A7881F83E
:10FB90009920FF280FD001F19B029A310CF004FB51
:10FBA000002808BFFFDF286890F89A1041F0020192
:10FBB00080F89A100DE068680278C2F3801281F82C
:10FBC0009A20D0F80320C1F89B20B0F80700A1F8D4
:10FBD0009F00286800F1A10490F836007F2808BF34
:10FBE000FFDF286890F83610217080F83690AEE775
:10FBF00090F822009BF80490C0F38014686864F3C6
:10FC00008619072107800DF02BFD002168680DF093
:10FC10001EFF494668680DF026FF0623002208F102
:10FC20000E0168680DF0F9FE2868417B68680DF0E8
:10FC300059FD68680DF0D0FD29688A8FC0F1FE017A
:10FC40008A42B8BF1146CFB2BA423DD9F81EC7B2F8
:10FC500049F0100A514668680DF005FF68680DF01C
:10FC6000F2FE3844431C2868B0F86610026E090999
:10FC700051FA82F190F85C20DFF800920A44C846FD
:10FC80004FF0000CE2FB098C4FEA1C116FF0240CC2
:10FC900001FB0C2180F85C1090F85B001A460121F2
:10FCA00000F080F90190BDF804009DF806100323D0
:10FCB00040EA01400290042202A968680DF0ADFEFE
:10FCC000514668680DF0CFFE34B1D5E9001001232C
:10FCD00006225D310DF0A1FE28683A46816B686806
:10FCE0000DF0EFFE2868A0F85670818F8F420CBF90
:10FCF0000121002180F8311007F079FE002818BF9B
:10FD0000FFDF8CE007E00DE128688078002840F0F4
:10FD1000F98000F0F5B88DF8000068680178C1F34B
:10FD20008019D0F803100191B0F80700ADF8080071
:10FD300069460520FFF724FE0028286873D08178E3
:10FD4000002972D090F85BA0D5E90104D0F80F101B
:10FD5000C4F80E10B0F813106182417D2175817DC9
:10FD60006175B0F81710E182B0F819106180B0F831
:10FD70001B10A180B0F81D10E18000F11F0104F1FB
:10FD8000080015F0B0FD686890F8241001F01F011C
:10FD9000217690F82400400984F8740184F854A076
:10FDA00084F855A0286890F8651084F8561090F8EB
:10FDB0005D0084F857009DF80010A86800F05BF91A
:10FDC000022008F0DEFB6868DBF800400DF1040A51
:10FDD000078008210DF044FC002168680DF037FE13
:10FDE000214668680DF03FFE0623002208F10E014F
:10FDF00068680DF012FE2868417B68680DF072FC9F
:10FE0000494668680DF07BFC06230122514668686C
:10FE10000DF003FE07F0EBFD002818BFFFDF032005
:10FE20002968487070E066E0FFE76868AC684FF0EA
:10FE300001080278617BC2F3401211406173D0F86F
:10FE40000F10C4F80E10B0F813106182417D2175B7
:10FE5000817D6175B0F81710E182B0F819106180EA
:10FE6000B0F81B10A180B0F81D10E18008E0000080
:10FE70000406002060000020145B020053E4B36E0F
:10FE800000F11F0104F1080015F02DFD686890F8DD
:10FE9000241001F01F01217690F82400400984F815
:10FEA000740184F8548084F85580286890F86510AF
:10FEB00084F8561090F85D0084F857009DF8001003
:10FEC000A86800F0D8F8286880F868A090F86A2040
:10FED000B0F86C100120FEF717FA2868477007F099
:10FEE00044F907F023F906F0FBFF07F079F8012049
:10FEF00008F047FB08E090F82200C0F3001008B1BA
:10FF0000012601E0FEF743FE286890F8330018B19F
:10FF100007F041F906F009FB66B100210120FFF767
:10FF200098F910E0286890F82200C0F3001000282B
:10FF3000E8D0E5E728688178012904D190F85B10C2
:10FF4000FF2006F0E1FC28684178002919BF4178BC
:10FF5000012903B0BDE8F08F4078032818BFFFDF08
:10FF600003B0BDE8F08F70B57E4C06460D462068A4
:10FF7000807858B106F07EFC21680346304691F83F
:10FF80005B202946BDE8704009F0C6B806F072FC57
:10FF900021680346304691F85A202946BDE8704052
:10FFA00009F0BAB878B50C4600210091082804BFC2
:10FFB0004FF4C87040210DD0042804BF4FF4BF7027
:10FFC000102107D0022807BF01F11800042101F118
:10FFD00028000821521D02FB010562489DF800100F
:10FFE000006890F85C2062F3050141F040068DF84E
:10FFF000006090F85B00012828D002282DD0082846
:020000040001F9
:1000000018BFFFDF2FD000BF26F080008DF8000062
:10001000C4EB041000EB80001E2101EB800005FB07
:1000200004045148844228BFFFDF5048A0FB04105D
:10003000BDF80110000960F30C01ADF80110BDF826
:1000400000009DF8021040EA014078BD9DF80200D2
:1000500020F0E0008DF80200D6E79DF8020020F0C5
:10006000E000203004E09DF8020020F0E000403085
:100070008DF80200C8E72DE9F0413A4D04460E46DE
:10008000286890F86800002818BFFFDF002728685C
:1000900080F86A702188A0F86C106188A0F882103E
:1000A000A188A0F88410E188A0F8861094F8741153
:1000B00080F8881090F82F1049B1427B00F10E01B2
:1000C000012A04D1497901F0C001402934D090F8C7
:1000D000301041B1427B00F10E01012A04BF497981
:1000E00011F0C00F28D000F1760015F0F3FB68681E
:1000F000FF2E0178C1F380116176D0F80310C4F8A7
:100100001A10B0F80700E08328681DD0C167E18BA2
:10011000A0F8801000F17002511E30460CF044F837
:10012000002808BFFFDF286890F86F1041F0020137
:1001300080F86F10BDE8F081D0F80E10C0F876108E
:10014000418AA0F87A10D2E7C767A0F88070617E74
:1001500080F86F10D4F81A100167E18BA0F87410C2
:10016000BDE8F08160000020C4BF03008988888852
:100170000178406829B190F8141190F8730038B9EB
:1001800001E001F0CDBD19B1042901D00120704773
:100190000020704770B50C460546062102F02AFC87
:1001A000606008B1002006E00721284602F022FC2A
:1001B000606018B101202070002070BD022070BD69
:1001C0002DE9FC470C4606466946FFF7E3FF002889
:1001D0007DD19DF8000050B1FEF727F9B0427CD0E8
:1001E000214630460AF088F9002873D12DE00DF041
:1001F000E7FEB04271D02146304613F027FB0028BD
:1002000068D1019D95F8D80022E0012000E000208F
:10021000804695F837004FF0010A4FF00009F0B121
:1002200095F8380080071AD584F8019084F800A06A
:1002300084F80490E68095F839102172698F618105
:10024000A98FA18185F8379044E0019D95F81401AC
:1002500058350028DBD1E87E0028D8D0D5E73046D5
:1002600002F00CFD070000D1FFDF384601F01CFF53
:1002700040B184F801900F212170E680208184F83C
:1002800004A027E0304602F0E7FC070000D1FFDFC2
:10029000B8F1000F21D0384601F05DFFB8B19DF8EC
:1002A000000038B90198D0F800014188B14201D16D
:1002B00080F80090304607F0E8FB84F801900C21AC
:1002C000217084F80490E680297F217200E004E028
:1002D00085F81B900120BDE8FC870020FBE71CB5DA
:1002E0006946FFF757FF00B1FFDF684601F024FDC4
:1002F000FB4900208968A1F8DA001CBD2DE9FC410A
:1003000004460E46062002F01DFB0546072002F0BB
:1003100019FB2844C7B20025A8463E4417E02088B0
:10032000401C80B22080B04202D34046A4F8008036
:1003300080B2B84204D3B04202D20020BDE8FC81B2
:100340006946FFF727FF0028F8D06D1CEDB2AE42DA
:10035000E5D84FF6FF7020801220EFE738B54FF652
:10036000FF70ADF800000DE00621BDF8000002F0BE
:1003700053FB04460721BDF8000002F04DFB0CB111
:1003800000B1FFDF00216846FFF7B8FF0028EBD07F
:1003900038BD70B507F0E6FB0BF0CDFCD14C4FF645
:1003A000FF7600256683A683CFA0257001680079BB
:1003B000A4F14002657042F8421FA11C1071601C3C
:1003C00013F065FB25721B2060814FF4A471A1819D
:1003D000E08121820321A1740422E274A082E082E0
:1003E000A4F13E00218305704680BD480C300570A5
:1003F000A4F110000570468070BD70B5B84C16466B
:100400000D466060217007F027FBFFF7A7FFFFF79D
:10041000C0FF207810F0CDFFB5480EF07CFA2178AF
:10042000606813F0D9FA20780AF0D4FE284608F064
:1004300010FCAF48FEF704F8217860680AF042F932
:100440003146207813F0DAFDBDE870400BF073BC44
:1004500010B501240AB1002010BD21B1012903D03B
:100460000024204610BD02210DF068FBF9E72DE9BC
:10047000F047040000D1FFDF9A4802211C3081467A
:10048000FFF73CFF00B1FFDF964D0620B5F81C805A
:1004900002F058FA0646072002F054FA3044C6B279
:1004A000701CC7B2A88BB04228D120460DF0FEFCCC
:1004B000B0B1207818283FD1207901283CD1E088BC
:1004C000062102F097FA040000D1FFDF208807F030
:1004D000DCFA2088062102F09FFA40B3FFDF2BE010
:1004E000287860B300266670142020702021201D1B
:1004F00015F0E5F8022020712E701DE0B84217D1EA
:100500002046FDF737FFD0B12078172814D1207985
:1005100068B1E088072102F06DFA40B1008807F069
:10052000B4FAE088072102F077FA00B1FFDF03E0B8
:100530002146FFF745FE10B10120BDE8F0870221FA
:100540004846FFF7DBFE10B9A98B4145AAD12046EA
:10055000BDE8F04713F098BD10B501F089FB08B174
:100560000C2010BD0BF03AFC002010BD10B5044665
:10057000007818B1012801D0122010BD01F089FBCC
:1005800020B10BF0DBFD08B10C2010BD207801F08C
:1005900036FBE21D04F11703611CBDE810400BF0AF
:1005A000C2BC10B5044601F063FB08B10C2010BDBD
:1005B000207828B1012803D0FF280BD0122010BDCD
:1005C00001F01DFB611C0BF0C9FB08B1002010BD40
:1005D000072010BD01200BF0FBFBF7E710B50BF077
:1005E000B0FD08B1002010BD302010BD10B504468C
:1005F00001F04FFB08B10C2010BD20460BF09BFD15
:10060000002010BD10B501F044FB20B10BF096FDA9
:1006100008B10C2010BD0BF0EBFC002010BDFF2139
:1006200081704FF6FF7181802D4949680A78827187
:100630008A880281498841810121417000207047E8
:100640007CB50025022A19D015DC12F10C0F15D04B
:1006500009DC12F1280F11D012F1140F0ED012F193
:10066000100F11D10AE012F1080F07D012F1040F98
:1006700004D04AB902E0D31E052B05D8012806D0C4
:10068000022808D003280AD0122528467CBD10462F
:10069000FEF75EFAF9E710460EF0E8F8F5E70846CF
:1006A00014466946FFF776FD08B10225EDE79DF88F
:1006B00000000198002580F85740E6E710B5134682
:1006C00001220CF0E5FB002010BD10B5044611F02E
:1006D00070FC05280ED0204610F05AFE002010BDF8
:1006E0006C000020E8070020FFFFFFFF1F00000054
:1006F000A80600200C20F2E710B5044601F0C9FA64
:1007000008B10C20EBE72146002007F02CFA00206E
:10071000E5E710B5044610F0C9FE50B108F02AFD17
:1007200038B1207808F0BBFA20780EF0DBFB00200F
:10073000D5E70C20D3E710B5044601F0AAFA08B1BA
:100740000C20CCE72146012007F00DFA0020C6E777
:1007500038B504464FF6FF70ADF80000A079E17996
:10076000884216D02079FDF766FD90B16079FDF7DB
:1007700062FD70B10022A079114614F0B3F840B9BF
:100780000022E079114614F0ADF810B9207A07285C
:1007900001D9122038BD08F0FAFC60B911F009FC4B
:1007A00048B900216846FFF7A9FD20B1204606F0B0
:1007B00086F8002038BD0C2038BD2DE9FC41817839
:1007C00005461A2925D00EDC16292DD2DFE801F0C6
:1007D0002C2C2C2C2C212C2C2C2C2C2C2C2C2C2C64
:1007E0002C2C2C2121212A291ED00BDCA1F11E0149
:1007F0000C2919D2DFE801F0181818181818181861
:100800001818180D3A3904290ED2DFE801F00D024C
:100810000D022888B0F5706F06D201276946FFF7F0
:10082000B9FC18B1022089E5122087E59DF8000087
:1008300001F0ECF9019C08B1FC3401E004F5BC7452
:100840009DF8000001F0E2F9019E08B1FD3601E0DB
:1008500006F279166846FFF78BFC08B1207808B1DC
:100860000C206BE52770A8783070684601F064FAB8
:10087000002063E57CB50D466946FFF78BFC00263A
:1008800018B12E602E7102207CBD9DF8000001F091
:10089000BDF9019C9DF80000583401F0B7F90198AA
:1008A00084F8406081682960017B297194F84010C8
:1008B0000029F5D100207CBD70B5044691F85500A3
:1008C00091F856300D4610F00C0F00D1002321890D
:1008D000A0880CF0A1FC696A81421DD2401A401C1C
:1008E000A1884008091A8AB2A2802189081A2081A9
:1008F000668895F8541010460CF035FC864200D2FC
:1009000030466080E68895F8551020890CF02BFC65
:10091000864200D23046E08070BDF0B585B00D460D
:10092000064603A9FFF736FC00282DD19DF80C00E0
:1009300060B300220499FB20B1F84A30FB2B00D3AE
:100940000346B1F84C40FB20FB2C00D30446DFF8F3
:100950003CCC9CE8811000900197CDF808C0ADF820
:100960000230ADF806406846FFF7A6FF6E80BDF87E
:100970000400E880BDF808006881BDF80200A88086
:10098000BDF806002881002005B0F0BD0122D1E7A6
:100990002DE9F04186B0044600886946FFF7FAFB6E
:1009A000002876D12189E08801F0D5F9002870D19E
:1009B000A188608801F0CFF900286AD12189E088F8
:1009C00001F0D7F9002864D1A188608801F0D1F93D
:1009D00007005ED1208802A9FFF79FFF00B1FFDF6B
:1009E000BDF8101062880920914252D3BDF80C1056
:1009F000E28891424DD3BDF81210BDF80E20238934
:100A00001144A2881A44914243D39DF80010019DDD
:100A10004FF00008012640F6480041B185F8A36177
:100A2000019991F8E61105F5D17541B91AE085F8FB
:100A30000D61019991F8301105F5867509B13A27D4
:100A400024E0E18869806188E9802189814200D3BE
:100A50000146A980A188814200D20846288101224E
:100A600001990FE0E18869806188E98021898142EC
:100A700000D30146A980A188814200D2084628817E
:100A8000019900222846FFF717FF2E7085F8018094
:100A9000384606B0BDE8F0817AE710B5044601F0AB
:100AA000F8F820B10BF04AFB08B10C2017E62078CB
:100AB00001F0A5F8E279611C0BF0C1FC08B100203F
:100AC0000DE602200BE610B503780446002B4068C3
:100AD00013460A46014609D05FF001000CF0A5FB61
:100AE0006168496A884203D90120F8E50020F5E7EA
:100AF0000020F4E52DE9F04117468A781E4680462D
:100B000042B11546C87838B10446690706D52AB1FE
:100B1000012104E00725F5E70724F6E70021620735
:100B200002D508B1012000E00020014206D00122D8
:100B300011464046FFF7C7FF98B93BE051B100228C
:100B400001214046FFF7BFFF58B9600732D50122A7
:100B500011461FE058B1012200214046FFF7B3FFC4
:100B600008B1092096E7680724D5012206E0680746
:100B70004FEA44700AD5002813DB002201214046C9
:100B8000FFF7A1FFB0B125F0040513E0002811DA4A
:100B9000012200214046FFF796FF58B124F00404DB
:100BA00008E0012211464046FFF78DFF10B125F005
:100BB0000405F3E73D70347000206BE710B586B094
:100BC0000446008803A9FFF7E5FA002806D1A088AB
:100BD00030B1012804D0022802D0122006B07EE5F0
:100BE0006B4602AA214603A8FFF784FF0028F5D12F
:100BF0009DF80C3000220121002B049B06D083F8C5
:100C0000AD11049B93F8FA316BBB24E083F8171104
:100C1000049B93F83C313BB9049B93F816311BB904
:100C2000049B93F87D300BB13A2010E0049B83F8CD
:100C30001611049B9DF8081083F81811049B9DF869
:100C4000001083F81911049BA188A3F81A110499C4
:100C500081F81721C2E7049B93F8AC311BB9049BC0
:100C600093F87D300BB13A2010E0049B83F8AC116F
:100C7000049B9DF8081083F8AE11049B9DF80010AA
:100C800083F8AF11049BA188A3F8B011049981F8EF
:100C9000AD21A3E710B504460020A17801B90120D9
:100CA000E2780AB940F0020001F06CF8002803D1A4
:100CB0002046BDE8104081E711E570B51C460D46A1
:100CC00018B1012801D0122070BD1946104601F05C
:100CD00069F830B12146284601F06EF808B10020CD
:100CE00070BD302070BD70B5044600780E460128F6
:100CF00004D018B1022801D0032841D1607828B16E
:100D0000012803D0022801D0032839D1E07B10B993
:100D1000A078012834D1A07830F0050130D110F04E
:100D2000050F2DD06289E188E0783346FFF7C5FFD3
:100D3000002826D1A07805281ED16589A28921899D
:100D400020793346FFF7B9FF00281AD15FF0010080
:100D500004EB40014A8915442218D37892789342D3
:100D60000ED1CA8889888A420AD1401CC0B20228A2
:100D7000EED3E088A84203D3A07B08B1072801D9AD
:100D8000122070BD002070BD10B586B0044600F082
:100D900062FF08B10C2021E7022104F10A0001F0F2
:100DA0001EF8A0788DF80800A0788DF80000607813
:100DB0008DF8040020788DF80300A07B8DF80500E5
:100DC000E07B00B101208DF80600A078C10717D0A4
:100DD000E07800F0FBFF8DF80100E088ADF80A0034
:100DE0006089ADF80C00A078400716D5207900F096
:100DF000EDFF8DF802002089ADF80E00A0890AE011
:100E000040070AD5E07800F0E1FF8DF80200E088A5
:100E1000ADF80E006089ADF8100002A810F052FB8A
:100E20000028B8D168460EF062F8D7E610B504463F
:100E30000121FFF758FF002803D12046BDE81040EC
:100E4000A2E74CE40278012A01D0BAB118E0427856
:100E50003AB1012A05D0022A12D189B1818879B12B
:100E600000E059B1418849B1808838B101EB810176
:100E7000490000EB8000B1EB002F01D20020704749
:100E80001220704770B5044600780D46012809D03D
:100E900011F08FF8052803D010F025FA002800D0B3
:100EA0000C2070BD0DF0F0FE88B10DF002FF0DF0CA
:100EB000FBFF0028F5D125B160780DF08CFF0028EC
:100EC000EFD1A1886088BDE8704010F021BB1220EE
:100ED00070BD10B504460121FFF7B4FF002804D10E
:100EE0002046BDE810400121CCE704E42DE9F0479D
:100EF0000746B0F84C50FB2092460E46FB2D00D31F
:100F00000546DFF88C86B8F80A00A84200D20546EC
:100F100097F85510284600F08DFEB8F80C10814265
:100F200000D208468146B7F84A40FB20FB2C00D38C
:100F30000446B8F80E00A04200D2044697F85410B8
:100F4000204600F077FEB8F81010814200D2084623
:100F50004FF4A4721B2C01D0904203D11B2D25D03D
:100F6000914523D0F580A6F808907480B080524651
:100F700039463046FFF7A0FC01203070F0881B385E
:100F8000E02800D9FFDF70881B38E02800D9FFDF98
:100F9000308940F64814A0F5A470A04200D9FFDFC4
:100FA000B088A0F5A470A04200D9FFDFBDE8F087AB
:100FB000F0B5871FDDE9056540F67B44A74213D2F3
:100FC0008F1FA74210D288420ED8B2F5FA7F0BD2FB
:100FD000A3F10A00241FA04206D2521C4A43B2EBDE
:100FE000830F01DAAE4201D90020F0BD0120F0BD2F
:100FF0002DE9FC47477A8946044617F0050F7DD056
:10100000F8087BD194F83A0008B9012F76D1002571
:10101000A8462E46F90789F0010A19D0208A5146C0
:1010200000F0C0FEF0B36089514600F0C5FEC8B3C1
:10103000208A6189884261D8A18EE08DCDE90001C6
:10104000238D628CA18BE08AFFF7B2FF50B301259C
:10105000B8070ED504EB4500828EC18DCDE9001294
:10106000038D428C818BC08AFFF7A2FFD0B1A846C6
:101070006D1C78071ED504EB45065146308A00F0FA
:1010800091FE78B17089514600F096FE50B1308AD9
:10109000718988425ED8B18EF08DCDE90001338D23
:1010A000728C00E00AE0B18BF08AFFF781FF28B173
:1010B0002E466D1CB9F1000F03D030E03020BDE8A2
:1010C000FC87F80707D0780705D504EB460160894F
:1010D000498988423ED1228A01211BE0414503D043
:1010E00004EB4100008A024404EB4100C38A868A73
:1010F000B3422FD1838B468BB34200E02AE029D143
:10110000438C068CB34225D1038DC08C834221D100
:10111000491CC9B2A942E1D3608990421AD3207810
:1011200010B1012816D10DE0A078B9F1000F07D059
:1011300040B1012806D0022804D003280AD101E0DA
:101140000028EED1607838B1012805D0022803D0FC
:10115000032801D01220B2E70020B0E7002147E7C2
:101160000178C90702D0406812F061BF12F02EBFAB
:101170002DE9F04788B00D46AFF69422D2E90092EF
:10118000014690462846FFF733FF06000CD100F0D9
:1011900062FD40B9FE4F387828B90CF011FFA0F578
:1011A0007F41FF3902D00C2008B0FFE6032105F192
:1011B000100000F014FEF64801AA3E380190F548F0
:1011C0000290F34806211038039007A801F0E0FBD5
:1011D000040035D003210BF0BBFBB98AA4F84A10F8
:1011E000FA8AA4F84C20FB7C0093BA46BB7C20888A
:1011F00001F0BBFC00B1FFDF208806F045FC218830
:1012000004F10E0000F04FFDE3A004F112070068A6
:1012100000900321684604F007FE002069460A5C3E
:101220003A54401CC0B20328F9D3A88B6080688C64
:10123000A080288DE080687A410703D508270AE05E
:101240000920B1E7C10701D0012704E0800701D5DB
:10125000022700E000273A46BAF81800114610F0BD
:10126000EBF90146A062204610F0F4F917F00C0FDC
:1012700009D001231A46214600200BF0D6FF616AEF
:10128000884200D90926002784F85E7084F85F70D0
:10129000A87800F0B4FC6076D5F80300C4F81A0012
:1012A000B5F80700E083C4F8089084F80C800120AA
:1012B00084F80801024604F586712046FFF716FE01
:1012C0008DF800700121684604F0AEFD9DF8000025
:1012D00000F00701C0F3C1021144C0F340100844FC
:1012E0008DF80000401D2076092801D208302076B4
:1012F000002120460BF02CFB68780DF0D0FCEEBBF3
:10130000A9782878EA1C0DF092FC48B10DF0D1FCC8
:10131000A9782878EA1C0DF038FD060002D052E0CA
:10132000122650E0687A00F005010020CA0700D0BC
:1013300001208A0701D540F00200490701D540F09D
:1013400008000DF05DFC06003DD1214603200DF0A4
:1013500046FD060037D10DF04CFD060033D1697A09
:1013600001F005018DF81010697AC90708D0688965
:10137000ADF81200288AADF8140000E023E0012047
:10138000697A8A0700D5401C490707D505EB40005C
:101390004189ADF81610008AADF8180004A810F0C5
:1013A00091F8064695F83A0000B101200DF03AFC9C
:1013B0004EB90DF079FD060005D1A98F204610F039
:1013C00023F8060008D0208806F05FFB208806215D
:1013D00001F022FB00B1FFDF3046E5E601460020C8
:1013E000C6E638B56A48007878B910F0E2FD0528FD
:1013F00005D00CF0E5FDA0F57F41FF3905D068462A
:1014000010F0C9F8040002D00CE00C2038BD0098A0
:10141000008806F03AFB00980621008801F0FCFAEB
:1014200000B1FFDF204638BD1CB582894189CDE976
:1014300000120389C28881884088FFF7B9FD08B18E
:1014400000201CBD30201CBD70B50546FFF7ECFF29
:1014500000280ED12888062101F0CCFA040007D01C
:1014600000F05EFC20B1D4F80001017831B901E050
:10147000022070BDD4F84C11097809B13A2070BD32
:1014800005218171D4F8001100200881D4F80011E1
:10149000A8884881D4F80011E8888881D4F8001120
:1014A0002889C881D4F80001028941898A4204D878
:1014B0008279082A01D88A4201D3122070BD298876
:1014C0004180D4F8001102200870002070BD3EB5A4
:1014D00004460BF06FFCB0B12D480125A0F140028D
:1014E0004570236842F8423F23790021137141700F
:1014F0006946062001F007FA00B1FFDF684601F0F7
:10150000E0F910B10EE012203EBDBDF80440029893
:1015100080F80851684601F0D4F918B9BDF8040004
:10152000A042F4D100203EBD70B5054600880621DA
:1015300001F060FA040007D000F0F2FB20B1D4F80B
:101540000011087830B901E0022070BDD4F84C01D8
:10155000007808B13A2070BD9620005D10F0010FB0
:1015600024D0D5F802004860D5F806008860D4F889
:101570000001698910228181D4F8000105F10C0174
:101580000E3004F5807413F0F9FF07E0385B0200B9
:10159000E807002078000020112233002168032092
:1015A0000870216828884880002070BD0C2070BD1C
:1015B00038B504460078EF284DD86088ADF80000B3
:1015C000009800F01DFC88B36188080708D4D4E9AE
:1015D000012082423FD8202A3DD3B0F5804F3AD82F
:1015E000207B18B3072836D8607B28B1012803D0A8
:1015F000022801D003282ED14A0703D4022801D0A3
:10160000032805D1A07B08B1012824D1480707D4BD
:10161000607D28B1012803D0022801D003281AD107
:10162000C806E07D03D5012815D110E013E001289C
:1016300001D003280FD1C80609D4607E012803D049
:10164000022801D0032806D1A07E0F2803D8E07E0F
:1016500018B1012801D0122038BD002038BDF8B5DE
:1016600014460D46064607F092FD08B10C20F8BD61
:101670003046FFF79DFF0028F9D1FDF76EFA28707C
:10168000B07554B9FF208DF8000069460020FDF7C1
:1016900053FA69460020FDF743FA3046BDE8F840AA
:1016A000FDF797B90022DAE770B50C46054612B18E
:1016B0001F2907D80CE0FF2C04D8FCF704FF18B151
:1016C0001F2C01D9122070BD2846FCF7E6FE08B198
:1016D000002070BD422070BD10B50446408810B196
:1016E000FDF701FA78B12078618800F00102607896
:1016F000FFF7DAFF002805D1FDF7DDF962888242A5
:1017000003D9072010BD122010BD10466168FDF7F7
:1017100013FA002010BD10B50446408810B1FCF744
:10172000C4FE70B12078618800F001026078FFF794
:10173000BBFF002804D160886168FDF7F1F9002043
:1017400010BD122010BD7CB504464078422501280A
:1017500008D8A078FCF7A1FE20B120781225012836
:1017600002D090B128467CBDFDF703FA20B1A088D5
:101770000028F7D08028F5D8FDF702FA60B160782C
:101780000028EFD02078012808D006F09DFA044602
:1017900007F0BCF900287DD00C207CBDFDF732F8A5
:1017A00010B9FDF7DFF990B307F0F1FC0028F3D191
:1017B000FCF73BFEA0F57F41FF39EDD1FDF744F882
:1017C000A68842F210704643A079FDF79DF9FCF718
:1017D00073FEF8B10022072101A801F0D9F8040036
:1017E00043D0FA480321846020460AF0B6FF204621
:1017F000FDF72CFDF64DA88AA4F84A00E88AA4F863
:101800004C00FCF760FE60B1288B01210DE0FFE782
:1018100012207CBD3146002007F044FAD8B3FFDF28
:101820004CE0FDF7AFF90146288B07F0F0FA0146CE
:10183000A0620022204606F04AFAFCF744FEB0B946
:10184000FDF7A0F910F00C0F11D001231A46214624
:1018500018460BF0EAFC616A884208D90721BDF8F6
:10186000040001F0D9F800B1FFDF09207CBDE87C5D
:101870000090AB7CEA8AA98A208801F076F900B151
:10188000FFDF208806F000F93146204607F00AFA0B
:1018900018B101E008E011E0FFDF002204F5D1718A
:1018A0002046FFF723FB09E044B1208806F0EDF85D
:1018B0002088072101F0B0F800B1FFDF00207CBDD7
:1018C000002140E770B50D46072101F093F80400B0
:1018D00003D094F87B0110B10AE0022070BD94F8A7
:1018E0006500142801D0152802D194F8C80108B168
:1018F0000C2070BD1022294604F5BE7013F03EFE88
:10190000012084F87B01002070BD10B5072101F093
:1019100071F818B190F87B1111B107E0022010BDE9
:1019200090F86510142903D0152901D00C2010BDA2
:10193000022180F87B11002010BD2DE9FC410C46EE
:101940004BF68032122194421DD8E4B16946FEF76D
:1019500021FC002815D19DF8000000F057F9019EE8
:101960009DF80000583600F051F9019DAD1C2F88FC
:101970002246394630460AF0E6FE2888B842F6D1BB
:101980000020BDE8FC810846FBE77CB504460088E2
:101990006946FEF7FFFB002810D19DF8000000F01B
:1019A00035F9019D9DF80000583500F02FF9019898
:1019B000A27890F82C10914201D10C207CBD7F219F
:1019C0002972A9720021E972E17880F82D1021793D
:1019D00080F82E10A17880F82C1000207CBD1CB55A
:1019E0000C466946FEF7D6FB00280AD19DF8000098
:1019F00000F00CF9019890F8730000B101202070FC
:101A000000201CBD7CB50D4614466946FEF7C2FB9E
:101A1000002809D19DF8000000F0F8F8019890F82E
:101A20002C00012801D00C207CBD9DF8000000F0A6
:101A3000EDF8019890F86010297090F8610020701E
:101A400000207CBD70B50D461646072100F0D2FF80
:101A500018B381880124C388428804EB4104AC4256
:101A600017D842F210746343A4106243B3FBF2F23E
:101A7000521E94B24FF4FA72944200D91446A54211
:101A800000D22C46491C641CB4FBF1F24A43521E9E
:101A900091B290F8B4211AB901E0022070BD01841E
:101AA0003180002070BD10B50C46072100F0A2FF68
:101AB00048B180F8E74024B190F8E51009B107F08B
:101AC000BCF9002010BD022010BD017899B1417809
:101AD00089B141881B290ED381881B290BD3C1886A
:101AE000022908D33A490268403941F8522F406828
:101AF0004860002070471220704710B504460FF070
:101B000097FD204607F052F9002010BD10B507F0F0
:101B100050F9002010BD2DE9F04115460F4606464C
:101B20000122114638460FF087FD04460121384650
:101B300007F06DF9844200D2044601213046653C2D
:101B400000F069F806460121002000F064F83044F6
:101B500001219630844206D900F19601201AB0FB8B
:101B6000F1F0401C81B229800020BDE8F08110B561
:101B7000044600F08EF808B10C2010BD601C0AF07D
:101B800039FC207800F00100FCF759FE207800F0C5
:101B900001000DF089F8002010BD10B507F003F921
:101BA000002010BD10B50446072000F0BDFE08B1AE
:101BB0000C2010BD2078C00716D000226078114696
:101BC00012F090FE30B1122010BD00006C00002019
:101BD000E8070020A06809F0D4F86078D4F8041071
:101BE00009F0D8F80020EFE7002009F0CAF800213A
:101BF0000846F5E710B505F02BFB0020E4E718B127
:101C0000022801D0012070470020704708B1002051
:101C100070470120704710B5012904D0022905D072
:101C2000FFDF2046D0E7C000503001E080002C30BC
:101C300084B2F6E711F00C0F04D04FF4747101EB8D
:101C4000801006E0022902D0C000703001E0800060
:101C50003C3080B2704710B510F0ABF9042805D0C5
:101C600010F0A7F9052801D00020ADE70120ABE76F
:101C700010B5FFF7F0FF10B10DF0DAF828B907F052
:101C800086FA20B1FCF7B6FD08B101209CE70020E0
:101C90009AE710B5FFF7DFFF18B907F078FA0028C8
:101CA00092D0012090E72DE9FE4300250F468046A3
:101CB0000A260421404604F0E0F840460BF01BF8E9
:101CC000062000F03FFE044615E06946062000F0BD
:101CD0001AFE0AE0BDF80400B84206D002980422B9
:101CE00041460E3013F01EFC50B1684600F0E9FD8D
:101CF0000500EFD0641E002C06DD002DE5D005E0C8
:101D000040460BF001F8F5E705B9FFDFD8F8000011
:101D10000BF015F8761E01D00028CAD0BDE8FE836E
:101D200090F8D81090F8730020B919B1042901D0A7
:101D30000120704700207047017800290AD04168CF
:101D400091F8E520002A05D0002281F8E5204068BE
:101D500007F073B870471B38E12806D2B1F5A47FAD
:101D600003D344F29020814201D912207047002011
:101D70007047FB2802D8B1F5296F01D911207047AF
:101D80000020704770B514460546012200F05CF84B
:101D9000002806D121462846BDE87040002200F008
:101DA00053B870BD042803D321B9B0F5804F01D9D1
:101DB0000020704701207047042803D321B9B0F5F3
:101DC000804F01D90020704701207047012802D0C0
:101DD00018B100207047022070470120704710B5ED
:101DE00000224FF4C84408E030F81230A34200D972
:101DF000234620F81230521CD2B28A42F4D3E3E6D2
:101E000080B2C1060BD401071CD481064FEAC07111
:101E100001D5B9B900E099B1800713D410E04106AB
:101E200010D481060ED4C1074FEA807104D0002976
:101E300002DB400704D405E0010703D4400701D4C6
:101E400001207047002070470AB1012200E0022201
:101E5000024202D1C80802D109B100207047112006
:101E60007047000030B5058825F4004421448CB249
:101E70004FF4004194420AD2121B92B21B339A4291
:101E800001D2A94307E005F40041214303E0A21A6F
:101E900092B2A9431143018030BD08440830504339
:101EA0004A31084480B2704770B51D4616460B464D
:101EB000044629463046049AFFF7EFFF0646B34230
:101EC00000D2FFDF2821204613F0F9FB4FF6FF7008
:101ED000A082283EB0B265776080B0F5004F00D98F
:101EE000FFDF618805F13C00814200D2FFDF60889E
:101EF0000835401B343880B220801B2800D21B20BC
:101F000020800020A07770BD8161886170472DE935
:101F1000F05F0D46C188044600F12809008921F4CC
:101F2000004620F4004800F062FB10B10020BDE83C
:101F3000F09F4FF0000A4FF0010BB0450CD9617FC4
:101F4000A8EB0600401A0838854219DC09EB0600A8
:101F50000021058041801AE06088617F801B471A5C
:101F6000083F0DD41B2F00DAFFDFBD4201DC2946FC
:101F700000E0B9B2681A0204120C04D0424502DD36
:101F800084F817A0D2E709EB06000180428084F8AC
:101F900017B0CCE770B5044600F12802C088E37D95
:101FA00020F400402BB110440288438813448B4234
:101FB00001D2002070BD00258A4202D301804580F5
:101FC00008E0891A0904090C418003D0A01D00F023
:101FD0001EFB08E0637F00880833184481B26288E2
:101FE000A01DFFF73FFFE575012070BD70B50346EA
:101FF00000F12804C588808820F400462644A842C1
:1020000002D10020188270BD98893588A84206D375
:10201000401B75882D1A2044ADB2C01E05E02C1A55
:10202000A5B25C7F20443044401D0C88AC4200D9EE
:102030000D809C8924B1002414700988198270BD18
:102040000124F9E770B5044600F12801808820F4E6
:1020500000404518208A002825D0A189084480B274
:10206000A08129886A881144814200D2FFDF288834
:10207000698800260844A189884212D1A069807F1E
:102080002871698819B1201D00F0C1FA08E0637F4A
:1020900028880833184481B26288201DFFF7E2FEC9
:1020A000A6812682012070BD2DE9F04141898788F3
:1020B0000026044600F12805B94218D004F10A08A8
:1020C00021F400402844418819B1404600F09FFAAD
:1020D00008E0637F00880833184481B26288404674
:1020E000FFF7C0FE761C6189B6B2B942E8D130462E
:1020F000BDE8F0812DE9F04104460B4627892830E0
